:020000040800F2
:100000000004012001020008950E0008990E000866
:10001000ED0E0008990E0008C10E0008030200084A
:10002000030200080302000803020008C9300008A8
:10003000030200080302000803020008030200088C
:10004000030200080302000803020008030200087C
:10005000030200080302000825330008513300089A
:100060007D330008A9330008D533000803020008D7
:10007000030200080302000803020008030200084C
:10008000030200080302000803020008030200083C
:1000900003020008030200080302000801340008FC
:1000A000030200080302000803020008030200081C
:1000B0004931000803020008030200080302000897
:1000C00003020008030200080302000803020008FC
:1000D00003020008030200080302000803020008EC
:1000E0006934000803020008030200080302000844
:1000F00003020008030200080302000803020008CC
:1001000003020008030200080302000803020008BB
:1001100003020008030200080302000803020008AB
:10012000030200080302000803020008030200089B
:10013000030200080302000803020008030200088B
:10014000030200080302000803020008C927000890
:10015000030200080302000803020008030200086B
:10016000030200080302000803020008030200085B
:10017000030200080302000803020008030200084B
:10018000030200080302000803020008030200083B
:10019000030200080302000803020008030200082B
:1001A000030200080302000803020008030200081B
:1001B000030200080302000803020008030200080B
:1001C00003020008030200080302000803020008FB
:1001D00003020008030200080302000803020008EB
:1001E00003020008030200080302000803020008DB
:1001F00003020008030200080302000803020008CB
:1002000002E000F000F8FEE772B6394880F3088893
:10021000384880F3098838484EF60851CEF200017C
:10022000086040F20000CCF200004EF63471CEF2CD
:1002300000010860BFF34F8FBFF36F8F40F20000E3
:10024000C0F2F0004EF68851CEF200010860BFF314
:100250004F8FBFF36F8F4FF00000E1EE100A4EF6A4
:100260003C71CEF200010860062080F31488BFF3D1
:100270006F8F01F02DFF02F0AFFE4FF055301F4998
:100280001B4A91423CBF41F8040BFAE71C49194A4A
:1002900091423CBF41F8040BFAE71A491A4A1B4B3A
:1002A0009A423EBF51F8040B42F8040BF8E70020D5
:1002B0001749184A91423CBF41F8040BFAE701F094
:1002C0004BFF02F0F3FE144C144DAC4203DA54F829
:1002D000041B8847F9E700F03FF8114C114DAC4280
:1002E00003DA54F8041B8847F9E701F033BF000034
:1002F000000401200024012000000008000001206B
:100300000004012078380008002401205024012036
:10031000502401204830012000020008000200089B
:1003200000020008000200082DE9F04F2DED108AB0
:10033000C1F80CD0D0F80CD0BDEC108ABDE8F08F1D
:10034000002383F311882846A047002001F042FBD8
:1003500001F0EEFA00DFFEE71B4B6FF06E0270B5A6
:100360001A706FF07F0200245A720E225C709C702B
:10037000DC701C715C719C71DC711C729A72DC7295
:1003800001F068FE064601F09DFE054650B90F4B90
:100390009E4217D001339E4241F2883412BF054677
:1003A00000240125002001F05FFE0DB100F0B6F839
:1003B00000F044FD00F03CFC204600F051F900F054
:1003C000ADF8F9E70446EDE750240120010007B03D
:1003D00008B500F0CFFBA0F120035842584108BDFA
:1003E00007B5054B02211B88ADF8043001A800F0C9
:1003F0000FFC03B05DF804FB4C350008064991F88A
:10040000243033B100230822086A81F8243000F038
:1004100033BC0120704700BF702401202DE9F84F44
:10042000234C94F824300546884617468BBB2E464D
:10043000DFF87C90002F38D094F824A0BAF1000F98
:1004400005D12022FF214846266200F0E5FCCAF1D2
:100450000805BD4228BF3D465FFA85FBAD00414619
:100460002A4604EB8A0000F0ADFC94F82430A7EB98
:100470000B079B445FFA8BFBBBF1080F2E44A8448B
:10048000FFB284F824B0D5D1FFF7B8FF0028D1D14E
:1004900008E0266A06EB8306B042C9D0FFF7AEFF3C
:1004A0000028C4D10020BDE8F88F0120BDE8F88FF6
:1004B0007024012010B572B6202383F3118862B630
:1004C0001248C3680BB101F00DFB0023104A0F481E
:1004D0004FF47A7101F0CAFA002383F311880D4CAE
:1004E000236813B12368013B2360636813B1636819
:1004F000013B6360084B1B7833B9636823B9022062
:1005000000F056FC3223636010BD00BF5C24012064
:10051000B5040008A0250120982401202DE9F04110
:10052000454B464953F8042F013201D1BDE8F08113
:100530008B42F7D1424C434B22689A427AD9424BC4
:100540009B6803F1006303F5C0339A4272D2002026
:1005500000F08AFB3D4B0220187000F021FC3C4B60
:100560001A6C00221A64196E1A66196E596C5A6454
:10057000596E5A66596E596941F08001596159693D
:1005800021F0800159615969196941F000511961DF
:10059000196921F0005119611B6972B62D492E4B62
:1005A0000B601D682468BFF34F8FBFF36F8F2B4B19
:1005B000C3F88420BFF34F8F5A6922F480325A6106
:1005C000BFF34F8FD3F88020C2F3C906C2F34E3277
:1005D0005201B70743F6E07E02EA0E08384631467C
:1005E000013948EA000CB1F1FF3FC3F874C200F1D1
:1005F0004040F5D1203A12F1200FEDD1BFF34F8FDB
:10060000BFF36F8FBFF34F8FBFF36F8F5A6922F421
:1006100000325A610022C3F85022BFF34F8FBFF35C
:100620006F8F72B6202383F3118862B6AD4685F3CF
:1006300008882047BDE8F081FC7F01081C80010884
:1006400004800108FF7F0108502401209824012024
:100650000038024008ED00E00080010800ED00E0F5
:100660002DE9F04F99B0B44C01902022FF2110A841
:10067000A66800F0D1FBB14A1378A346B3B9B048DD
:1006800001211170C36072B6202383F3118862B612
:10069000C3680BB101F026FA0023AA4AA8484FF418
:1006A0007A7101F0E3F9002383F31188019B13B100
:1006B000A54B019A1A60A54AA349019F0292002303
:1006C00013704B6099461C461D469846012000F069
:1006D00067FB002F00F012829B4B1B68002B40F041
:1006E0000D8219B0BDE8F08F0220FFF771FE0028DF
:1006F00040F0FB81019BB9F1000F08BF1F46944BEE
:100700001B88ADF82C3002210BA800F081FADDE740
:100710004FF47A7000F02EFA031E0393EADB0220F6
:10072000FFF756FE82460028E4D0039B581E04289B
:1007300000F2DD81DFE800F0030E1114170018A8A5
:10074000052340F8343D042100F062FA54464FF08E
:10075000000856E004217848F6E704217D48F3E7D5
:1007600004217D48F0E71C24204600F07FFA043481
:100770000B9004210BA800F04BFA2C2CF4D1E5E7E8
:10078000002DB7D0002CB5D00220FFF721FE054682
:10079000002800F0AF8101206C4C00F065FA0220C7
:1007A000207000F0FDFA4FF000095FFA89FA504618
:1007B00000F06AFA074658B1504600F075FA09F1A0
:1007C00001090028F1D12C46A9460027634B97E781
:1007D00001230220237000F0D9FA3E46DBF80830EE
:1007E0009E4206D2304600F041FA0130EBD1043689
:1007F000F4E7029B00261E70534BA9465E602C4610
:10080000374600F011FB15B1002C18BF0027FFF789
:10081000E7FD5BE7002D3FF46DAF002C3FF46AAFBE
:10082000029B0220187000F0BBFA322000F0A2F9FF
:10083000B0F1000AC0F25E811AF0030540F05A815F
:10084000DBF8082006EB0A03934200F25381BAF565
:10085000807F00F24F8155450DDA4FF47A7000F039
:1008600089F90490049B002BC0F244813C4A049B0C
:10087000AB540135EFE7C820FFF7AAFD0546002875
:1008800000F038811F2E11D8C6F12004544528BF2E
:10089000544610AB26F0030022463149184400F0BC
:1008A00091FA2246FF212E4800F0B6FA4FEAAA0A32
:1008B0005FFA8AF22A493046FFF7B0FD0446002865
:1008C00000F01A8106EB8A0605469AE70220FFF738
:1008D0007FFD00283FF40EAFFFF790FD00283FF4A6
:1008E00009AF4FF0000A5346DBF8082092451CD2AE
:1008F000BAF11F0F12D8109A01320FD02AF003025A
:1009000018A90A4452F8202C0B92184604220BA96D
:1009100000F000FB0AF1040A0346E5E750460393A2
:1009200000F0A4F9039B0B90EFE718A8042140F80E
:100930004C3D00F06DF964E7502401209C25012016
:100940005C240120B5040008A02501209824012082
:100950004E35000854240120582401205035000849
:100960009C24012018A8002340F8343D642100F0A5
:100970002BF900287FF4BEAE0220FFF729FD0028E6
:100980003FF4B8AE0B9800F0A1F918AB43F8480D4E
:1009900004211846CDE718A8002340F8343D64210F
:1009A00000F012F900287FF4A5AE0220FFF710FD39
:1009B00000283FF49FAE0B9800F096F918AB43F86F
:1009C000440DE5E70220FFF703FD00283FF492AE57
:1009D00000F090F918AB43F8400DD9E70220FFF77B
:1009E000F7FC00283FF486AE0BA9142000F088F92C
:1009F000824618A8042140F83CAD00F009F95146A0
:100A00000BA896E7322000F0B5F8B0F1000AFFF627
:100A100071AE1AF0030F7FF46DAEDBF808200AEB1D
:100A2000080393423FF666AE0220FFF7D1FC002890
:100A30003FF460AE2AF0030AC244D0453FF4E1AE71
:100A4000404600F013F904210A900AA800F0E0F8EB
:100A500008F10408F1E74FF47A70FFF7B9FC0028B9
:100A60003FF448AEFFF7CAFC00283FF4AFAE109B3E
:100A700001330CD0082210A90020FFF7CFFC00287A
:100A80003FF4A4AE2022FF2110A800F0C5F9FFF723
:100A9000A7FC374800F0A6FF23E6002D3FF42AAE5E
:100AA000002C3FF427AE18A8002340F8343D642101
:100AB00000F08AF8824600287FF41CAE0220FFF77F
:100AC00087FC00283FF416AE0390FFF789FC41F243
:100AD000883000F087FF0B9800F0DAF900F0A4F9F5
:100AE000039B57461C461D46F0E5054689E64FF038
:100AF0000008FFE52546FDE52C4667E6002000F0EE
:100B000039F80490049B002BFFF6E3AD012000F0C0
:100B10003DF9049B213B122B3FF6D8AD01A252F8C0
:100B200023F000BFE906000811070008810700084C
:100B3000CD060008CD060008CD06000815080008FF
:100B4000050A0008CD080008650900089709000893
:100B5000C5090008CD060008DD090008CD0600081B
:100B6000570A000803080008CD0600089B0A000881
:100B7000A086010037B5114B1A780132D2B2002499
:100B8000012A01468DF8074011D80D4803681D6AF7
:100B90004FF47A734B4301220DF10701A847012856
:100BA00005D1084B9DF807001C7003B030BD4FF411
:100BB000FA7000F017FF4FF0FF30F6E70024012035
:100BC00070260120AC25012038B50E4B1A78013271
:100BD000D2B2012A05460ED80B4803681C6A4FF4AE
:100BE0007A734B4304222946A047042803D1074BBC
:100BF0000020187038BD4FF4FA7000F0F3FE4FF08B
:100C0000FF3038BD0024012070260120AC250120D2
:100C100030B4054C2368DD69044B0A46AC460146F6
:100C2000204630BC604700BF70260120A08601002E
:100C3000F8B501F013F9094C094E0A4F2070002550
:100C400030682378834207D901F002F933680544FC
:100C50000133BD423360F3D9F8BD00BFAD2501209B
:100C6000A8250120FF7F010001F0A6B900F1006076
:100C700000F5C0300068704700F10060920000F598
:100C8000C03001F031B90000054B1A68054B1B78E4
:100C90009B1A834202D9104401F0DAB80020704751
:100CA000A8250120AD25012038B5074D0446286848
:100CB000204401F0D5F828B928682044BDE8384020
:100CC00001F0E6B838BD00BFA825012010F00303ED
:100CD00008D1B0F5806F05D800F10050A0F5712063
:100CE0000068704700207047014BC058704700BF34
:100CF00020F4F01F014B1868704700BF002004E08B
:100D0000F0B5204B1E68204B1F885D6893F90840A2
:100D1000C6F30B02BA424FEA164622D09F89BA4266
:100D200021D01F8BBA4206D102220C2404FB0233CD
:100D30005D6893F90840B6F5805F16D041F2010373
:100D40009E4208BF5A24421E0A44013D0B4693426C
:100D500015D215F9016F581C4EB1034600F8016C0D
:100D6000F5E70022E1E70122DFE74124EBE72C254C
:100D700082421D7001D9981C5C70401AF0BD184663
:100D8000FBE700BF002004E004240120022802BF8A
:100D9000024B4FF480229A61704700BF000002406E
:100DA000022802BF014B04229A61704700000240F2
:100DB000022801BF024A536983F00403536170475C
:100DC0000000024010B50023934203D0CC5CC45411
:100DD0000133F9E710BD000030B5441E14F9010FCE
:100DE0000B4660B193F90050854201F1010106D133
:100DF0001AB993F90020801A30BD013AEEE7002AB3
:100E0000F7D1104630BD000002460346981A13F988
:100E1000011B0029FAD1704702440346934202D0D5
:100E200003F8011BFAE77047024B1A78024B1A705D
:100E3000704700BFAC2501200024012038B5104DBB
:100E4000104C284600F008F92146284600F030F9F9
:100E500024680D48E26ED2F8043843F00203C2F869
:100E6000043800F0BFFD0949204600F035FAE26E73
:100E7000D2F8043823F00203C2F8043838BD00BFAA
:100E800070260120FC35000840420F00243600087F
:100E900070470000FEE7000000B59BB0EFF309814A
:100EA00068226846FFF78EFFEFF30583034B9A6BCA
:100EB0009A6A9A6A9A6A9A6A9B6AFEE700ED00E06B
:100EC00000B59BB0EFF3098168226846FFF77AFF0F
:100ED000EFF30583044B9A6B9A6A9A6A9A6A9A6A44
:100EE0009A6A9B6AFEE700BF00ED00E000B59BB088
:100EF000EFF3098168226846FFF764FFEFF305838B
:100F0000034B5A6B9A6A9A6A9A6A9A6A9B6AFEE7D4
:100F100000ED00E030B5084D0A4491420BD011F8C5
:100F2000013B09245840013CF7D040F300032B401B
:100F300083EA5000F7E730BD2083B8ED0023044971
:100F40001A465A50C8180833802B4260F9D17047AE
:100F5000B025012072B6202383F3118862B6704752
:100F6000026843681143016003B1184770470000ED
:100F700013B5446BD4F894341A681178042915D148
:100F8000217C022912D11979128901238B40134245
:100F90000CD101A904F14C0001F092FED4F8944464
:100FA000019B21790246206800F0E6F902B010BDED
:100FB000143001F017BE00004FF0FF33143001F081
:100FC00011BE00004C3001F0E7BE00004FF0FF33CF
:100FD0004C3001F0E1BE0000143001F0E7BD00002C
:100FE0004FF0FF31143001F0E1BD00004C3001F052
:100FF000B3BE00004FF0FF324C3001F0ADBE000038
:10100000D0F8942438B5136819780429054601D01E
:10101000012038BD017C0229FAD112795C890120B6
:1010200090400440F4D105F1140001F079FD02462E
:101030000028EDD0D5F894544FF48073286869796E
:1010400000F088F9204638BD406BFFF7D9BF00009B
:1010500000207047704700007FB5124B03600023EB
:1010600043608360C360012502260F4B057404466C
:101070000290019300F18402294600964FF4807398
:10108000143001F029FD094B0193029400964FF4AE
:10109000807304F52372294604F14C0001F0ECFD45
:1010A00004B070BD8035000849100008710F0008B9
:1010B00008B50A68FFF74EFF0B7902EB830318624D
:1010C0004B790D3342F823008B7913B102EB830285
:1010D000106202230374C0F89414002383F3118870
:1010E00008BD000038B5037F044613B190F85430B2
:1010F000ABB9201D01250221FFF732FF04F11400D6
:1011000025776FF0010100F095FC84F8545004F14C
:101110004C006FF00101BDE8384000F08BBC38BDD9
:1011200010B5012104460430FFF71AFF002323778E
:1011300084F8543010BD000038B504460025143042
:1011400001F0E2FC04F14C00257701F0ADFD201D1B
:1011500084F854500121FFF703FF2046BDE83840D2
:10116000FFF74EBF90F85C3003F06003202B19D1DD
:1011700090F85D20212A0AD0222A4FF000030ED0D9
:10118000202A0FD1084A02650722426504E0064B77
:1011900003650723436500238365012070470365CA
:1011A0004365F9E70020704728240120D0F89434E3
:1011B00037B51A681178042904461AD1017C02292E
:1011C00017D11979128901238B40134211D100F1F3
:1011D0004C05284601F026FE58B101A9284601F029
:1011E0006FFDD4F89444019B21790246206800F0F9
:1011F000C3F803B030BD000000EB8103F7B51C6AF3
:1012000005460E46ECB105EB8607FFF7A3FE201D51
:101210000821FFF7A5FEFB685B691B684C3413B11E
:10122000204601F05BFD01A9204601F049FD024680
:1012300048B1019B3146284600F09EF8002383F315
:10124000118803B0F0BDFB685A691268002AF5D016
:101250001B8A013B1340F1D105F15C02EAE7000073
:101260000D3138B550F82140D4B1FFF773FED4F8F2
:1012700094241368527903EB8203DB689B695D68F1
:1012800045B104216018FFF76BFE294604F11400F4
:1012900001F050FC2046FFF7B3FE002383F31188D2
:1012A00038BD00007047000072B6202383F3118818
:1012B00062B6704700F0D6BF01230370002343607D
:1012C00000F1240200F1380142F8043B8A42136124
:1012D000FAD103814381704738B50446FFF7E4FF34
:1012E00000254160C560056145618561C561056294
:1012F00000F0C8FF0223237085F3118838BD000079
:1013000070B500EB810305465069DA600E4614465D
:1013100018B110220021FFF77FFDA06918B110223B
:101320000021FFF779FD31462846BDE8704001F005
:1013300073B80000028902F001020281428902F0C2
:10134000010242810022026142618261C261026245
:1013500001F0F6B8F0B400EB81044789E468012598
:10136000A4698D403D43458123600023A2606360F2
:10137000F0BC01F011B90000F0B400EB8104078962
:10138000E468012564698D403D43058123600023A5
:10139000A2606360F0BC01F08DB9000070B502235B
:1013A000002504460370A0F8645080F8665080F869
:1013B000675005814581C560056145618561C561ED
:1013C000056280F84C5000F0C3FF63681B6823B1CE
:1013D00029462046BDE87040184770BD4368027832
:1013E0001B6880F86820052202700BB104211847A1
:1013F00070470000436890F868201B6802700BB1CA
:10140000052118477047000090F84C3070B504462D
:1014100013B1002380F84C3004F15C02204601F047
:10142000B1F863689B6863BB94F85C5015F0600684
:1014300015D194F85D3005F07F0545EA032540F2AB
:1014400002339D4200F00B8159D8022D00F0D98063
:101450003DD8002D00F08580012D00F0CC800021CA
:10146000204601F0FFFA0021204601F0F1FA6368FE
:101470001B6813B1062120469847062384F84C3098
:1014800070BD204698470028CED094F8632094F889
:10149000623043EA0223626D934238BF636594F978
:1014A0005C30656D002B80F2FC80002D00F0EB803D
:1014B000092384F84C30FFF7F7FE636D226D00219D
:1014C0002046FFF759FF002383F3118870BDB5F55F
:1014D000817F00F0B080B5F5407F49D0B5F5807FC1
:1014E000BDD194F85E30012BB9D1B4F8643023F04B
:1014F0000203A4F8643026656665A665C5E740F278
:1015000001639D421ED8B5F5C06F3BD2B5F5A06F03
:10151000A5D1B4F85C30B3F5A06F0ED194F85E306D
:1015200084F86630204600F06BFF63681B6813B1D7
:101530000121204698470323237000232365636518
:10154000A365A2E7B5F5106F32D040F602439D4285
:1015500051D0B5F5006F82D104F1670323650123F3
:1015600024E004F16403236502236365A5658CE729
:1015700094F85E30012B7FF472AFB4F8643043F01E
:101580000203B6E794F86120616894F860304D6812
:1015900094F85F1043EA0223204694F85E20A8479F
:1015A00000283FF45CAF4368236503686365A4E7E4
:1015B0002378042B0FD1FFF777FE2046FFF7BAFE02
:1015C00086F31188636884F867601B6803212170C3
:1015D0000BB12046984794F85E30002BADD084F8CC
:1015E00067300423237063681B68002BA5D0022199
:1015F00020469847A1E7374B236502236365002304
:101600009EE794F8601011F0800F204601F00F0162
:101610000ED000F0A9FF012806D002287FF41FAFEA
:101620002D4B2365606568E72C4B2365656564E792
:1016300000F08CFFEFE794F85E30002B7FF40FAFE3
:1016400094F8603013F00F013FF477AF1A0620468C
:1016500002D501F01BFA70E701F00EFA6DE794F87D
:101660005E30002B7FF4FBAE94F8603013F00F0176
:101670003FF463AF1B06204602D501F0F3F95CE7A7
:1016800001F0E6F959E7142384F84C30FFF70CFE1B
:101690002B462A4629462046FFF75CFE85F3118833
:1016A00070BD5DB1152384F84C30FFF7FDFD636D0F
:1016B000226D00212046FFF74DFE04E70B2384F83E
:1016C0004C30FFF7F1FD2B462A4629462046FFF70E
:1016D00053FEE3E7B0350008A8350008AC35000834
:1016E00038B590F84C300446152B28D8DFE803F0C5
:1016F0003C27272727273C27270B2837272727275B
:10170000272727273C3C90F8631090F86220436D10
:1017100042EA01229A4213D9C268128AB3FBF2F557
:1017200002FB153565B9FFF7BFFD2B462A46294652
:10173000FFF722FE85F311880A2384F84C3038BD68
:10174000142384F84C30FFF7AFFD00231A461946E6
:101750002046FFF7FFFD002383F3118838BD836D1A
:1017600003B198470023E8E7002101F07BF900214D
:10177000204601F06DF963681B6813B1062120460D
:1017800098470623D9E7000090F84C20152A38B571
:10179000044621D80123934040F6416213421CD1F4
:1017A00013F480150ED19B0216D50B2380F84C3014
:1017B000FFF77AFD2B462A462946FFF7DDFD85F324
:1017C000118838BDC3689B695B682BB9836D03B111
:1017D0009847002384F84C3038BD002101F042F9CD
:1017E0000021204601F034F963681B6813B106211B
:1017F000204698470623EDE7024B00221B605B6002
:101800009A60704730260120002303748268054BDC
:101810001B6899689142FBD25A680360426010606D
:10182000586070473026012008B572B6202383F334
:10183000118862B6037C032B05D0042B0DD02BB985
:1018400083F3118808BD436900221A604FF0FF330B
:101850004361FFF7D9FF0023F2E790E80C001A601C
:1018600002685360F2E70000002303748268054BAE
:101870001B6899689142FBD85A6803604260106007
:101880005860704730260120054B196908741868A4
:1018900002681A605360186101230374FEF744BDA7
:1018A0003026012030B54B1C87B005460A4C10D0BD
:1018B00023690A4A01A800F0D9F82846FFF7E4FF97
:1018C000049B13B101A800F00DF92369586907B012
:1018D00030BDFFF7D9FFF8E73026012029180008AE
:1018E00038B50C4D41612B6981689A689142044674
:1018F00003D8BDE83840FFF787BF1846FFF784FFDD
:1019000001232C61014623742046BDE83840FEF7D0
:101910000BBD00BF30260120044B1A681B6990687C
:101920009B68984294BF0020012070473026012018
:1019300010B5084C236820691A682260546001229F
:1019400023611A74FFF790FF01462069BDE810403B
:10195000FEF7EABC3026012072B6202383F31188FB
:1019600062B670478260022202740022427470479D
:101970008368A3F17C0243F80C2C026943F83C2CE9
:10198000426943F8382C074A43F81C2CC26843F8D4
:10199000102C022203F8082C002203F8072CA3F1D4
:1019A000180070474103000810B5FFF7D5FFFFF797
:1019B000DFFF00210446FFF793FF002383F3118824
:1019C000204610BD024B1B6958610F20FFF75CBF1A
:1019D0003026012008B5FFF7BFFFBDE80840FFF73C
:1019E000F1BF000008B50146FFF7B6FF0820FFF77A
:1019F00059FF002383F3118808BD000049B1064B4D
:101A000042681B6918605A60136043600420FFF746
:101A100049BF4FF0FF3070473026012003689842DD
:101A200006D01A680260506059611846FFF7ECBE94
:101A30007047000038B504460D462068844200D146
:101A400038BD036823605C604561FFF7DDFEF4E7A5
:101A5000054B03F114025A619A614FF0FF32DA61CB
:101A600000221A62704700BF30260120F8B50361DA
:101A70004FF08043C2605C6A194B1A46022952F843
:101A8000145F38BF0221954206461F460AD15861AD
:101A900098611C620560456081600819BDE8F840E6
:101AA00001F0E2B9186AAB68241A0C1902D3E41ADF
:101AB0002D6804E09C4202D2204401F0E3F9AB68B7
:101AC0009C42F4D86B68736035601E606E60B460D1
:101AD000A9684FF0FF33091BA960FB61F8BD00BF87
:101AE0003026012010B41B4C234653F8141F8142AA
:101AF00010D0416802680A60026851609A424FF053
:101B00000001C16003D0936881680B4493605DF865
:101B1000044B70470A68626100209A425360C860B3
:101B200003D15DF8044B01F0A7B9936888680344BA
:101B300093604FF08042206A526A121A9342E6D9AB
:101B4000991A012998BF931C18445DF8044B01F0C1
:101B500099B900BF3026012000207047FEE7000041
:101B6000704700004FF0FF307047000072B620232E
:101B700083F3118862B67047022906D0032906D084
:101B80000129064818BF0020704705487047032AFE
:101B90009ABF044800EBC20000207047803600085E
:101BA000343600083024012070B59AB001AD0646E5
:101BB00008462946144600F091F82846FFF724F914
:101BC000C0B2431C5B0086E81800237003236370D7
:101BD000002302341946DAB2904204F1020401D81B
:101BE0001AB070BDEA5C04F8022C04F8011C013341
:101BF000F1E7000008B5FFF7B9FF0348FFF7D6FA91
:101C0000002383F3118808BD7026012010B5044617
:101C1000052915D8DFE801F015140315151BFFF78A
:101C2000A5FF0E4A0121FFF76BFB20460C4A02215B
:101C3000FFF766FB0B48FFF77FFA002383F3118859
:101C400010BDFFF793FF0748FFF74CFAF5E7FFF7E2
:101C50008DFF0448FFF764FAEFE700BFB4350008D2
:101C6000D83500087026012038B50C4D0C4C0D49B4
:101C70002A4604F10800FFF797FF05F1CA0204F1B4
:101C800010000949FFF790FF05F5CA7204F118002A
:101C90000649BDE83840FFF787BF00BF382B012059
:101CA00030240120043600080E36000819360008DA
:101CB00070B5044608460D46FFF7A6F8C6B22046A2
:101CC000013403780BB9184670BD32462946FFF738
:101CD00083F80028F3D1012070BD00002DE9F84FF2
:101CE00005460C46FFF790F82B49C6B22846FFF789
:101CF000DFFF08B10536F6B228492846FFF7D8FFBE
:101D000008B11036F6B2632E0DD8DFF88C80DFF8FC
:101D10008C90234FDFF890A0DFF890B02E7846B972
:101D20002670BDE8F88F29462046BDE8F84F01F03F
:101D300005BC252E2CD1072241462846FFF74CF83A
:101D400058B9DBF800302360DBF804306360DBF85F
:101D50000830A36007350C34E0E7082249462846DE
:101D6000FFF73AF8A0B90F4BA21C13F8011F09099D
:101D70005345C95D02F8021C197801F00F0102F108
:101D80000202C95D02F8031CEFD118340835C5E71B
:101D9000267001350134C1E7A03600081936000865
:101DA000B53600081FF4F01F2BF4F01FA83600080A
:101DB000BFF34F8F024AD368DB03FCD4704700BFE8
:101DC000003C024008B5074B1B7853B9FFF7F0FF02
:101DD000054B1A69002ABFBF044A5A6002F18832D3
:101DE0005A6008BD962D0120003C02402301674542
:101DF00008B5054B1B7833B9FFF7DAFF034A1369BF
:101E000043F00043136108BD962D0120003C0240C1
:101E1000072870B513D80B4A0B4C137863B90B4ED7
:101E20004FF0006144F8231056F823500133082B7B
:101E30002944F7D10123137054F8200070BD00200D
:101E400070BD00BFB82D0120982D0120C8360008B4
:101E5000014B53F820007047C8360008082070472F
:101E6000072810B5044601D9002010BDFFF7D0FFA8
:101E7000064B53F824301844C21A0BB9012010BD88
:101E800012680132F0D1043BF6E700BFC836000803
:101E9000072810B5044621D8FFF78AFFFFF792FF05
:101EA0000F4AF323D360C300DBB243F4007343F063
:101EB00002031361136943F480331361FFF778FF62
:101EC000FFF7A6FF074B53F8241000F0DDF8FFF7EB
:101ED0008FFF2046BDE81040FFF7C2BF002010BDB5
:101EE000003C0240C83600082DE9F84312F0010317
:101EF000154640D18218B2F1016F3CD22C4B1B68C1
:101F000013F0010337D02B4CFFF75CFFF323E360A2
:101F1000FFF74EFF40F20127032D01D9830713D0AD
:101F2000244C0F46401A40F20118EB1B0B44012BC6
:101F300000EB0706236924D823F001032361FFF790
:101F400057FF0120BDE8F883236923F44073236120
:101F500023693B43236151F8046B0660BFF34F8F45
:101F6000FFF726FF03689E4208D0236923F0010390
:101F70002361FFF73DFF0020BDE8F883043D0430F6
:101F8000CAE723F440732361236943EA080323610A
:101F9000B94637F8023B3380BFF34F8FFFF708FF96
:101FA0003688B9F80030B6B2B342BED0DDE700BF24
:101FB00000380240003C0240084908B50B7828B1BF
:101FC00053B9FFF7FFFE01230B7008BD23B1BDE835
:101FD00008400870FFF70CBF08BD00BF962D012018
:101FE00010B50244064B0439D2B2904200D110BD64
:101FF000441C00B253F8200041F8040FE0B2F4E7AB
:1020000050280040104B30B51C6F240407D41C6FBF
:1020100044F400741C671C6F44F400441C670B4CB0
:10202000236843F4807323600244094B0439D2B21D
:10203000904200D130BD441C00B251F8045F43F817
:102040002050E0B2F4E700BF0038024000700040CA
:102050005028004007B5012201A90020FFF7C0FF6A
:10206000019803B05DF804FB13B50446FFF7F2FFD7
:10207000A04206D002A9012241F8044D0020FFF73A
:10208000C1FF02B010BD00000144BFF34F8F064BEB
:10209000884204D3BFF34F8FBFF36F8F7047C3F8ED
:1020A0005C022030F4E700BF00ED00E0034B1B684A
:1020B0009B0042BF024B01221A70704774380240E5
:1020C000B92D0120014B1878704700BFB92D0120B0
:1020D000F0B5BFF34F8FBFF36F8F1D4B0021C3F8D7
:1020E0005012BFF34F8FBFF36F8F5A6942F4003223
:1020F0005A61BFF34F8FBFF36F8FC3F88410BFF3E4
:102100004F8FD3F88020C2F3C904C2F34E3252017C
:10211000A50743F6E07602EA060E284621464EEA77
:1021200000070139C3F860724F1C00F14040F6D13E
:10213000203A12F1200FEED1BFF34F8F5A6942F4CB
:1021400080325A61BFF34F8FBFF36F8FF0BD00BF76
:1021500000ED00E0FEE70000084A094B09498B4208
:1021600004D3094A0021934205D3704752F8040F63
:1021700043F8040BF3E743F8041BF4E7C438000802
:10218000483001204830012048300120036F30B52D
:1021900000229D68C46E11464FF0FF3004EB4213DD
:1021A00001329542C3F80019C3F81019C3F80809A1
:1021B000C3F8001BC3F8101BC3F8080BEED24FF096
:1021C0000113C4F81C3830BD890141F020010161C0
:1021D00003699B06FCD4122000F0E4BE204B03EB05
:1021E00080022DE9F047D2F80CE0DD6EDEF8142015
:1021F000461CD2F800C005EB063605EB40185168C6
:1022000061450BD3D5F83428012303FA00F022EA04
:102210000000C5F834081846BDE8F087BEF8104045
:10222000ACEB0103A34228BF2346D8F81849A4B257
:10223000B3EB840F10D894681F46A4F1040959F831
:1022400004AFC6F800A0042F01D9043FF7E71C44EF
:102250000B4494605360D2E70020BDE8F08700BFD4
:10226000BC2D012010B5054C2046FFF725F84FF096
:10227000A043E366024B236710BD00BFBC2D0120C5
:102280000C3700080378012B70B5054650D12A4B56
:10229000C46E98421BD1294B5A6B42F080025A639C
:1022A0005A6D42F080025A655A6D5A6942F08002B6
:1022B0005A615A6922F080025A610E2143205B69FB
:1022C00000F0EEFB1E4BE3601E4BC4F80038002309
:1022D000C4F8003EC0232360EE6E4FF40413A363E2
:1022E0003369002BFCDA012333610C2000F05AFE25
:1022F0003369DB07FCD4122000F054FE3369002B55
:10230000FCDA0026A6602846FFF740FF6B68C4F899
:102310001068DB68C4F81468C4F81C684BB90A4B31
:10232000A3614FF0FF336361A36843F00103A3602F
:1023300070BD064BF4E700BFBC2D01200038024001
:102340004014004003002002003C30C0083C30C074
:10235000F8B5C46E054600212046FFF735FF296F0A
:1023600000234FF001128F68C4F834384FF0006634
:10237000C4F81C284FF0FF3004EB431201339F4296
:10238000C2F80069C2F8006BC2F80809C2F8080B6D
:10239000F2D20B68EA6E6B676362102313611669F1
:1023A00016F01006FBD1122000F0FCFDD4F8003826
:1023B00023F4FE63C4F80038A36943F4402343F0D8
:1023C0001003A3610923C4F81038C4F814380A4B69
:1023D000EB604FF0C043C4F8103B084BC4F8003B1F
:1023E000C4F81069C4F800396B6F03F1100243F4AC
:1023F00080136A67A362F8BDE836000840800010C9
:10240000C26E90F86610D2F8003823F4FE6343EAF7
:102410000113C2F8003870472DE9F0410EB200EB0D
:1024200086080D46D8F80C100F6807F00303022B3E
:1024300050D0032B50D03D4A3D4F012B18BF1746BB
:10244000C46E4FEA451E04EB0E030022C3F8102BA6
:102450008A6905F1100C002A40D04A8A05F1580318
:102460005B013A43E2500123D4F81C2803FA0CF331
:102470001343A6444A69C4F81C380023CEF8103927
:1024800005F13F03002A39D00A8A898B9208012975
:1024900088BF4A43416F04EB8303561841EA024266
:1024A000466729465A602046FFF78EFED8F80C3062
:1024B0001B8A43EA85531F4305F148035B01E7503C
:1024C0000123D4F81C2803FA05F51543C4F81C5859
:1024D000BDE8F081174FB3E7174FB1E704EB4613A0
:1024E000D3F8002B22F40042C3F8002BD4F81C28A8
:1024F000012303FA0CF322EA0303BAE704EB830394
:102500000E4A5A6004EB461629462046FFF75CFE49
:10251000D6F8003923F40043C6F80039D4F81C3843
:10252000012202FA05F523EA0505CFE70080001035
:10253000008004100080081000800C1000040002CD
:10254000026F12684267FFF721BE00005831C36E68
:1025500049015B5813F4004004D013F4001F14BF6A
:1025600001200220704700004831C36E49015B58CA
:1025700013F4004004D013F4001F14BF0120022004
:102580007047000000EB8101CB68196A0B6813608B
:102590004B6853607047000000EB810330B5DD6885
:1025A000AA691368D36019B9402B84BF4023136014
:1025B0006B8A1468C26E1C44013CB4FBF3F46343A1
:1025C000033323F0030302EB411043EAC44343F017
:1025D000C043C0F8103B2B6803F00303012B09B282
:1025E0000ED1D2F8083802EB411013F4807FD0F8F6
:1025F000003B14BF43F0805343F00053C0F8003B4E
:1026000002EB4112D2F8003B43F00443C2F8003B16
:1026100030BD00002DE9F041254DEE6E06EB401374
:102620000446D3F8087BC3F8087B38070AD5D6F8E8
:102630001438190706D505EB84032146DB682846C4
:102640005B689847FA0731D5D6F81438DB072DD5E3
:1026500005EB8403D968DCB98B69488A5E68B6FBF0
:10266000F0F200FB12629AB91868DA6890420FD251
:10267000121A83E8140072B6202383F3118862B61D
:102680000B482146FFF788FF84F31188BDE8F081ED
:10269000012303FA04F26B8923EA02036B81CB68FE
:1026A00023B121460248BDE8F0411847BDE8F0815A
:1026B000BC2D012000EB810370B5DD68C36E6C6931
:1026C0002668E6604A0156BB1A444FF40020C2F85F
:1026D00010092A6802F00302012A0AB20ED1D3F8C7
:1026E000080803EB421410F4807FD4F8000914BFEB
:1026F00040F0805040F00050C4F8000903EB421253
:10270000D2F8000940F00440C2F80009D3F83408B8
:10271000012202FA01F10143C3F8341870BD19B95E
:10272000402E84BF4020206020682E8A841940F00B
:102730000050013C1A44B4FBF6F440EAC440C6E73A
:10274000F8B504461F48C56E05EB4413D3F8086975
:10275000C3F80869F10719D5D5F81038DA0715D587
:1027600000EB8403D9684B691F68DA6897421AD274
:10277000D21B00271A605F6072B6202383F3118892
:1027800062B62146FFF796FF87F31188330617D507
:10279000D5F834280123A340134211D02046BDE8C8
:1027A000F840FFF71BBD012303FA04F2038923EA73
:1027B000020303818B68002BE8D021469847E5E7A8
:1027C000F8BD00BFBC2D0120A0482DE9F84FC56E13
:1027D0006E69AB691E4016F4805F6E61044605D0D9
:1027E000FEF7DCFDBDE8F84F00F07EBC002E12DAEB
:1027F000D5F8003E95489B071EBFD5F8003E23F054
:102800000303C5F8003ED5F8043823F00103C5F8EA
:102810000438FEF7EFFD370502D58C48FEF7DEFDE4
:10282000B0040CD5D5F8083813F0060FEB6823F484
:1028300070530CBF43F4105343F4A053EB603107C3
:1028400004D56368DB680BB180489847F2026FD407
:10285000B3020CD5D4F86C80DFF8F0A100274FF05C
:102860000109236F9B68F9B28B4280F09C80F706C8
:1028700019D5E16E0A6AC2F30A1702F00F0302F4D7
:10288000F012B2F5802F00F0B680B2F5402F0AD1D9
:1028900004EB830301F58051DB68186A00231A46B4
:1028A0009F4240F09C803303D5F818481DD5E703BC
:1028B00002D50020FFF7AEFEA50302D50120FFF7E9
:1028C000A9FE600302D50220FFF7A4FE210302D572
:1028D0000320FFF79FFEE20202D50420FFF79AFED5
:1028E000A30202D50520FFF795FE77037FF57AAFA7
:1028F000E60702D50020FFF723FFA50702D5012038
:10290000FFF71EFF600702D50220FFF719FF21071E
:1029100002D50320FFF714FFE20602D50420FFF7DB
:102920000FFFA3067FF55EAF0520FFF709FF59E70C
:10293000D4F86C80DFF814A100274FF00109236F51
:102940009B685FFA87FB5B4582D308EB4B13D3F898
:10295000002902F44022B2F5802F22D1D3F80029B9
:10296000002A1EDAD3F8002942F09042C3F8002969
:10297000D3F80029002AFBDB5946E06EFFF724FC60
:10298000228909FA0BF322EA0303238104EB8B0368
:10299000DB689B6813B15946504698475846FFF785
:1029A0001DFC0137CBE708EB4112D2F8003B03F4E2
:1029B0004023B3F5802F10D1D2F8003B002B0CDA66
:1029C000628909FA01F322EA0303638104EB8103BC
:1029D000DB68DB680BB150469847013741E79C073D
:1029E00008BF0A68072B98BF027003F101039CBF60
:1029F000120A013054E7023304EB830201F58051DF
:102A0000526890690268D0F808C04068A2EB000ED6
:102A10000022104697420AD104EB830463689B6945
:102A20009A683A449A605A6817445F603BE712F02C
:102A3000030F08BF0868964588BF8CF8000002F1B4
:102A4000010284BF000A0CF1010CE3E7BC2D012058
:102A5000C36E03EB4111D1F8003B43F40013C1F8FE
:102A6000003B7047C36E03EB4111D1F8003943F4CA
:102A70000013C1F800397047C36E03EB4111D1F860
:102A8000003B23F40013C1F8003B7047C36E03EB17
:102A90004111D1F8003923F40013C1F8003970470F
:102AA00000F1604300F01F02400903F56143090192
:102AB0008000C9B200F1604083F8001300F5614066
:102AC00001239340C0F880310360704772B6202321
:102AD00083F3118862B6704730B5039C01720433EA
:102AE00004FB0325C361049B03630021059B006075
:102AF0004060C1604261026185610462426281623C
:102B0000C162436330BD00000022416A416101613E
:102B1000C2608262C2626FF00101FEF78BBF0000EB
:102B200003694269934203D1C2680AB10020704729
:102B3000181D704703691960C2680132C260C2691A
:102B4000134482690361934224BF436A03610021F5
:102B5000FEF764BF38B504460D46E3683BB16269D1
:102B6000131D1268A3621344E362002038BD237A68
:102B700033B929462046FEF741FF0028EDDA38BD7B
:102B80006FF00100FBE70000C368C269013BC3604E
:102B90004369134482694361934224BF436A43619A
:102BA00000238362036B03B11847704770B5044676
:102BB000FFF78CFF866A3EB9FFF7CCFF054618B1D8
:102BC00086F31188284670BDA36AE26A13F8015B98
:102BD000A362934202D32046FFF7D6FF002383F37C
:102BE0001188EFE72DE9F04704460E461746984650
:102BF000FFF76CFF0025A946D4F828A0BAF1000F12
:102C000009D141462046FFF7A5FF20B18AF311887C
:102C10002846BDE8F087A16AE36AA7EB050A5B1ABC
:102C20009A4528BF9A46BAF1400F1BD9334601F1A5
:102C3000400251F8040B43F8040B9142F9D1A36A06
:102C400040334036A3624035A26AE36A9A4202D317
:102C50002046FFF799FF89F31188BD42D8D2FFF7CC
:102C600035FFC9E730465246FEF7ACF8A36A534435
:102C70005644A3625544E7E710B5029C0172043341
:102C800003FB0421C36100238362C362039B0363CC
:102C9000049B00604060C460426102618161046223
:102CA0004262436310BD0000026AC260426A426130
:102CB000026100228262C2626FF00101FEF7BABEB9
:102CC000436902699A4203D1C2680AB10020704781
:102CD000184650F8043B0B6070470000C368C26997
:102CE0000133C3604369134482694361934224BF43
:102CF000436A43610021FEF791BE000038B50446E7
:102D00000D46E3683BB123691A1DA262E2691344D0
:102D1000E362002038BD237A33B929462046FEF706
:102D20006DFE0028EDDA38BD6FF00100FBE7000012
:102D300003691960C268013AC260C26913448269BA
:102D40000361934224BF436A036100238362036BE0
:102D500003B118477047000070B504460E46FFF7F0
:102D6000B5FE856A35B91146FFF7C8FF10B185F386
:102D7000118870BDA36A1E70A36AE26A0133934290
:102D8000A36204D3E16920460439FFF7D1FF002094
:102D900080F3118870BD00002DE9F04704460D4610
:102DA00090469946FFF792FE0026B246A76A4FB9B1
:102DB00049462046FFF7A2FF20B187F3118830462D
:102DC000BDE8F087A06AE76AA8EB06033F1A9F42B6
:102DD00028BF1F46402F1BD905F1400355F8042B8F
:102DE00040F8042B9D42F9D1A36A4033A3624036D8
:102DF000A26AE36A9A4204D3E16920460439FFF7E4
:102E000097FF8AF311884645D9D2FFF75FFECDE7D9
:102E100029463A46FDF7D6FFA36A3B443D44A362E8
:102E20003E44E5E7026943699A4203D1C3681BB98E
:102E3000184670470023FBE7836A002BF8D0043B59
:102E40009B1AF5D01360C368013BC360C3691A4481
:102E5000836902619A4224BF436A0361002383624B
:102E60000123E5E700F086B94FF080430022586364
:102E70001A610222DA6070474FF080430022DA6064
:102E8000704700004FF0804358637047FEE7000032
:102E900010B5194CFEF7B0FCFEF7DAFD8022174999
:102EA0002046FEF75FFD012344F8180C0374144B11
:102EB000144AD96821F4E0610904090C0A43124953
:102EC000DA60CA6842F08072CA60104A1049C2F8DB
:102ED000B01F116841F0010111601022DA77202241
:102EE00083F82220002383F3118862B60948BDE8E5
:102EF0001040FEF759BD00BF5826012018370008C2
:102F000000ED00E00003FA05F0ED00E0001000E045
:102F100055CEACC5203700082DE9F84F204C4FF0B6
:102F20000008656904F11407C1464FF08043266A22
:102F30005B6AAA689E1B96421FD34FF0200AAA68BC
:102F4000236AD5F80CB0134423622B68BB425F6040
:102F5000A6EB02066361C5F80C8001D1FFF78CFF78
:102F600089F311882869D84772B68AF3118862B646
:102F70006569AB689E42E2D2D7E76269BA420CD07B
:102F8000916823628E1B9660A86802282CBF1818CF
:102F9000981CBDE8F84FFFF775BFBDE8F88F00BF7C
:102FA00030260120034B59685A68521A9042FBD8C8
:102FB000704700BF001000E04B6843608B6883607F
:102FC000CB68C3600B6943614B6903628B694362E1
:102FD0000B6803607047000008B5274B27481A6943
:102FE00040F2FF710A431A611A6922F4FF6222F06B
:102FF00007021A611A691A6B0A431A631A6D0A43A7
:103000001A651F4A1B6D1146FFF7D6FF1D4802F1D6
:103010001C01FFF7D1FF1C4802F13801FFF7CCFF7C
:103020001A4802F15401FFF7C7FF194802F1700175
:10303000FFF7C2FF174802F18C01FFF7BDFF1648EA
:1030400002F1A801FFF7B8FF144802F1C401FFF72D
:10305000B3FF134802F1E001FFF7AEFF114802F1A0
:10306000FC01FFF7A9FF104802F58C71FFF7A4FFE0
:10307000BDE8084000F0E0B800380240000002401F
:10308000403700080004024000080240000C0240E3
:10309000001002400014024000180240001C0240D0
:1030A00000200240002402400028024008B500F041
:1030B00035FAFFF7EDFEFEF7F9FFBDE80840FEF731
:1030C000D3BD000070470000064A536823F0010397
:1030D0005360EFF30983683383F30988002383F394
:1030E0001188704730EF00E010B572B6202383F3EB
:1030F000118862B6104B5B6813F4006318D0F1EED0
:10310000103AEFF309844FF0807344F84C3C0B4BBA
:10311000DB6844F8083CA4F1680383F30988FEF7F0
:10312000FBFB18B1064B44F8503C10BD054BFAE7C9
:1031300083F3118810BD00BF00ED00E030EF00E028
:1031400051030008540300084FF0804310B51A697A
:1031500092070AD500241C6172B6202383F31188DC
:1031600062B6FFF7D9FE84F31188BDE81040FFF77F
:10317000BBBF0000104B1A6C42F001021A641A6EB9
:1031800042F001021A660D4A1B6E936843F0010378
:1031900093604FF080436B229A624FF0FF32DA6205
:1031A00000229A615A63DA605A6001225A6108214A
:1031B0001A601C20FFF774BC00380240002004E0B5
:1031C0001B4B1A696FEA42526FEA52521A611A692E
:1031D000C2F30A021A614FF0FF301A695A69586146
:1031E00000215A6959615A691A6A62F080521A625A
:1031F0001A6A02F080521A621A6A5A6A58625A6A45
:1032000059625A6A0B4A106840F480701060186F57
:1032100000F44070B0F5007F1EBF4FF48030186797
:103220001967536823F40073536000F057B900BF67
:103230000038024000700040354B4FF080521A6455
:10324000344A4FF4404111601A6842F001021A609A
:103250001A689207FCD59A6822F003029A602C4BF8
:1032600019469A6812F00C02FBD1186800F0F900B8
:1032700018609A601A6842F480321A600B689B03E7
:10328000FCD54B6F43F001034B67214B5A6F9007FE
:10329000FCD5214A5A601A6842F080721A601D4BB0
:1032A0001A4659684904FCD5196841F480311960FF
:1032B0005368D803FCD5136843F400331360154AF0
:1032C00053689903FCD5124B1A689201FCD5134A36
:1032D0009A6040F20112C3F88C200022C3F89020BB
:1032E0000F4A40F2073111609A6842F002029A6078
:1032F000074B9A6802F00C02082AFAD15A6C42F481
:1033000080425A645A6E42F480425A665B6E70473D
:103310000038024000700040086C40090094883872
:10332000003C0240084A08B5536911680B4003F09D
:103330000103536123B1054A13680BB150689847E4
:10334000BDE80840FFF7D0BE003C0140B025012099
:10335000084A08B5536911680B4003F00203536132
:1033600023B1054A93680BB1D0689847BDE808407F
:10337000FFF7BABE003C0140B0250120084A08B55D
:10338000536911680B4003F00403536123B1054AEC
:1033900013690BB150699847BDE80840FFF7A4BE18
:1033A000003C0140B0250120084A08B55369116866
:1033B0000B4003F00803536123B1054A93690BB135
:1033C000D0699847BDE80840FFF78EBE003C014039
:1033D000B0250120084A08B5536911680B4003F075
:1033E0001003536123B1054A136A0BB1506A984721
:1033F000BDE80840FFF778BE003C0140B025012041
:10340000174B10B55C691A68144004F478725A615D
:10341000A30604D5134A936A0BB1D06A9847600695
:1034200004D5104A136B0BB1506B9847210604D595
:103430000C4A936B0BB1D06B9847E20504D5094A4F
:10344000136C0BB1506C9847A30504D5054A936CD7
:103450000BB1D06C9847BDE81040FFF745BE00BFE8
:10346000003C0140B02501201A4B10B55C691A6878
:10347000144004F47C425A61620504D5164A136D67
:103480000BB1506D9847230504D5134A936D0BB1CA
:10349000D06D9847E00404D50F4A136E0BB1506EFF
:1034A0009847A10404D50C4A936E0BB1D06E98478F
:1034B000620404D5084A136F0BB1506F9847230478
:1034C00004D5054A936F0BB1D06F9847BDE8104003
:1034D000FFF70ABE003C0140B0250120062108B5D7
:1034E0000846FFF7DDFA06210720FFF7D9FA062183
:1034F0000820FFF7D5FA06210920FFF7D1FA0621A7
:103500000A20FFF7CDFA06211720FFF7C9FA062196
:103510002820BDE80840FFF7C3BA000008B5FFF750
:103520004FFEFDF70BFDFDF7C5FEFDF793FDFFF721
:10353000C9FDBDE80840FFF795BC0000034611F83F
:10354000012B03F8012B002AF9D170471210121336
:103550001211000053544D3332463F3F3F3F3F3F2F
:103560000053544D333246375B347C355D7800531D
:10357000544D333246375B367C375D7800000000AF
:1035800000000000CD0F0008B90F0008F50F00087B
:10359000E10F0008ED0F0008D90F0008C50F000863
:1035A000B10F0008511000080000000001000000E9
:1035B000000000000200000000000000F9110008F7
:1035C0006112000840004000082B0120182B012048
:1035D00002000000000000000300000000000000E6
:1035E000A51200080000000010000000282B012098
:1035F000000000000100000000000000BC2D0120C0
:10360000010102004172647550696C6F74002542BB
:103610004F415244252D424C002553455249414CBF
:10362000250000000D1C0008791B0008651100082A
:10363000F51B0008430000003C3600080902430067
:10364000020100C032090400000102020100052449
:1036500000100105240100010424020205240600D3
:1036600001070582030800FF09040100020A0000A7
:10367000000705010240000007058102400000002C
:1036800012000000883600081201100102000040FC
:10369000091241570002010203010000040309045A
:1036A00025424F41524425004B616B757465463786
:1036B0004D696E690030313233343536373839412F
:1036C00042434445460000000080000000800000A6
:1036D00000800000008000000000020000000400E4
:1036E00000000400000004000000000009140008AD
:1036F000E11600088917000840004000342E012020
:10370000342E012001000000442E01208000000022
:1037100040010000050000006D61696E00000000BE
:1037200038370008502E01204830012001000000E9
:103730008D2E00080000000069646C650000000028
:103740001001802A00000000AAAAAAAA0001000015
:10375000FBFF00000000000000A00A0000000001C4
:1037600000000000AAAAAAAA00000001FFFF0000B2
:103770000000000000000000000000000000000049
:10378000AAAAAAAA00000000FFFF00000000000093
:10379000000000000000004000000000AAAAAAAA41
:1037A00000000080FF7F000000000000000000001B
:1037B0000001000000000000AAAAAAAA000100005F
:1037C000FFFF0000000000000000000000000000FB
:1037D00000000000AAAAAAAA00000000FFFF000043
:1037E00000000000000000000000000000000000D9
:1037F000AAAAAAAA00000000FFFF00000000000023
:103800000000000000000000000000000A000000AE
:1038100000000000030000000000000000000000A5
:103820000000000000000000000000000000000098
:103830000000000000000000000000000000000088
:103840000000000000000000000000000000000078
:103850000000000000000000000000000000000068
:103860000000000000000000000000000000000058
:103870000000000000000000FF0000000000000049
:10388000543500083F00000049040000613500087D
:103890003F000000510400006F3500083F000000A9
:1038A0000096000000000800040000009C3600089C
:1038B0000000000000000000000000000000000008
:1038C0000000000000000000FFFFFFFFFFFFFFFF00
:1038D000FFFFFFFFFFFFFFFFFFFFFFFFFFFFFFFFF8
:1038E000FFFFFFFFFFFFFFFFFFFFFFFFFFFFFFFFE8
:1038F000FFFFFFFFFFFFFFFFFFFFFFFFFFFFFFFFD8
:10390000FFFFFFFFFFFFFFFFFFFFFFFFFFFFFFFFC7
:020000040801F1
:1080000000060120A99201082D3A070889390708BE
:10801000F539070889390708C1390708AB92010803
:10802000AB920108AB920108AB9201089D1A0908B6
:10803000AB920108AB920108AB920108AB92010828
:10804000AB920108AB920108AB920108AB92010818
:10805000AB920108AB920108A5270908CD270908B2
:10806000F52709081D280908452809080DD808081A
:1080700035D8080861D808088DD80808B9D8080884
:10808000E1D808080DD908088DD70808AB92010877
:10809000AB920108AB920108AB9201086D28090868
:1080A000B9290908BD290908D1290908D5290908CC
:1080B000D9290908E9290908FD2909087DDE0808E8
:1080C000A1DF0808AB920108AB920108AB9201084E
:1080D000AB920108412909085529090869290908AD
:1080E000D1280908AB920108AB920108252A09089A
:1080F000292A09083D2A0908412A090839D9080806
:10810000AB920108AB920108112A0908AB92010851
:108110007D290908AB920108AB920108AB920108D6
:1081200065D908088DD90808B9D90808E5D908081B
:1081300011DA0808AB920108AB920108AB92010872
:10814000AB920108AB920108AB920108B122090879
:1081500039DA080865DA080891DA08089129090867
:10816000AB920108AB920108AB920108AB920108F7
:10817000AB920108AB920108AB920108AB920108E7
:10818000AB920108AB920108A5290908AB9201083E
:10819000AB920108AB920108AB920108AB920108C7
:1081A000AB920108AB920108AB920108AB920108B7
:1081B000AB920108AB920108AB920108AB920108A7
:1081C000AB920108AB920108AB920108AB92010897
:1081D000AB920108AB920108AB920108AB92010887
:1081E000AB920108AB920108AB920108AB92010877
:1081F000AB920108AB920108AB920108AB92010867
:1082000099A50108192D02081D79030841FC0408ED
:10821000E1180508C56A05080974050851770508BD
:10822000ADDF0508ADE4050869FC0508AD75060875
:10823000F532070859CD07085D530808657A080824
:10824000D590080849C108081DC70808FFFFFFFFAF
:1082500081F0004102E000BF83F0004330B54FEAF7
:1082600041044FEA430594EA050F08BF90EA020F64
:108270001FBF54EA000C55EA020C7FEA645C7FEAF7
:10828000655C00F0E2804FEA5454D4EB5555B8BF1A
:108290006D420CDD2C4480EA020281EA030382EA8B
:1082A000000083EA010180EA020281EA0303362D1D
:1082B00088BF30BD11F0004F4FEA01314FF4801CF0
:1082C0004CEA113102D0404261EB410113F0004F02
:1082D0004FEA03334CEA133302D0524263EB4303B9
:1082E00094EA050F00F0A780A4F10104D5F1200E57
:1082F0000DDB02FA0EFC22FA05F2801841F10001B2
:1083000003FA0EF2801843FA05F359410EE0A5F185
:1083100020050EF1200E012A03FA0EFC28BF4CF0B6
:10832000020C43FA05F3C01851EBE37101F000456C
:1083300007D54FF0000EDCF1000C7EEB00006EEB79
:108340000101B1F5801F1BD3B1F5001F0CD3490803
:108350005FEA30004FEA3C0C04F101044FEA44525A
:1083600012F5800F80F09A80BCF1004F08BF5FEAE1
:10837000500C50F1000041EB045141EA050130BDC1
:108380005FEA4C0C404141EB0101013C28BFB1F5D3
:10839000801FE9D291F0000F04BF01460020B1FA1E
:1083A00081F308BF2033A3F10B03B3F120020CDAF1
:1083B0000C3208DD02F1140CC2F10C0201FA0CF0CF
:1083C00021FA02F10CE002F11402D8BFC2F1200C34
:1083D00001FA02F120FA0CFCDCBF41EA0C019040EA
:1083E000E41AA2BF01EB0451294330BD6FEA040433
:1083F0001F3C1CDA0C340EDC04F11404C4F120021E
:1084000020FA04F001FA02F340EA030021FA04F32F
:1084100045EA030130BDC4F10C04C4F1200220FA86
:1084200002F001FA04F340EA0300294630BD21FAC4
:1084300004F0294630BD94F0000F83F4801306BF8A
:1084400081F480110134013D4EE77FEA645C18BF7E
:108450007FEA655C29D094EA050F08BF90EA020F15
:1084600005D054EA000C04BF1946104630BD91EA0D
:10847000030F1EBF0021002030BD5FEA545C05D110
:108480004000494128BF41F0004130BD14F580044F
:108490003CBF01F5801130BD01F0004545F0FE41C3
:1084A00041F470014FF0000030BD7FEA645C1ABFF8
:1084B000194610467FEA655C1CBF0B46024650EA2F
:1084C000013406BF52EA033591EA030F41F400215B
:1084D00030BD00BF90F0000F04BF0021704730B5E1
:1084E0004FF4806404F132044FF000054FF00001B6
:1084F00050E700BF90F0000F04BF0021704730B577
:108500004FF4806404F1320410F0004548BF40424B
:108510004FF000013EE700BF42004FEAE2014FEAA0
:1085200031014FEA02701FBF12F07F4393F07F4F7B
:1085300081F06051704732F07F4208BF704793F07E
:108540007F4F04BF41F40021704730B54FF4607491
:1085500001F0004521F000411CE700BF50EA010294
:1085600008BF704730B54FF000050AE050EA01023D
:1085700008BF704730B511F0004502D5404261EBAD
:1085800041014FF4806404F132045FEA915C3FF4EE
:10859000D8AE4FF003025FEADC0C18BF03325FEA8B
:1085A000DC0C18BF033202EBDC02C2F1200300FA3C
:1085B00003FC20FA02F001FA03FE40EA0E0021FA61
:1085C00002F11444BDE600BF70B54FF0FF0C4CF44F
:1085D000E06C1CEA11541DBF1CEA135594EA0C0F01
:1085E00095EA0C0F00F0DEF82C4481EA030621EA3C
:1085F0004C5123EA4C5350EA013518BF52EA033577
:1086000041F4801143F4801338D0A0FB02CE4FF028
:108610000005E1FB02E506F00042E0FB03E54FF058
:108620000006E1FB03569CF0000F18BF4EF0010E50
:10863000A4F1FF04B6F5007F64F5407404D25FEA4C
:108640004E0E6D4146EB060642EAC62141EA5551FF
:108650004FEAC52040EA5E504FEACE2EB4F1FD0C41
:1086600088BFBCF5E06F1ED8BEF1004F08BF5FEABF
:10867000500E50F1000041EB045170BD06F0004671
:1086800046EA010140EA020081EA0301B4EB5C041E
:10869000C2BFD4EB0C0541EA045170BD41F4801116
:1086A0004FF0000E013C00F3AB8014F1360FDEBF3B
:1086B000002001F0004170BDC4F10004203C35DA17
:1086C0000C341BDC04F11404C4F1200500FA05F39A
:1086D00020FA04F001FA05F240EA020001F000423B
:1086E00021F0004110EBD37021FA04F642EB0601B1
:1086F0005EEA430E08BF20EAD37070BDC4F10C04DB
:10870000C4F1200500FA04F320FA05F001FA04F29E
:1087100040EA020001F0004110EBD37041F100018A
:108720005EEA430E08BF20EAD37070BDC4F1200595
:1087300000FA05F24EEA020E20FA04F301FA05F2FD
:1087400043EA020321FA04F001F0004121FA04F2A5
:1087500020EA020000EBD3705EEA430E08BF20EA75
:10876000D37070BD94F0000F0FD101F000464000AF
:1087700041EB010111F4801F08BF013CF7D041EA31
:10878000060195F0000F18BF704703F00046520035
:1087900043EB030313F4801F08BF013DF7D043EA06
:1087A0000603704794EA0C0F0CEA135518BF95EABC
:1087B0000C0F0CD050EA410618BF52EA4306D1D143
:1087C00081EA030101F000414FF0000070BD50EA62
:1087D000410606BF1046194652EA430619D094EAEC
:1087E0000C0F02D150EA013613D195EA0C0F05D1D6
:1087F00052EA03361CBF104619460AD181EA03012A
:1088000001F0004141F0FE4141F470014FF00000E1
:1088100070BD41F0FE4141F4780170BD70B54FF07C
:10882000FF0C4CF4E06C1CEA11541DBF1CEA1355FC
:1088300094EA0C0F95EA0C0F00F0A7F8A4EB0504DE
:1088400081EA030E52EA03354FEA013100F08880D5
:108850004FEA03334FF0805545EA131343EA12639E
:108860004FEA022245EA111545EA10654FEA002653
:108870000EF000419D4208BF964244F1FD0404F50C
:10888000407402D25B084FEA3202B61A65EB030568
:108890005B084FEA32024FF480104FF4002CB6EB25
:1088A000020E75EB030E22BFB61A754640EA0C00A5
:1088B0005B084FEA3202B6EB020E75EB030E22BFE5
:1088C000B61A754640EA5C005B084FEA3202B6EB26
:1088D000020E75EB030E22BFB61A754640EA9C00E5
:1088E0005B084FEA3202B6EB020E75EB030E22BFB5
:1088F000B61A754640EADC0055EA060E18D04FEA73
:10890000051545EA16754FEA06164FEAC30343EA12
:1089100052734FEAC2025FEA1C1CC0D111F4801FDF
:108920000BD141EA00014FF000004FF0004CB6E7D8
:1089300011F4801F04BF01430020B4F1FD0C88BF77
:10894000BCF5E06F3FF6AFAEB5EB030C04BFB6EB82
:10895000020C5FEA500C50F1000041EB045170BD75
:108960000EF0004E4EEA113114EB5C04C2BFD4EBA2
:108970000C0541EA045170BD41F480114FF0000E26
:10898000013C90E645EA060E8DE60CEA135594EAA2
:108990000C0F08BF95EA0C0F3FF43BAF94EA0C0FA5
:1089A0000AD150EA01347FF434AF95EA0C0F7FF41A
:1089B00025AF104619462CE795EA0C0F06D152EA6E
:1089C00003353FF4FDAE1046194622E750EA410652
:1089D00018BF52EA43067FF4C5AE50EA41047FF463
:1089E0000DAF52EA43057FF4EBAE12E74FF0FF3CC8
:1089F00006E000BF4FF0010C02E000BF4FF0010C99
:108A00004DF804CD4FEA410C7FEA6C5C4FEA430C11
:108A100018BF7FEA6C5C1BD001B050EA410C0CBF60
:108A200052EA430C91EA030F02BF90EA020F0020C2
:108A3000704710F1000F91EA030F58BF994208BF29
:108A400090422CBFD8176FEAE37040F001007047E6
:108A50004FEA410C7FEA6C5C02D150EA013C07D13D
:108A60004FEA430C7FEA6C5CD6D152EA033CD3D088
:108A70005DF8040B704700BF8446104662468C4682
:108A80001946634600E000BF01B5FFF7B7FF0028B5
:108A900048BF10F1000F01BD4DF808EDFFF7F4FFDE
:108AA0000CBF012000205DF808FB00BF4DF808ED69
:108AB000FFF7EAFF34BF012000205DF808FB00BF8C
:108AC0004DF808EDFFF7E0FF94BF012000205DF8AE
:108AD00008FB00BF4DF808EDFFF7CEFF94BF012063
:108AE00000205DF808FB00BF4DF808EDFFF7C4FF5C
:108AF00034BF012000205DF808FB00BF4FEA410CA5
:108B00007FEA6C5C02D150EA013C0AD14FEA430C87
:108B10007FEA6C5C02D152EA033C02D14FF00000C4
:108B200070474FF0010070474FEA410212F5001202
:108B300015D211D56FF47873B3EB625212D94FEAA4
:108B4000C12343F0004343EA505311F0004F23FA8E
:108B500002F018BF404270474FF00000704750EAE3
:108B6000013005D111F0004008BF6FF000407047A0
:108B70004FF00000704700BF4A0011D212F50012FA
:108B800011D20DD56FF47873B3EB62520ED44FEA65
:108B9000C12343F0004343EA505323FA02F07047E5
:108BA0004FF00000704750EA013002D14FF0FF3023
:108BB00070474FF0000070474FEA4102B2F1E043C6
:108BC00024BFB3F5001CDCF1FE5C0DD901F0004CB4
:108BD0004FEAC0024CEA5070B2F1004F40EB830004
:108BE00008BF20F00100704711F0804F21D113F130
:108BF0003872BCBF01F00040704741F480114FEA69
:108C00005252C2F11802C2F1200C10FA0CF320FAF1
:108C100002F018BF40F001004FEAC1234FEAD3230E
:108C200003FA0CFC40EA0C0023FA02F34FEA430378
:108C3000CCE77FEA625307D150EA01331EBF4FF001
:108C4000FE4040F44000704701F0004040F0FE401C
:108C500040F40000704700BF80F0004002E000BF19
:108C600081F0004142001FBF5FEA410392EA030F17
:108C70007FEA226C7FEA236C6AD04FEA1262D2EB61
:108C80001363C1BFD218414048404140B8BF5B4266
:108C9000192B88BF704710F0004F40F4000020F0FF
:108CA0007F4018BF404211F0004F41F4000121F015
:108CB0007F4118BF494292EA030F3FD0A2F101025F
:108CC00041FA03FC10EB0C00C3F1200301FA03F19D
:108CD00000F0004302D5494260EB4000B0F5000FC0
:108CE00013D3B0F1807F06D340084FEA310102F17F
:108CF0000102FE2A51D2B1F1004F40EBC25008BF31
:108D000020F0010040EA03007047490040EB0000FA
:108D1000013A28BFB0F5000FEDD2B0FA80FCACF1FB
:108D2000080CB2EB0C0200FA0CF0AABF00EBC25028
:108D300052421843BCBFD0401843704792F0000F16
:108D400081F4000106BF80F400000132013BB5E769
:108D50004FEA41037FEA226C18BF7FEA236C21D0DF
:108D600092EA030F04D092F0000F08BF0846704744
:108D700090EA010F1CBF0020704712F07F4F04D112
:108D8000400028BF40F00040704712F100723CBF25
:108D900000F50000704700F0004343F0FE4040F44F
:108DA000000070477FEA226216BF08467FEA23630D
:108DB0000146420206BF5FEA412390EA010F40F4F8
:108DC000800070474FF0000304E000BF10F0004344
:108DD00048BF40425FEA000C08BF704743F096432B
:108DE00001464FF000001CE050EA010208BF704746
:108DF0004FF000030AE000BF50EA010208BF7047CD
:108E000011F0004302D5404261EB41015FEA010CE1
:108E100002BF84460146002043F0B64308BFA3F1D9
:108E20008053A3F50003BCFA8CF2083AA3EBC253BB
:108E300010DB01FA02FC634400FA02FCC2F12002DA
:108E4000BCF1004F20FA02F243EB020008BF20F011
:108E50000100704702F1200201FA02FCC2F1200277
:108E600050EA4C0021FA02F243EB020008BF20EA6C
:108E7000DC7070477BB972B90029BEBF00204FF08B
:108E8000004106E008BF00281CBF6FF000414FF012
:108E9000FF3000F007BAADF1080C6DE904CE0029EF
:108EA00009DB002B1ADB00F095F8DDF804E0DDE9C2
:108EB000022304B07047404261EB4101002B1BDBF1
:108EC00000F088F8DDF804E0DDE9022304B0404258
:108ED00061EB4101524263EB43037047524263EB43
:108EE000430300F077F8DDF804E0DDE9022304B085
:108EF000404261EB41017047524263EB430300F093
:108F000069F8DDF804E0DDE9022304B0524263EBC6
:108F10004303704753B94AB9002908BF00281CBF52
:108F20004FF0FF314FF0FF3000F0BCB9ADF1080C4D
:108F30006DE904CE00F04EF8DDF804E0DDE902232F
:108F400004B07047430803F05533C01A830803F098
:108F5000333300F03330184400EB101000F00F30C2
:108F600000EB002000EB0040000E704707EE900A77
:108F7000F5EEC07AF1EE10FA01D400F00BB8F1EE84
:108F8000677A08B517EE900A00F004F8404261EBEA
:108F9000410108BDD0B5FFF7BFFA0C4B00220646D1
:108FA0000F46FFF711FBFFF7E7FD0446FFF792FAC4
:108FB000074B0022FFF708FB02460B4630463946B6
:108FC000FFF74AF9FFF7D8FD2146D0BD0000F03D7C
:108FD0000000F0412DE9F047089D04468E46002B25
:108FE0004DD18A42944669D9B2FA82F252B101FA5D
:108FF00002F3C2F1200120FA01F10CFA02FC41EA6D
:10900000030E94404FEA1C48210CBEFBF8F61FFAF1
:109010008CF708FB16E341EA034306FB07F199428C
:109020000AD91CEB030306F1FF3080F01F8199423F
:1090300040F21C81023E63445B1AA4B2B3FBF8F019
:1090400008FB103344EA034400FB07F7A7420AD9A0
:109050001CEB040400F1FF3380F00A81A74240F2C8
:1090600007816444023840EA0640E41B00261DB133
:10907000D4400023C5E900433146BDE8F0878B4268
:1090800009D9002D00F0EF800026C5E90001304627
:109090003146BDE8F087B3FA83F6002E4AD18B4201
:1090A00002D3824200F2F980841A61EB03030120AB
:1090B0009E46002DE0D0C5E9004EDDE702B9FFDE97
:1090C000B2FA82F2002A40F09280A1EB0C014FEA42
:1090D0001C471FFA8CFE0126200CB1FBF7F307FB9F
:1090E000131140EA01410EFB03F0884208D91CEB42
:1090F000010103F1FF3802D2884200F2CB804346DF
:10910000091AA4B2B1FBF7F007FB101144EA0144BD
:109110000EFB00FEA64508D91CEB040400F1FF314C
:1091200002D2A64500F2BB800846A4EB0E0440EA3A
:1091300003409CE7C6F12007B34022FA07FC4CEA43
:10914000030C20FA07F401FA06F31C43F9404FEA36
:109150001C4900FA06F3B1FBF9F8200C1FFA8CFE4B
:1091600009FB181140EA014108FB0EF0884202FA9F
:1091700006F20BD91CEB010108F1FF3A80F0888060
:10918000884240F28580A8F102086144091AA4B21D
:10919000B1FBF9F009FB101144EA014100FB0EFE9E
:1091A0008E4508D91CEB010100F1FF346CD28E45CD
:1091B0006AD90238614440EA0840A0FB0294A1EB5E
:1091C0000E01A142C846A64656D353D05DB1B3EBBB
:1091D000080261EB0E0101FA07F722FA06F3F140EB
:1091E0001F43C5E9007100263146BDE8F087C2F192
:1091F0002003D8400CFA02FC21FA03F3914001430A
:109200004FEA1C471FFA8CFEB3FBF7F007FB103642
:109210000B0C43EA064300FB0EF69E4204FA02F4EE
:1092200008D91CEB030300F1FF382FD29E422DD941
:10923000023863449B1B89B2B3FBF7F607FB163376
:1092400041EA034106FB0EF38B4208D91CEB0101F6
:1092500006F1FF3816D28B4214D9023E6144C91A76
:1092600046EA004638E72E46284605E70646E3E686
:109270001846F8E64B45A9D2B9EB020864EB0C0E90
:109280000138A3E74646EAE7204694E74046D1E79F
:10929000D0467BE7023B614432E7304609E764444D
:1092A000023842E7704700BF02E000F000F8FEE736
:1092B00072B6374880F30888364880F30988364804
:1092C0003649086040F20000CCF200004EF63471DE
:1092D000CEF200010860BFF34F8FBFF36F8F40F2F3
:1092E0000000C0F2F0004EF68851CEF20001086096
:1092F000BFF34F8FBFF36F8F4FF00000E1EE100A06
:109300004EF63C71CEF200010860062080F314880E
:10931000BFF36F8F78F026FC79F084FE4FF0553064
:109320001F491B4A91423CBF41F8040BFAE71D4913
:10933000184A91423CBF41F8040BFAE71A491B4A0C
:109340001B4B9A423EBF51F8040B42F8040BF8E75E
:1093500000201849184A91423CBF41F8040BFAE733
:1093600078F03EFC79F0BEFE144C154DAC4203DAA9
:1093700054F8041B8847F9E701F0FEF8114C124D30
:10938000AC4203DA54F8041B8847F9E778F026BCAE
:1093900000060120002201200080010808ED00E005
:1093A0000000012000060120081A0B0800220120FD
:1093B000E4250120E8250120001E0220008201088A
:1093C0004C8201084C8201084C8201082DE9F04FC3
:1093D0002DED108AC1F80CD0D0F80CD0BDEC108A5D
:1093E000BDE8F08F002383F311882846A0470020B2
:1093F00077F006FBFEE777F05DF900DFFEE700009F
:1094000001F0FF01102A2BDB10F0070F08D010F835
:10941000013B013A8B422DD010F0070F42B3F6D139
:10942000F0B441EA012141EA014122F007047FF052
:1094300000070023F0E80256083C85EA010586EAA9
:10944000010685FA47F5A3FA87F586FA47F6A5FAE5
:1094500087F68EB9EED1F0BC01F0FF0102F00702F1
:1094600032B110F8013B013A83EA010313B1F8D19C
:109470000020704701387047002D06BF354603387D
:10948000073815F0010F07D1013015F4807F02BFB6
:10949000013015F4C03F0130F0BC0138704700BF07
:1094A00010F8012B11F8013B012A28BF9A42F7D08E
:1094B000D01A7047034613F8012B002AFBD1181A63
:1094C0000138704738B50022002304460D46FFF7E7
:1094D000EDFA28B920462946BDE8384000F00AB820
:1094E000204605F1004100F005F8404261EB4101E2
:1094F00038BD00BFD0B50C4B002206460F46FFF723
:1095000063F8FFF739FB0446FEF7E4FF074B002240
:10951000FFF75AF802460B4630463946FEF79CFEE6
:10952000FFF72AFB2146D0BD0000F03D0000F041CE
:10953000036800221B6818470120704737B5019166
:109540002021044658F0E0F8D0B10E4B93F95613A1
:10955000A1B1B3F95813D3F8F03A019AB3F90C500A
:1095600001F10A039D4203DD40F28D33994205DC8F
:109570002046054B202158F0CDF8002003B030BD27
:109580000120FBE7F04501204C9E090808B505F0D5
:109590008DFDBDE80840012104F0C6BE2DE9F04371
:1095A0008FB00E46054605F081FD002780462E222D
:1095B000394602A801977CF0C7FA322301AA39463E
:1095C000404605F05BF8044648B9184A01AB3146FD
:1095D000284658F08FFA20460FB0BDE8F083DFF838
:1095E0005890D9F8680703689B6898470028F2D01C
:1095F000A9F5405003F0C8FC814630B90C4A314609
:10960000284658F077FA4C46E5E76946404604F0AC
:109610007DFE0028DFD09DF801305B06DBD5054AD2
:109620003146284658F066FA3C46D4E7609E090861
:10963000699E0908809E0908F055012008B5064B6F
:1096400093F8293D9B0704D5044A58F053FA0020AB
:1096500008BD0120FCE700BFF0450120909E0908ED
:1096600070B50C4C0546D4F868070368DB680E46F5
:10967000984710B10124204670BDA4F5405003F076
:109680009FFC04460028F5D1034A3146284658F08D
:1096900031FAF0E7F0550120A09E09082DE970434A
:1096A000274BD3F82C3D1D7B814688465DB9254B61
:1096B0001B68986A03685B6B984738B9224A414631
:1096C000484658F017FA2846BDE8708344F0E8FE93
:1096D000202145F04FFE38B144F0E2FE1F2145F055
:1096E00049FE08B1194AEAE7484658F005F838B982
:1096F000D9F80030414648465B6BBDE870431847D7
:1097000041464846FFF71AFF41460646484658F08C
:1097100053FE20210640484657F0F6FF4146484692
:10972000FFF78CFFF5B2054041464846FFF798FF2A
:1097300041460540484659F003F80540C3E700BFDD
:10974000F0450120605E0120B49E0908CB9E090807
:1097500008B5FFF7A3FF054A92F8181D60F3410111
:1097600082F8181D024A907108BD00BFF045012023
:109770000D5F01202DE9F04106460F4657F0FAFF34
:10978000044668B30221304657F0BEFF40B305F0EF
:109790008DFC4FF48071804604F0C6FD0546F8B993
:1097A0004FF40071404604F0BFFDC8B10E4859F0B7
:1097B000E3F90E4BD3EDA47AF8EEE77A30EE670AC0
:1097C000DFED0B7AB0EEC00AB4EEE70AF1EE10FA64
:1097D00006DD084B3A460221304657F09BFF2C46E7
:1097E0002046BDE8F08100BF78590120F0550120E6
:1097F0000000C842E89E0908F8B504460F4658F034
:1098000007FA10210546204657F07EFF58B1204642
:10981000FFF7BCFE064630B9044B3A4610212046FD
:1098200057F078FF35462846F8BD00BFFC9E090872
:1098300070B505460E4657F0E1FE044678B180212A
:10984000284657F061FF50B1094B93F88D3243B170
:10985000084B32468021284657F05CFF0024204602
:1098600070BD31462846BDE8704058F097BB00BF38
:10987000F0550120109F09082DE9F04180460E4661
:10988000FFF78CFE1A4F044610B90024FC710AE061
:10989000184D05F54053D3F8680703689B6898474F
:1098A00020B90123FB712046BDE8F0810821404624
:1098B00057F02AFF0028F4D095F8E433B02202FBD9
:1098C000035305F50055B3F8EE21B5F954339A4228
:1098D00006DD094B32460821404657F01BFFD4E70E
:1098E0003146404658F036F80028DAD1CDE700BFBF
:1098F0000D5F0120F0250120249F090858F04CBC81
:1099000070B505460E46FFF749FE084B0446D87170
:1099100031462846FFF7A4FE31460028284608BFF6
:10992000002458F0D3FD204070BD00BF0D5F012022
:109930002DE9F843414F3B788146002B7BD1404CC9
:10994000D4F82C5D2D7B01263E701DB13B7028465E
:10995000BDE8F88358F0B2FF054630B9394A38708F
:10996000137843F001031370F1E7DFF8F48039F066
:1099700047FE314638F06AFF88F804600B2632F063
:109980000BFE013E32F0A6FD16F0FF06F7D12E4980
:10999000484658F0A9FE05F089FBD0F80C22C4F81F
:1099A0003C2D90F89432DA0733D404F0D5FE39F028
:1099B00027FE3C2139F060FD04F6245300221A6092
:1099C000224B1B68D86A036801211B689847D4F8AA
:1099D0002C2D137B1BB90123137388F8043039F045
:1099E0000FFE94F81D2D94F81C1D39F01FF937F067
:1099F000DDF836F007FC00233B705AF04BF8144BAF
:109A0000C3F85C0794F8193D43F0200384F8193D2E
:109A10009DE79B07D4D431460E4802F06DF90E48FD
:109A200059F0AAF8DFED0D7A20EE270A04F6245348
:109A300083ED000AC4E7002589E700BFE82501207F
:109A4000F04501202C5F0120349F0908605E012051
:109A5000F0550120F0250120785901200AD7233C38
:109A60000D5F01202DE9F043364DD5F82C3D1B7BD1
:109A700087B006460C46002B61D000294BD021460A
:109A8000304658F0D3FF0446002853D02E493046C4
:109A900058F02AFE05F00AFB074609F001FF804650
:109AA000384604F0A9F8D8B198F92430022B17D120
:109AB00000264FF00009F1B203AA38460191CDF813
:109AC0000C90CDF81090CDF8149004F073FC01992F
:109AD00018B103AA404609F0EFFB0136032EEAD184
:109AE000D5F82C2D137B1BB100231373174A137168
:109AF00039F086FD002138F0A9FE154B1B68D86AA5
:109B0000036800211B68984795F8193D6FF34513CA
:109B100085F8193D0FE005F580530192D3F86807E9
:109B20000368DB689847019A0028A8D195F8183D8A
:109B3000DB06A4D40024204607B0BDE8F08301244E
:109B4000F9E700BFF0450120449F09080D5F01209F
:109B5000605E012008B500F5005090F8183DC3F391
:109B600080028A420BD061F3820380F8183D31B144
:109B700039F046FDBDE808400F2139F07DBC08BD35
:109B800010B500F500520C4692F8293D03F0010192
:109B9000A14209D064F3000382F8293DDB0704D415
:109BA00002F0EEFA024B9C7210BD02F097FBF9E74F
:109BB0000D5F012000F5005090F8293D61F341034D
:109BC00080F8293D014B1973704700BF0D5F0120DC
:109BD0000020704700207047002070470020704729
:109BE0000020704700207047002070470020704719
:109BF0000020704700207047002070470020704709
:109C0000704700007047000000F50D502430704789
:109C10000048704720C9090800F5005090F81C0D55
:109C200070470000034808601C21117008221A6068
:109C3000704700BF10A2090836F004BF16F070BECE
:109C400038F082BF44F036B842F0EEB902F0B8BA4C
:109C500002F0ECB902F018B932F03CBC48F01EBA80
:109C600044F0E6BA11F0F4BC02F034B802F0E4BCFF
:109C700002F0A6B902F036BC02F0B0BF17F06CB922
:109C800003F0B2B902F0D0BA02F082BB70B51F4B3C
:109C9000036000F500530446D3F8AC0C1C4AC3F82B
:109CA000542B08B109F04AF81A4B236004F580538D
:109CB00093F84C2F42B9D3F8485F2DB1284615F0E0
:109CC00041FC284609F036F804F589500C3057F06D
:109CD0002FF804F58750103046F020FC04F6C445F8
:109CE00004F66446B54204D0183D284615F060F8E5
:109CF000F8E7094BC4F8983804F694103BF0D8FC08
:109D000004F510603BF0D4FC204670BD4CA409085B
:109D10002C770A08EC560A08942C0A0838B5474BE9
:109D2000044640F8043B46F08FFD04F1100008F0B3
:109D3000EFFB04F1680036F013FC04F5907010F0AE
:109D400023F904F5866007F0EBF904F2545009F0AA
:109D500029F804F6980016F08DFC04F5446046F0EE
:109D6000FBFC04F5516036F019F904F58150183008
:109D700038F0BCFC04F58750103046F0B7FB04F512
:109D800089500C3056F0C0FF04F58A50083036F088
:109D9000A3FF04F591501C3047F004FF04F58053F5
:109DA00004F593520025104683F86052244B10307E
:109DB0001A6032F015FA294604F5965003F00EFCAD
:109DC00004F5CA5018304FF021FE04F5EE501C3057
:109DD00054F016F804F5F750143056F0EFF804F587
:109DE000FA50183056F024FD04F5FD50103007F0FD
:109DF00095F804F50450103050F096FA04F506502A
:109E000010304CF05DFE04F50A50203045F0FCFFA8
:109E100004F5005304F50C5083F80853094D203025
:109E200057F04AFB2B6813B1074859F003FE204650
:109E3000064935F063F92C60204638BDEC560A0817
:109E4000D0690120E05F0120989F090824560A0884
:109E500010B502F09BFF44F023FB0368BDE81040FF
:109E60005B681847FFF7F4BF38B500F53555044671
:109E7000284608F027FA09F013FD90F92130D3B1F4
:109E800090F84033BBB12846002107F0E1FFDFED39
:109E90000A7A04F2AC7393ED287A20EE270ADFEDFC
:109EA000077AA7EE270A04F2545083ED280ABDE88A
:109EB000384009F005BC38BDCDCCCC3D6666663F68
:109EC000FFF7D2BF10B50121044603F0B1F810B17D
:109ED000204601F0D9F84FF48051204603F0A8F84D
:109EE00020B12046BDE8104001F090B810BD000040
:109EF000FFF7E8BF38B50221044603F099F838B1FE
:109F00000121204603F094F810B9204601F0BCF876
:109F10000221204603F08CF858B3204601F0C2F825
:109F20004021204603F084F868B104F581551835C6
:109F3000284637F061FF04F5805393F9F03013B1F0
:109F4000284638F0A3F84FF48061204603F070F8FB
:109F500020B104F58150183037F0F0FF8021204601
:109F600003F066F860B118F039F8BDE8384016F033
:109F700095B90121204603F05BF80028CDD1CFE749
:109F80004FF48021204603F053F80028EBD14FF422
:109F90000021204603F04CF80028E4D138BD000031
:109FA000FFF7A8BF10B50121044603F041F810B136
:109FB000204601F077F88021204603F039F828B1D7
:109FC00018F00CF8BDE8104016F044B910BD0000C0
:109FD000FFF7E8BF38B54FF6FF71044603F028F8E5
:109FE00004F5005528B1D5F8182D0721204601F0B9
:109FF00061F845F033FE45F057FC95F8183D074AE7
:10A0000083F01003C3F30013537136F0CFFD36F025
:10A0100021FABDE8384002484FF004B80D5F012036
:10A02000645C0120FFF7D6BFF0B52DED028B00F583
:10A0300096549FB005460121204604F0BDFF05F56A
:10A040004A513031204604F021FE05F54B510831CC
:10A05000204603F0E5FE05F5B05104F54B701031D4
:10A060001AF066FD05F5405405F54B50D4F8B022C2
:10A07000D4F8B43284EDB50A1CA91C301C921D938F
:10A080003BF036F805F54A5105F54C503831203093
:10A09000B0EE608AF0EE408A3AF0C2FE05F54B5110
:10A0A00005F54D501431C4EDAF8A84EDB08A84EDCE
:10A0B000B10A14303AF0B4FE84EDB60A39F0A0FAD1
:10A0C000054659F0EFFC2B4B074618680E46FEF785
:10A0D00023FACDE91801D4F8D002FEF71DFACDE934
:10A0E0001601D4F8CC02FEF717FACDE91401D4F822
:10A0F000C802FEF711FACDE91201D4F8D802FEF732
:10A100000BFACDE91001D4F8D402FEF705FACDE937
:10A110000E01D4F8C402FEF7FFF9CDE90C01D4F822
:10A12000B802FEF7F9F9CDE90A01D4F8C002FEF74A
:10A13000F3F9CDE90801D4F8B402FEF7EDF9CDE961
:10A140000601D4F8BC02FEF7E7F9CDE90401D4F822
:10A15000B002FEF7E1F9CDE90076CDE90201064B48
:10A16000064A0749284638F0BDFF1FB0BDEC028BF8
:10A17000F0BD00BFC83A0120AC9F0908BA9F09088A
:10A18000E79F0908FFF750BF10B5044602F088FEAC
:10A190001021204602F04CFF28B117F01FFFBDE848
:10A1A000104016F049B910BDFFF7EEBF00F5805022
:10A1B00000F5A56300F23450D3ED005AD0ED006AEB
:10A1C000D1ED017A91ED006A26EEE77A67EEA57A85
:10A1D000A6EE257AE6EE267A81ED007AC1ED017AC7
:10A1E0007047000000F5805000F5A56300F2345080
:10A1F000D3ED005AD0ED006AD1ED017A91ED006AFD
:10A2000027EEA67A67EEA57AA6EE257AE6EE667ABE
:10A2100081ED007AC1ED017A704700002DE9F0412F
:10A220002DED028B054686B0FFF778FDB94B2B600C
:10A2300005F50E50183005F5005401F01FFC05F52A
:10A240000D531C3305F52C56C4F8F83A062384F850
:10A25000FC3A304657F0DEF904AFAF4BC4F8003B90
:10A260003946301D4FF0010805F52D568DF8108048
:10A27000143635F05FFDA94BC4F8543B06F10800D5
:10A2800058F066FD1E23C4F8B03C0023A4F8B43C8B
:10A2900084F8A88C4FF4E16008F04AFDC4F8AC0CD7
:10A2A00005F53250383058F053FD05F533503C3049
:10A2B00058F04EFD9A4B1A6802B91E6099499FEDFD
:10A2C0009A8A304634F01AFF984BC4F8543B05F58F
:10A2D00034500123A4F81C3D1E3058F0E1FB944B90
:10A2E0000593944B0495009397E80C004FF400718C
:10A2F00005F5355007F0E2FC05F54A5003A9F7EEE5
:10A30000008A1430CDED038A3AF0F6FA05F54A508A
:10A31000203008F0E3F905F540549FED872A84EDDD
:10A32000AC8A05F59653B0EE083A05F54E50C4F8E0
:10A33000A033F0EE432AF0EE420AB0EE430AF0EE0C
:10A34000481AB0EE481A84EDAD8A84EDAE8A84EDE9
:10A35000AF8A84EDB08A84EDB18A84EDB28A84ED4F
:10A36000B38A84EDB48A84EDC08A84EDC18A84ED19
:10A37000C28A84EDC38A84EDC48A84EDC58A84EDE3
:10A38000C68A84EDC78A84EDE28A84EDE38A84ED8F
:10A39000E48A84EDE58A84EDE68A84EDE78A243058
:10A3A0004EF0E6FFB0EE083A05F55150F0EE432AC4
:10A3B000B0EE682AF0EE481AB0EE481AF7EE080A36
:10A3C000B1EE0C0A18304FF081F9B0EE083A05F5FD
:10A3D0005350F0EE432AB0EE430A9FED572ADFEDCB
:10A3E000570AF0EE481AB0EE481A10304FF06EF9E6
:10A3F000B0EE083A05F55550F0EE432A9FED502A8D
:10A40000DFED500AF0EE481AB0EE481AB0EE680AD6
:10A4100008304EF0ADFFB0EE083A05F55750F0EEBB
:10A42000432A9FED490AB0EE482AF0EE481AB0EEF2
:10A43000481AF0EE480A3C304FF048F9F0EE083A7E
:10A4400005F559509FED410AB0EE485AF0EE684AC2
:10A45000B0EE484AB0EE633AF0EE632AB0EE002A5E
:10A46000F0EE481AB0EE481AF6EE000A34304EF01C
:10A4700089FD374B3748186005F55D5224320023BB
:10A4800014279EB207FB06010133097C0029F8D18D
:10A49000314B1E80314B196811B1314859F0CAFA5D
:10A4A00005F55D502C30C4F868071A6002F07EF89C
:10A4B0002C4BC4F86C3705F55E501C3002F076F872
:10A4C000294BC4F89C3705F55F500C3002F06EF84C
:10A4D000264BC4F8CC3705F55F503C3002F066F8E7
:10A4E000234BC4F8FC3705F5605004F62C0383EDCC
:10A4F000008A83ED018A83ED028A3C3002F056F82F
:10A500001C4BC4F83C38284606B0BDEC028BBDE8B5
:10A51000F08100BF4CA40908609F09082C770A0845
:10A52000006301202C730A08000000000CA5090834
:10A53000899C010840A40908CDCC4C3ECDCCCC3E32
:10A54000CDCCCC3DCDCC4C3D3333333F9A99993F64
:10A55000A85F0120A8DA0908A45F0120645F012038
:10A56000EC9F0908F0E3090830E30908A4E40908AE
:10A5700090E3090840E4090838B5054B1C682368D6
:10A580000A461D68034B01462046A847002038BDF7
:10A59000605E0120F025012010B558F0A7FE064CA2
:10A5A000064B18602046FFF739FE2046044A05494D
:10A5B000BDE8104078F0C2BDF0250120605E0120AA
:10A5C00064C301208D9C010810B504460180024936
:10A5D00034F094FD204610BDD4A4090810B5002322
:10A5E0004FF07C52274C03654FF07E51C0F880300D
:10A5F000C0F89030C0F8A030C0F8C0304365C0F853
:10A600008430C0F89430C0F8A430C0F8C4308366F9
:10A610008367C0F89830C0F8A830C0F8B830C36677
:10A62000C367C0F89C30C0F8AC30C0F8BC304FF005
:10A630003F430267C0F8B0204267C0F8B420C0F8BA
:10A640008820C0F8C820C0F88C2001664466846564
:10A65000C165C0F8CC304FF47A71212045F0ACF8D8
:10A660004FF47A71222045F0A7F84FF47A71232035
:10A6700045F0A2F8BDE810404FF47A71242045F06F
:10A680009BB800BF000080BFF8B52DED068B037BA3
:10A69000044643B90023C0F8D430C0F8D830C0F81D
:10A6A000E030C0F8DC30D4ED371A94ED381AD4ED30
:10A6B000360A94ED350A8548DFED858A00F03AFCCC
:10A6C0005820B7EE001AFFEE000A94ED350A18F094
:10A6D00047F9592084ED350AB7EE001AFFEE000A5B
:10A6E00094ED360A18F03CF95A2084ED360AB7EE9C
:10A6F000001AFFEE000A94ED380A18F031F95B20D9
:10A7000084ED380AB7EE001AFFEE000A94ED370A1E
:10A7100018F026F984ED370A59F0B2F907EE900ADD
:10A720009FED6C7AF8EE677A04F1100567EE877A90
:10A730002126C4ED027A2F46F7EE009A94ED35AA51
:10A74000D5ED100AB0EE680A6AEE200A78F0A2FE93
:10A7500094ED368AD5ED140AB0EE409A68EE200AE0
:10A76000B0EE680A78F096FED4ED385AD5ED186A46
:10A7700094ED376A95ED1C7A65EEA66A79EE007A5B
:10A78000F0EEE66A26EE077A77EEA67AB0EEC77AA2
:10A7900077EE877AB5EEC09AE5EC017A95ED235A0B
:10A7A000C5ED079A28EE058A95ED1F5AAAEE058A8F
:10A7B00095ED275AA5EE858AD5ED2B5AA6EE258A6A
:10A7C000F1EE10FACCBF01230023B5EEC00A85EDEF
:10A7D000038AF1EE10FA84F8D030C8BF94F8D03074
:10A7E000F5EEC06AC4BF013384F8D030F1EE10FA40
:10A7F000C8BF94F8D030B5EEC07AC4BF013384F836
:10A80000D030F1EE10FAC2BF94F8D030013384F8A2
:10A81000D03094F9D030002BC1BF07EE103AB8EE1B
:10A82000C77AC8EE076AC5ED036A95ED038AB0EEF4
:10A83000C87A77EE877AF4EEE97AF1EE10FAC4BFBF
:10A8400079EEC77A45ED017A94F9E83015ED019A71
:10A8500083B1DFED217AB4EEE79AF1EE10FA09D870
:10A86000DFED1E7AB4EEE77AF1EE10FAA4BF4FF0F6
:10A870008043EB6194ED390AD5ED077A20EE270A83
:10A88000D4ED027A20EE270ADFED157A30EE000AC9
:10A8900020EE270A78F078FDA9EE008A30B2013662
:10A8A0009FED100A85ED0B8A28EE000AB6B244F03F
:10A8B0005FFF252E7FF442AFBDEC068B04F1200232
:10A8C00039460248BDE8F84000F066BBF02501209B
:10A8D00000000000BD3786359A99193FCDCCCC3E9B
:10A8E000DB0F494000007A440022C0F8D420C0F8B1
:10A8F000D820C0F8E020C0F8DC20FFF7C5BE00007B
:10A9000000207047002070470120704790F82C30DD
:10A910008B4286BF0C3150F82100002070470000A8
:10A9200090F82C308B4286BF0C3150F8210000206B
:10A9300070470000FA207047D0E9083242F4E05234
:10A940004262826A43F4F84342F4E0528262036254
:10A9500070470000014802F085BB00BFF0250120D0
:10A9600013B54FF45870019108F0DCF9044620B19A
:10A97000019942F075FA024B2360204602B010BDE7
:10A9800054A5090870470000704700000020704778
:10A9900070470000002070477047000070470000BB
:10A9A0000320704708207047064BD3F82C3D3BB17D
:10A9B0001B7B002B0CBF5020D02040F001007047C3
:10A9C0005020FAE7F0450120704700007047000072
:10A9D00010B52DED028B174BD3F82C4D3CB3D4EDB5
:10A9E000360A94ED380AF0EEE00AB0EEC00A78F0CC
:10A9F00051FDD4ED370AB0EE408A94ED350AF0EE01
:10AA0000E00AB0EEC00A78F045FDF0EE400AB0EE84
:10AA1000480A78F03FFDDFED087A20EE270ABDEE08
:10AA2000C00A10EE103A18B2BDEC028B10BD2046E1
:10AA3000FAE700BFF04501200000C8423DF074BBBA
:10AA400010B504463EF07CFD054802F00BFB054ABC
:10AA5000034606212046BDE810403EF059BD00BF28
:10AA6000F025012040A509083DF024BE08B50846A0
:10AA700007F01EFF00280CBF0420002008BD0000C6
:10AA8000162A01D03DF088BB03220A7001207047CE
:10AA900041F09CBC08B53DF025FD40F41C6040F041
:10AAA0000D0008BD10B5044608F044F9204610BD5D
:10AAB00008B5094B93F8182DD2060BD403F5805333
:10AAC000D3F868070368DB6A984700280CBF0220A8
:10AAD000042008BD0120FCE7F0450120044B187854
:10AAE00020B9044B93F8190DC0F38010704700BFD4
:10AAF000B85E0120F04501201FB5002301930293A9
:10AB0000039304F0D3FA01A904F09CF828B101A83A
:10AB10001AF090FB05B05DF804FB10F0D7FD90F83B
:10AB2000C432B02202FB030090ED2F0AF2E70000CE
:10AB30000C4B93F88D228AB9A3F5805393F8292DF5
:10AB400051070BD193F8182DD20609D493F8193D6B
:10AB500013F0020F14BF0420012070470520704736
:10AB600003207047F05501202DE9F04F354F97F83D
:10AB70001C3D012B8DB0044652D9334EDFF8E8A0BE
:10AB8000082516F9018BB7F9703308F1FF3B43FA3A
:10AB90000BF3D90740D5207C3BF0EEFD8146207CAD
:10ABA0003CF0B4FD00F12103994505D2207C0DB0A5
:10ABB000BDE8F04F3DF012BABBF1070F2CD8DFE82B
:10ABC0000BF03E04323436383A3C204B1869596950
:10ABD0005A6AD3F804B0D3F818E0D3F80CC0D3ED18
:10ABE000007A1B6ACDF82520CDF829306222212376
:10ABF000CDE9003207900891207CCDED037A19232E
:10AC000003AAC221CDF810B0CDF814E0CDF818C0D9
:10AC10008DF824803BF01AFE013D15F0FF05B0D100
:10AC20000DB0BDE8F08F0A4BD0E70A4BCEE70A4BD8
:10AC3000CCE70A4BCAE75346C8E7094BC6E7094BBE
:10AC4000C4E700BFF045012018A60908005A0120FA
:10AC5000785A0120F05A0120785B0120A45B012082
:10AC6000F85C0120D45901201C5C0120084BD3F86A
:10AC70009C23920701D43DF081BA03F5805393EDF4
:10AC8000A90ADFED047AB8EEC00A20EE270A704761
:10AC9000F04501200AD7233C10B594B0044603A820
:10ACA00007F01CFD1A4BD3F86807036803A95B6B18
:10ACB000984750B3247C58F0EDFE059BDDED047AF7
:10ACC0000893069B09930023F8EEE77A9FED117A2B
:10ACD0000B930C930D930E930F9310931193129368
:10ACE0004FF6F853ADF84C300023962267EE877A82
:10ACF0008DF84E303323CDE90032079007AA572153
:10AD00002046CDED0A7A3BF0A1FD14B010BD00BF86
:10AD1000F05501200AD7233CF0B5254D0E460746D5
:10AD20000FCD95B003AC0FC42B682360731EDBB24C
:10AD3000042B29D814AA02EB830353F8445C2B6834
:10AD400028461B6A98472B6804469B6A2846984702
:10AD5000002305223D7C089009938DF828208DF86A
:10AD600029608DF82A3094B9232221460DF12B0059
:10AD70007AF0EAFE86222E23CDE9003240F2B311AA
:10AD800008AA28463BF062FD052015B0F0BD20461C
:10AD90000DF12B0304F1200250F8041B43F8041BAF
:10ADA0009042F9D102881A8082789A70E2E700BF57
:10ADB0005C9D0908014802F053B900BFF02501204D
:10ADC000014B93F81C0D7047F0450120024B93F89E
:10ADD000190DC0F340007047F045012030B52DED4E
:10ADE000028B154B91ED018A0546D3F8680703687D
:10ADF00085B0DB690C46984728B9BDEEC88A18EEC5
:10AE0000103ADB0712D5D4E9040117F059FF68B1F5
:10AE1000684607F063FC6A462146284641F0FCF983
:10AE200020B10649684607F04FFD00B1022005B089
:10AE3000BDEC028B30BD00BFF055012090580120C1
:10AE40008B8B162B05D0C02B01D1FFF7C7BF42F06B
:10AE500037BC00207047000030B52DED028B8DB05F
:10AE60000023054603930493059304F01FF903A9F7
:10AE700003F0E8FE58B304F019F900F5607393E8A5
:10AE8000070006AC84E80700DDED060A9DED070A21
:10AE90002D7CF1EE600AB1EE400A78F097FC204676
:10AEA000B0EE408A1AF0C6F9DFED0B7A089B0B93DF
:10AEB000012228EE278A0C23CDE90032A82109AA15
:10AEC00028468DED098A8DED0A0A3BF0BFFC0DB0D6
:10AED000BDEC028B30BD00BFE02E6542242938B5A1
:10AEE000054605D040290DD0BDE8384041F034BDBD
:10AEF0000C213DF085F8044610B12846FFF7ACFF61
:10AF0000204638BD0124FBE708B591ED007AF6EE46
:10AF1000007AB4EEE77AF1EE10FA06DD0448012279
:10AF20000521FEF79FFD002008BD0420FCE700BFBF
:10AF3000F05001202DE9F04188B080461B2200210D
:10AF400001A810EE107A10EE906A11EE105A11EE70
:10AF5000904A7AF0F9FDA3238DF8043095238DF8FB
:10AF600005300B238DF8063058F09CFDCDF8070016
:10AF700008F58150CDF80B101B2201A91830CDF82F
:10AF80000F70CDF81360CDF81750CDF81B4037F097
:10AF900075FC08B0BDE8F08170B58CB00D46144664
:10AFA00006462B22002101A87AF0CEFDA3238DF8BE
:10AFB000043095238DF805300C238DF8063058F0B9
:10AFC00071FD2B68CDF80F302368CDF813306B6816
:10AFD000CDF817306368CDF81B30AB68CDF81F3063
:10AFE000A368CDF80700CDF8233006F58150EB6853
:10AFF000CDF80B10CDF827302B22E368CDF82B309D
:10B0000001A9183037F03AFC0CB070BD70B500F5EE
:10B010008154183400F54E56054606F16402204668
:10B020000E2137F0EBFA06F1900220460F2137F09F
:10B03000E5FA05F5525220460832102137F0DEFAC3
:10B0400005F5555605F554522046112137F0D6FA2C
:10B0500006F1480220466C2137F0D0FA06F174025E
:10B0600020466D2137F0CAFA05F5585220462C3299
:10B070000D2137F0C3FA05F55C5220460832BDE8D1
:10B080007040692137F0BABA1FB5002301A900F555
:10B09000965001930293039302F09EF905B05DF878
:10B0A00004FB000008B504F001F8BDE8084003F017
:10B0B00015BD00007FB50E464FF6FF7104461546DC
:10B0C00001F0B6FFE8B11022002168467AF03CFD9D
:10B0D000A3238DF8003095238DF8013004238DF8DB
:10B0E000023058F0DFFCCDF8030004F58150CDF8B4
:10B0F00007101022694618308DF80B60039537F061
:10B100003DFC04B070BD0000A120704738B5044676
:10B1100000F5815501F0A6FF183502460B49284677
:10B1200037F048FD04F50053284693F81D2D93F899
:10B130001C1D37F07BFD04F5965004F06FF904F503
:10B140009070BDE838400FF025BB00BF40A509084E
:10B1500037B5069D044600B92C7801B9697802B963
:10B16000AA7803B9EB78002064F3070061F30F209D
:10B1700062F3174063F31F6003B030BD2DE9F04F59
:10B180002DED0C8B9DB0E04C0D93D4ED379ADFED97
:10B19000DF5A90ED006A04F50054F7EE006AD4F827
:10B1A0002C3DD3ED367A93ED387AF0EEE77AB0EEB7
:10B1B000C77A77EE877A9246F4EEE67AF1EE10FAE5
:10B1C000C8BF86EEA78A06460F46DFEDD17AD8BF04
:10B1D000B0EE668A28EE277AA6EE257A80ED007A10
:10B1E000D4F82C3D93ED357A93ED376AB0EEC77AFB
:10B1F000B0EEC66A37EE067AB4EEE67AF1EE10FAF1
:10B20000CCBFC6EE878AF7EE008A90ED017A68EE31
:10B21000A77AE7EE257AC0ED017A38F0F1F9054614
:10B2200058F040FC814618EE900A8846FDF774F904
:10B23000CDE9080118EE100AFDF76EF9CDE9060117
:10B240007068FDF769F9CDE904013068FDF764F92C
:10B25000B04BB14ACDE90201CDE900982846AF498B
:10B26000AF4D37F03FFFAF4995ED00AA384619F0D2
:10B27000CDFB8DED160A9AED000ACDED170A30EEE2
:10B280004A0A8DED181A17F057FB9DED167AD4ED8A
:10B29000E47AB0EEC77AB4EEE77AA5F59B63F1EEF7
:10B2A00010FA0C9300F10F82D4F82C3D1B7B002B7D
:10B2B00000F00982B4F88E93C9F340099DED177A26
:10B2C000B0EEC77AF4EEC77AF1EE10FA00F3FE8121
:10B2D000D4F82C3D1B7B002B00F0F881B4F88E33A2
:10B2E00003F001039DED187A0B93B0EEC77AF4EEEC
:10B2F000C77AF1EE10FA00F3EB81D4F82C3D1B7BFA
:10B30000002B00F0E581B4F88E33C3F38008B0EE73
:10B31000C00AF4EEC07AF1EE10FA00F3DC81D4F842
:10B320002C3D1B7B002B00F0D681B4F88E33C3F389
:10B33000C00B0DAB00930B999FED7B8A5B46424699
:10B340004846FFF705FFC3B20BEE103AC0F30723E0
:10B350000AEE903AC0F307430CEE903A030E0DEE5E
:10B36000103A9DF834300F90002B40F0B7819DF8D3
:10B370003530002B40F0B281F8EE4B7A694ACDEDC2
:10B38000197AF8EE6A7AB0EE690ACDED1A7AF8EE1B
:10B390006C7A19AB394602F52070CDED1B7A4EF070
:10B3A00073F98DED140ACDED150AB0EE409AF0EE6A
:10B3B000608A9DF836305D4C002B40F094811CEE85
:10B3C000901AD4EDB40A97ED020AB0EE691A04F2AD
:10B3D000FC504EF077FAB0EE40CA9DF83730002BA3
:10B3E00040F084819AED000A30EE4A0A17F0A4FA80
:10B3F0001DEE101A4E48F0EE690A4DF079FF04F583
:10B40000E163DAF800201A6004F20C73F0EE40BA3F
:10B4100083ED00AA474D95EDDD1A4720F1EE410A74
:10B42000B0EE490A17F09CFA95EDDD1AB0EE40AA8D
:10B43000F1EE410A4820B0EE680A17F091FA95ED56
:10B44000DE1AB0EE409AF1EE410A4920B0EE4C0A05
:10B4500017F086FA95EDDF1AF0EE408A4A20B0EE3A
:10B460006B0AF1EE410A17F07BFA96ED007AD6ED01
:10B47000017A9DF834308DED148A6AEE076AF0EE99
:10B4800040BACDED106A69EE276A8DED158ACDEDD3
:10B49000116AD4EDAF6A27EE267AD4EDB06A8DED4D
:10B4A000127A67EEA67ACDED137AB3B99DF83530EE
:10B4B0009BB9B8EE4BBAF8EE6AAAB0EE690A1E481C
:10B4C0008DED19BA19AB12AA10A9CDED1AAA4DF03B
:10B4D000C7FF8DED140ACDED150A9DF83630002B0F
:10B4E00040F0078196ED000AD4EDB10A134860EEF2
:10B4F000200A1CEE901A28EE800AB0EE691A4EF06F
:10B50000E1F9F0EE40AA1BE0F0250120A4707D3F98
:10B5100000D7233C85AB090898D70908B1D709089B
:10B52000C83A0120B858012000000000F055012061
:10B53000645C0120F045012094590120485A012003
:10B54000844814A9FEF74EFE9DF83730002B40F0DA
:10B55000D38096ED010AD4EDB60A7F4860EE200A4A
:10B56000B0EE691A1DEE101A20EE2B0A4EF0AAF961
:10B57000F0EE409AD5F82C3D1B7B7BBB19A9774890
:10B580008DED198A8DED1A8A4EF094F89FED740AAC
:10B5900074484EF0B3F99FED720A73484DF0D4FE33
:10B5A00019A972488DED198A8DED1A8A4EF082F82C
:10B5B0009FED6B0A6E484EF0A1F967489FED680A4F
:10B5C0004EF09CF904F5327393E807000C9B87E872
:10B5D000070003F59B631B68CAF80030B9F1000F40
:10B5E00000F08D80D5F82C3D83ED368A0B9B002B27
:10B5F00000F09080D5F82C3D83ED358AB8F1000F2E
:10B6000000F09380D5F82C3D83ED388ABBF1000F14
:10B6100000F09580D5F82C3D83ED378A9FED558A53
:10B620009FED4F4AD4EDAF2A94EDB21AD7ED000A40
:10B6300062EE882A2AEE082A21EE081A60EE880AAD
:10B64000F0EE443AB0EE443AF0EE441AB0EE440A5A
:10B6500057F0E2FA9FED424AD4EDB02A94EDB31AC6
:10B66000D7ED010A62EE882A29EE082A21EE081A8F
:10B6700060EE880AF0EE443AB0EE443AF0EE441A36
:10B68000B0EE440A57F0CCFA9FED354AD4EDB12A1A
:10B6900094EDB41AD7ED020A62EEC82A28EEC82A41
:10B6A00021EE481A60EEC80AF0EE443AB0EE443A91
:10B6B000F0EE441AB0EE440A57F0B6FA1DB0BDECF5
:10B6C0000C8BBDE8F08F4FF00109F7E5012309E687
:10B6D0004FF001081BE64FF0010B2AE6F0EE488A16
:10B6E000B0EE489A65E69FED1ECA76E6DFED1CBA1D
:10B6F00090E6DFED1BAA23E7DFED199A3AE79DF804
:10B700003430002B7FF472AFD5F82C3D149AC3F877
:10B71000D8206BE79DF83530002B7FF46FAFD5F85C
:10B720002C3D159AC3F8D42068E79DF83630002BDD
:10B730007FF46CAFD5F82C3DC3ED38AA66E79DF8D1
:10B740003730002B7FF46AAFD5F82C3DC3ED379A24
:10B7500064E700BFF0250120C05A0120385B0120BA
:10B7600000000000EC5B0120645C01209459012082
:10B77000485A01200000C8422DE9F04F2DED068BFC
:10B780008FB0B74C0393D4ED37AA04F5005480462C
:10B79000D4F82C3D1B7B0D461746002B00F02E8164
:10B7A000B4F88E63C6F3400B06F0010AC6F38009B5
:10B7B00016F0080600D0012603AB4A465146009316
:10B7C00058463346FFF7C4FC94EDDD1A95ED000AA8
:10B7D0000590F1EE410A9A2017F0C2F894EDDD1AB7
:10B7E000F0EE409AF1EE410A95ED010A9B2017F028
:10B7F000B7F894EDDE1AB0EE409AF1EE410A95EDFD
:10B80000020A984D9C2017F0ABF894EDDF1AF0EE89
:10B81000408A9D2097ED000AF1EE410A17F0A0F84A
:10B8200098ED007AD8ED017A9DF80C3069EE876AC0
:10B830000027CDED066A69EE276AB0EE408ACDEDAD
:10B84000076AD5EDAF6A0A9727EE267AD5EDB06A7A
:10B850008DED087A67EEA67A0B97CDED097AFBB9E4
:10B860009DF80D30E3B99DF8143007EE103A9DF8BD
:10B87000153007EE903AB8EE477AF8EE677AB0EEF8
:10B880006A0A0CAB08AA06A905F569708DED0C7A59
:10B89000CDED0D7A4DF0E4FD8DED0A0ACDED0B0AEC
:10B8A0009DF80E30002B40F0AE8098ED000AD5EDEB
:10B8B000B10A9DF816106C4860EE200AB0EE6A1AC4
:10B8C00028EE800A4DF0FEFFB0EE40AA64480AA9B7
:10B8D000FEF788FC9DF80F30002B40F0978098ED24
:10B8E000010AD5EDB60A9DF81710604860EE200AEF
:10B8F000B0EE6A1A20EE080A4DF0E4FFB0EE408A7E
:10B90000D4F82C3D1B7B7BB959480C970CA90D979B
:10B910004DF0D0FE9FED570A53484DF0EFFF9FEDDD
:10B92000550A52484DF0EAFFBBF1000F71D0D4F830
:10B930002C3DC3F8D870BAF1000F74D0D4F82C3D68
:10B94000C3F8D470B9F1000F77D0D4F82C3DC3F808
:10B95000E070002E7AD0D4F82C3DC3F8DC709FED57
:10B96000468A9FED444AD5EDAF2A95EDB21A62EEB4
:10B97000882A29EE882A21EE081AF0EE443AB0EE21
:10B98000443AF0EE441AF0EE440AB0EE440A57F09E
:10B9900043F99FED384AD5EDB02A95EDB31A62EE22
:10B9A000882A29EE082A21EE081AF0EE443AB0EE71
:10B9B000443AF0EE441AF0EE440AB0EE440A57F06E
:10B9C0002FF99FED2C4AD5EDB12A95EDB41A62EE10
:10B9D000C82A28EEC82A21EE481AF0EE443AB0EE02
:10B9E000443AF0EE441AF0EE440AB0EE440A57F03E
:10B9F0001BF90FB0BDEC068BBDE8F08F4FF00109CD
:10BA0000CA46CB46D7E69FED1BAA5FE79FED198A92
:10BA100076E79DF80C30002B8DD1D4F82C3D0A9A96
:10BA2000C3F8D82087E79DF80D30002B8AD1D4F8D1
:10BA30002C3D0B9AC3F8D42084E79DF80E30002BE0
:10BA400087D1D4F82C3D83ED38AA82E79DF80F30DA
:10BA5000002B84D1D4F82C3D83ED378A7FE700BFDB
:10BA6000F0250120F0550120485A0120C05A01203C
:10BA700094590120000000000000C84270B504463F
:10BA8000103042F02BFB0B4E0B4B23613825601915
:10BA900042F042FD66513035B5F54E7FF7D104F5E1
:10BAA0004E7043F0B5FF2046044933F027FB204693
:10BAB00070BD00BFECE0090800E1090818DA0908C8
:10BAC00037B500F50D5101220831044635F0B4FBBD
:10BAD0001C4A1368D90706D41B4904F504531033D4
:10BAE0000B600123136004F50E5017490122183032
:10BAF00033F0BEF80125002304F58151CDE9005350
:10BB0000124A1831FD2033F045F8114B1A68D2075C
:10BB100005D4104A1D6004F58A54083414600D4899
:10BB2000012133F0C1F833F0EFFC0B4A0B481388C6
:10BB300043F0400313800421002203B0BDE83040ED
:10BB400033F024B8645E012000220120985D0A08C9
:10BB5000685E01200C220120985F012008DF09089F
:10BB60000069C0F3401070470F299DBF302303FBCD
:10BB70000100283000207047014B93F962037047A1
:10BB8000F0450120024B93F8290D00F001007047A9
:10BB9000F0450120014BD3F8F40A7047F04501202D
:10BBA000002910B517DB104C94F8FC2ACBB29A424E
:10BBB00011D3D4F8F83A0122595CA4F5005000F0F2
:10BBC00063FD94F8193D38B99A0704D5074A1378EC
:10BBD00043F00403137010BD9B07FCD5034A137890
:10BBE00043F00203F6E700BFF04501202C5F01207F
:10BBF000022A10B50F4C12D13522A4F5005000F0E6
:10BC000043FD94F8193D9B0705D50B4B1A7818B1E5
:10BC100042F002021A7010BD42F00402FAE794F8F2
:10BC20001C2D8A42F7D142F03BFCBDE8104042F0A7
:10BC30003BBB00BFF04501202C5F0120064A92F873
:10BC4000293D92F8282D03F00103134301D142F05E
:10BC50003BBA0020704700BFF0450120332901D0D6
:10BC600043F0F6B97047000008B50A68332A07D0D8
:10BC7000382A08D10A790321FFF7BAFF012008BD4D
:10BC80000A790121F8E7BDE8084042F087BF0000CB
:10BC900030B589B00446684606F020FD04F5965597
:10BCA00004A806F01BFD6946284602F0B3FF70B1F8
:10BCB00004A9284602F0DEFF48B104A9684606F050
:10BCC0003BFD236800221B6D69462046984709B05A
:10BCD00030BD000000F5805292F85425D2070AD4F6
:10BCE00000F50052D2F82C2D117B09B1FFF7D0BF1F
:10BCF0000368DB6C1847704710B586B0044602A88D
:10BD0000019106F0EBFC02A904F5965002F082FFC7
:10BD100028B12368019A1B6D02A92046984706B0F6
:10BD200010BD0000F0B5044685B0684604F596578E
:10BD30000E46154606F0D2FC6946384602F09AFFD8
:10BD400010B9002005B0F0BD3146384602F0B2FD12
:10BD50000028F6D0002DF5D004F58054284694F83C
:10BD6000543543F0020384F85435EBE710B500F581
:10BD70000054D4EDDB7AF5EEC07AF1EE10FA8AB019
:10BD80004FF0000343D907930893099306AB01933F
:10BD900007AB03AA04A9009300F5965005AB02F087
:10BDA00027FEDDED080A9DED070A77F073FBDDED58
:10BDB000090A77F06FFBD4EDDB7A9DED047A77EE1C
:10BDC000A76AB4EEE70AF1EE10FAF4EEC76AACBF68
:10BDD00001200020F1EE10FA0CD802309DED037A1C
:10BDE000F4EEC77AF1EE10FA0CD8003818BF012033
:10BDF0000AB010BDF4EEC77AF1EE10FA9CBF013024
:10BE0000C0B2EBE7012894BF00200120F0E700203A
:10BE1000EEE7000038B500F50055044695F8293DD9
:10BE20005A071AD443F0040385F8293D37F0E8FB9C
:10BE30000122112137F040FB084BD3F86807036853
:10BE40009B68984718B995F96933032B05D12046AB
:10BE50000621BDE8384000F015BD38BDF055012081
:10BE600008B500F5005090F8293D5A070BD56FF33F
:10BE7000820380F8293D37F0C3FBBDE8084000226B
:10BE8000112137F019BB08BD2DE9F043054685B0F7
:10BE9000684605F5965806F021FC6946404602F0D2
:10BEA000E9FEC8B105F50053424CD3F82C2D424FA2
:10BEB000127B32B1D3EDDB7AF5EEC07AF1EE10FAF7
:10BEC0000DD8238823F4FF7323F001032380284631
:10BED0000023FB73FFF7C4FF05B0BDE8F0832846DD
:10BEE00001F066F8064618B9284601F027F806461C
:10BEF0002846FFF73BFF814640B93EB12378002B2F
:10BF000041D1637803F00103FB73E5E76378DB0756
:10BF1000F7D423780133DBB2082B237006D12846EF
:10BF2000FFF724FF10B1404602F0CEFD2378092B25
:10BF300002D1404602F0C0FD2378092BE1D92388C5
:10BF400023F4FF7323F0010343F48573238037F058
:10BF500057FB0222102137F0AFFA57F09BFD6368C0
:10BF6000C01A47F23053984209D905F52D50134AAB
:10BF7000022114303BF028FE57F08CFD606028460B
:10BF8000FFF748FFBDE7013B23702388C3F3080395
:10BF9000B3F5807FB5D1637860F30003637037F049
:10BFA0002FFB4A46102137F087FA2846FFF758FF43
:10BFB000A7E700BF6C5E01200D5F01201CE10908AE
:10BFC00037B5044601A900F5965004F5005502F076
:10BFD000BBFBD5F8403B834206D0C5F8400B37F099
:10BFE0000FFB3E2137F048FA04F5805395F9441BC6
:10BFF00093F8E82593F9E835994213D0FF2A11D038
:10C0000085F8443B37F0FCFA95F8442B182137F0BB
:10C0100053FA04F52D5095F9443B034A042114309A
:10C020003BF0D2FD03B030BD2CE109082DE9F0430F
:10C0300095B0064657F02EFD03AB019306F59659D1
:10C0400002AB0024009305460EAB0BAA08A9484694
:10C05000089409940A940B940C940D940E940F94E4
:10C06000109402F0B3FCDFED437A9DED0A7AB4EE52
:10C07000E77AF1EE10FA074637DB9DED0D7AB4EE64
:10C08000E77AF1EE10FAACBF4FF001084FF000086C
:10C0900007AB019311AB009304AA06AB05A9484670
:10C0A00011941294139402F0A3FC06F50054002896
:10C0B00094F9DC3A08BF002783B17FB1D4F82C3D56
:10C0C0001B7B5BB1B8F1000F08D09DED057AF7EE50
:10C0D000007AB4EEE77AF1EE10FA09D594F8483B0D
:10C0E00073B90023C4F84C3B0FE04FF00008CFE7D2
:10C0F000D4F84C0B20BBC4F84C5BC4F8500B04E0E4
:10C10000D4F8500B20B9C4F8505B15B0BDE8F083EB
:10C11000281A43F698239842E3D9002584F8485B0F
:10C12000C4F8505B37F06CFA2A461D2137F0C4F989
:10C1300006F52D50104A022114303BF045FDD0E7A2
:10C140002D1AB5F57A7FE0D994F8483B002BDCD165
:10C15000012584F8485B37F053FA2A461D2137F051
:10C16000ABF906F52D50054A022114303BF02CFDA9
:10C17000CBE700BF0000003444E109085FE1090893
:10C1800010B5044637F03CFA0022052137F094F947
:10C1900004F52D50034ABDE81040042114303BF053
:10C1A00013BD00BF7CE1090800F5005090F8193D6F
:10C1B0009B065ABF90F8180DC0F30010012070477D
:10C1C00038B5044602F072FF4FF4804102F0ACF83B
:10C1D00004F50052054692F8193DC3F3001181425F
:10C1E0001CD060F3041304F52D5482F8193D143467
:10C1F00060B137F005FA02220B2137F05DF9084AE9
:10C2000020460221BDE838403BF0DEBC37F0F8F9AB
:10C210002A460B2137F050F9024AF1E738BD00BF3A
:10C2200094E109089FE1090870B500F5005504463E
:10C2300095F95233ABB3D5F8A46C96B357F02AFCFA
:10C2400005F6E42393ED000ADFED167A9FED161A4A
:10C25000DFED160A861B20EE270A692016F080FB08
:10C26000BCEEC00A10EE103A9E4209D295F8293D64
:10C270009A0716D520460021BDE87040FDF79ABC0C
:10C280000FD995F8293D9B070BD420460121FDF7D6
:10C2900091FC04F52C500122BDE870401221FDF7FD
:10C2A000E1BB70BD00007A440000804F0000000038
:10C2B0000B46012B10B4114604D0052B06D05DF8B7
:10C2C000044B70475DF8044B00F0DCBA5DF8044B9A
:10C2D0000122142100F52C50FDF7C4BB2DE9F041DB
:10C2E000044604F5005837F08BF90122052137F098
:10C2F000E3F898F956532046003D18BF0125FFF793
:10C3000053FF04F52D56143690B11D4A04213046D2
:10C310003BF05AFC0122102104F52C50FDF7A2FB42
:10C320000025294620460322BDE8F041FFF7C0BFA3
:10C3300004F54057D7F868070368DB6A984768B187
:10C3400097F88D3253B197F98C32012B06DC0D4AE8
:10C35000042130463BF038FC0125E2E7D7F86807B6
:10C360000368DB6A984718B1D8F8E03A1B0705D490
:10C37000054A042130463BF027FCD2E7034AE7E7B1
:10C38000B4E10908CFE10908FDE109080CE2090858
:10C3900070B50446154637F033F90122062137F00F
:10C3A0008BF82046FFF700FF04F52D56143690B1A8
:10C3B0000122072104F52C50FDF754FB144A0421F7
:10C3C00030463BF001FC0025294620460422BDE80A
:10C3D0007040FFF76DBF04F54053EDB2D3F8680726
:10C3E0000368DB6A984768B104F50053D3F8E03A74
:10C3F0001B0707D535B1074A042130463BF0E4FB63
:10C400000125E1E7044A042130463BF0DDFBDBE790
:10C4100030E20908D7E109084DE20908F8B50446F9
:10C4200057F02EFB284BB4F8BE201988274E9142B6
:10C4300005460ED01A80264B18603378A3B100242D
:10C44000347037F0DDF822461321BDE8F84037F0AC
:10C4500033B833781F4FC3B93B782BB11C4B1E4AFE
:10C460001B68C31A934200D8F8BD0123337004F54A
:10C470000053D3F82C0D037B0BB1FEF735FA37F0E0
:10C48000BFF80122132137F017F83B78002BEBD0CF
:10C490003378002BE8D00E4A10491368EB1A8B4210
:10C4A000E2D904F500541560D4F82C2D137B002B31
:10C4B000DAD0002313730A4AD4F82C0D1371BDE8A7
:10C4C000F840FEF7E1B800BF765E0120745E0120FF
:10C4D000785E0120755E012080841E0040420F00BE
:10C4E0000D5F01207FB500F5005300F54E5508356E
:10C4F00093F8481B0446284656F0ECFA04F5965685
:10C50000684606F0EBF86946304602F083FB04F516
:10C510004053029AC3F8A822039AC3F8AC22202100
:10C52000304601F001FFD0B1284656F025FB04F556
:10C530004A55FDEEC07A203504F5805417EE901A66
:10C540000222284617EE906A06F0CCF894F854358B
:10C55000DB0706D401223146284606F0C3F804B0B2
:10C5600070BD0121284606F065F90028F2D0F6E7F3
:10C57000012070470020704700207047002070475E
:10C58000002070470020704700207047002070474F
:10C590009FED010A704700BF000000009FED010AF7
:10C5A000704700BF0000000070470000104A0260A2
:10C5B000104A426002F15001816002F58251C1606F
:10C5C0000D49016102F6E411416102F6E811816151
:10C5D00002F5F461C16102F2A471016202F5F56134
:10C5E00002F2AC728262054A4162C262704700BFC9
:10C5F000D8E2090838490120B03801200827012075
:10C60000042917D8DFE801F003070B0F130000F52A
:10C610005E501C30704700F55D502C30704700F5BF
:10C620005F500C30704700F55F503C30704700F5AC
:10C630006050FAE70020704700F54050D0F86807D6
:10C6400003685B681847000038B500F5405504469C
:10C65000D5F8680703685B6998470A4B04F50052F0
:10C66000187492F81C2DD5F86807DA7003685B6AB5
:10C670009847014604F593501030BDE838402FF03C
:10C6800073BF00BF0D5F01202DE9F84F00F5005A80
:10C6900006469AF81C3D8B420F46914605D18AF812
:10C6A0001D2D01252846BDE8F88FFFF7A9FF044698
:10C6B00020B9304634F068FF2546F3E7DAF82C3D20
:10C6C0001B7B06F52D5883F0010B08F11408EBB91C
:10C6D000236859461B6820469847054680B306F5EF
:10C6E000405306F58150C3F868474A4639468AF8F0
:10C6F0001C7D8AF81D9D183036F098FA40460021BE
:10C7000040F08EFF3046FFF79FFFCBE703689B6842
:10C710009847E0B11C4800F037FC0546B8B92368DB
:10C7200020461B6A9847194A0346042140463BF0BD
:10C730004BFA36F065FF3A460A2136F0BDFEB1E706
:10C74000236820461B6A9847114A0346EDE70E48C6
:10C7500000F036FC0028BBD106F54053D3F868073B
:10C760000368DB6898470028B2D023682046DB685E
:10C77000984705460028ABD1236820461B6A984796
:10C78000044A0346D1E700BFF025012060E2090812
:10C79000B2E2090889E209080148FFF775BF00BF46
:10C7A000F025012070B5234B93F8293DDB070546A2
:10C7B0000C46164605D5002363602360A3603360F2
:10C7C00070BD41F06DFE037F002BF4D0EB699FED4F
:10C7D0001A7A1B68B3F90A3007EE903AF8EEE77A56
:10C7E000C7EE876AC4ED016A2B6A1B68B3F90A3089
:10C7F00007EE903AF8EEE77AC7EE876AC4ED006A72
:10C800006B6A1B68B3F90A305B4207EE903AF8EEA8
:10C81000E77AC7EE876AC4ED026AAB6A1B68B3F9B0
:10C820000A3007EE903AF8EEE77AC7EE876AC6ED6F
:10C83000006AC5E7F045012000007A4400207047F7
:10C840000120704700207047002070470048704763
:10C8500010370A080048704720E309080020704795
:10C8600043691A680023C2F8D43042691268C2F8DA
:10C87000D83042691268C2F8DC3042691268C2F8E6
:10C88000E03070470A4608B50021FFF7FDFE034A75
:10C89000137843F00803137008BD00BF2C5F01201C
:10C8A000012070470020704701207047002070472A
:10C8B0000048704778E309080048704780E309089A
:10C8C0000320704730B5084B03F54B52083204463D
:10C8D00000F1300507CA85E8070003F5A6531833B1
:10C8E00001201B68E36330BDF025012030B52DED3C
:10C8F000028B044687B0574D002301AA03A995ED8A
:10C90000378A039304930593FFF74CFF63689DED0B
:10C91000037AD3ED0E7A68EE277A27EE277A8DED2B
:10C92000037A9DED047A67EE277ACDED047AD3ED94
:10C930000F7A28EE277ADDED057A67EE877ACDED5E
:10C94000057AD3ED107A93F9443028EE278ADDED8D
:10C95000017A27EE888A8DED018A1BB903A9284642
:10C96000FDF724FC3C4A94ED0C7AD2EDB27A636870
:10C9700094ED0F0AD3ED0E6A77EE677AF0EEE77A60
:10C98000F4EEE67AF1EE10FA44BFDDED037A77EECD
:10C99000877A94ED0D7A48BFC4ED0C7AD2EDB37A64
:10C9A000D3ED0E6A77EE677AF0EEE77AF4EEE67A88
:10C9B000F1EE10FA44BFDDED047A77EE877A94ED5C
:10C9C0000E7A48BFC4ED0D7AD2EDB47AD3ED0F6A7A
:10C9D000236977EE677AF0EEE77AF4EEE67AF1EE25
:10C9E00010FA42BFDDED057A77EE877AC4ED0E7A54
:10C9F000D3ED867A30EE670A15F09EFF6368D3EDBB
:10CA0000107AB0EEC00AB4EEE70AF1EE10FA09D5DA
:10CA100094ED0F0ADDED017A30EE270A15F08CFF58
:10CA200084ED0F0A00230D488DF808308DF8093089
:10CA30008DF80A308DF80B30029BD0F8300D04F1E0
:10CA40003C0204F13001FEF799FB07B0BDEC028B0C
:10CA500030BD00BFF0250120F0550120F045012038
:10CA60000020704701207047012070470020704768
:10CA700000487047D8E3090800487047E0E3090818
:10CA8000012070471FB5044600236A4601A901939F
:10CA900002930393FFF786FE6369029A1B68C3F84B
:10CAA000D4206369019A1B68C3F8D8206369009A8F
:10CAB0001B68C3F8DC206369039A1B68C3F8E02095
:10CAC00004B010BD0120704700207047012070475E
:10CAD00000207047004870475EB009080048704762
:10CAE0005EB0090804207047012070477FB500231D
:10CAF0000393049305930193094800238DF80830AC
:10CB00008DF809308DF80A308DF80B30029BD0F883
:10CB1000300D01AA03A9FEF731FB07B05DF804FB55
:10CB2000F045012001207047002070470120704728
:10CB3000002070470048704788E4090800487047A3
:10CB400094E409080220704710B5044686B000231B
:10CB500001AA03A9039304930593FFF723FE6368D7
:10CB60009DED037AD3ED0B6ADDED047A93F9443041
:10CB700027EE267A67EEA67A8DED037ACDED047A5C
:10CB80001BB9144803A9FDF711FB6368DDED057AB5
:10CB900093ED0C7A104867EE877A93ED0D7ACDED20
:10CBA000057ADDED017AD0F8300D002367EE877A43
:10CBB0008DF808308DF809308DF80A308DF80B307B
:10CBC000029BCDED017A01AA03A9FEF7D5FD06B0BF
:10CBD00010BD00BFF0250120F045012038B5044606
:10CBE00042F06CFF43F03AF804F50054054642F079
:10CBF000CFFF42F0C1FCD4F82C0DFDF745FD2846CF
:10CC0000BDE8384042F0CCBF10B500F50054142107
:10CC1000D4F8E80A41F094FCD4F8EC0A142141F06D
:10CC20008FFCD4F8F00A1E2141F08AFCD4F8F40AF3
:10CC30001421BDE8104041F083BC000038B5054622
:10CC400041F02EFC41F080FB05F50054C4F8E80AE1
:10CC500041F026FC41F082FBC4F8EC0A41F020FCD4
:10CC600041F086FBC4F8F00A41F01AFC41F08AFB5F
:10CC70004FF47A71C4F8F40AD4F8E80A41F05CFC85
:10CC8000D4F8EC0A4FF47A7141F056FCD4F8F40A67
:10CC90004FF47A7141F050FCD4F8F00A4FF47A71F5
:10CCA00041F04AFC2846FFF7AFFF94F8193D43F0E6
:10CCB000080384F8193D38BD08B542F0CFFF42F0B3
:10CCC000F3FDBDE8084042F0A5BD000000F50050AE
:10CCD000D0F82C0DFDF708BE38B500F50054054618
:10CCE00094F956332BB900212846BDE83840FCF7AB
:10CCF00047BFB4F858338B4219D994F8293DDA0765
:10CD00000FD441F0CDFB037F1BB9D4F82C3D1B7B26
:10CD10003BB194F8283D01335BB2022B02DC84F86E
:10CD2000283D38BD032384F8283D0121DCE794F831
:10CD3000283D013B5BB2002BF1DC002384F8283D49
:10CD400094F8293DDB07CED4EBE7000038B50D465B
:10CD5000044656F09FFE002D0B4B09DD04F50054F0
:10CD6000186094F8193D6FF3C30384F8193D38BD7A
:10CD70001B68C01AB0F5C87FF9D904F5005494F8BF
:10CD8000193D43F00803F0E77C5E0120F7B5044647
:10CD900056F080FE064641F083FB41F055FB04F55A
:10CDA0000055B0B395F8183D43F0200385F8183DC1
:10CDB000D5F8F03A20461989FFF78EFFD5F8F03AFA
:10CDC00004F54057B3F90A102046FFF7BFFFD7F824
:10CDD00060379FED307AF31A07EE903AD5F8F03AC3
:10CDE000F8EE677AB3F90A3067EE877A04F54A50AD
:10CDF000CDED007A07EE903AF8EEE77A6A4601A99F
:10CE00001430CDED017A37F085FDC7F8606703B0C7
:10CE1000F0BD95F8293DDB07F9D404F54053D3F86C
:10CE20006007361A41F0F2F980BB41F039FB9FED03
:10CE30001A7AD0ED067A67EE877A9FED187AF4EECB
:10CE4000C77AF1EE10FAD8BFF0EE477AFCEEE77A37
:10CE500017EE903AB342DAD895F95633002BD6D074
:10CE600041F01EFB037F23B9D5F82C3D1B7B002B23
:10CE7000CDD036F0C5FB0222114636F01DFB012154
:10CE8000204603B0BDE8F040FCF77ABE4FF47A7359
:10CE9000E0E700BF6F12833A00007A440000C84206
:10CEA00038B5044600F58665284604F07DFB94F805
:10CEB00041049FED087A242202FB0055D5ED0B7A40
:10CEC00067EE877A04F54053FDEEE77AC3EDA47A66
:10CED00038BD00BF0000C842FEF718B90148FFF78F
:10CEE0009DBA00BFF025012010B5838F044643B9D9
:10CEF00034F060FE92224FF4801134F013FE638F01
:10CF0000A387A08F10BD000038B500F596550446E4
:10CF1000284600F0DBFC04F58053022283F8E0246D
:10CF200004F16800FFF7E0FF014604F6980015F0F1
:10CF3000BBF82846BDE8384000F0C2BD38B500F562
:10CF400096550446284600F00DFF08B9002038BD6C
:10CF500004F50054D4F82C3D1B7B63B910212846FE
:10CF600001F0E2F90028F2D14FF400712846BDE843
:10CF7000384001F0D9B98021284601F0D5F90028C0
:10CF8000E4D11021F2E7000038B500F50053054662
:10CF900093F8293D5B0709D4FFF7D0FF044618B981
:10CFA00005F5965000F0DEFE204638BD0024FBE774
:10CFB00008B500F5965000F0D5FE002008BD000031
:10CFC00010B500F59654204600F0CCFE50B1042177
:10CFD000204601F0A9F928B120462021BDE81040E3
:10CFE00001F0A2B9002010BD38B500F50055044687
:10CFF00095F8183D590719D5D5F82C3D1B7B2BB951
:10D0000020460021BDE83840FCF7A4BD00F54053A0
:10D01000D3F868070368DB68984738B195F8193D7D
:10D020001A0703D595F8293DDB07E9D538BD00007F
:10D0300037B500F581551835044604F500542846E7
:10D04000019135F03BFD94F8183D019960F3C3035D
:10D05000284684F8183D03B0BDE8304036F09ABA4F
:10D060000720704700487047ECE4090837B50546CB
:10D070001048FFF739FF0190EC2005F053FE0446FD
:10D0800010B10199FDF7A0FA05F50050C0F82C4D3C
:10D0900024B990F9A413084805F0EAFA0749204694
:10D0A00032F03AFA012031F063FC03B0BDE83040C1
:10D0B00032F02ABA58260120F4E40908D4A4090859
:10D0C00073B5044600F5935010302FF001FA204656
:10D0D000FFF7BAFA04F5355004F026FE04F5875040
:10D0E000103004F5866643F021FA304604F00EF95C
:10D0F00004F52D5014303DF09FF92046FFF79EFDBA
:10D100002046FFF7B3FF5F48FFF7EEFE082005F06B
:10D1100009FE18B14FF07E530360436004F50055DB
:10D12000C5F8300D41F0BCF99922292142F064F98B
:10D1300041F0B6F941F0D6F82046FFF7BDFD95F86D
:10D14000193D04F5915043F0400385F8193D1C301A
:10D1500044F0E6FE4C4B4D491B68986A03684FF457
:10D160007A72DB6A98470423C4F8743104F590702E
:10D170000CF086FF06F094FB4FF40053036306F0B7
:10D180008FFB07F029F88023C4F84434012130468E
:10D1900004F01AFB3E4B00933E4B019304F5815083
:10D1A00002AB13E90600183035F034FB2046FFF7D8
:10D1B000ABFE4FF40023C4F8A83BD5F82C0DFDF7C7
:10D1C0000DFA012104F52C50FCF7B6F910B12046F8
:10D1D000FFF77CFD04F168063046FFF785FED5F8C1
:10D1E0002C3D07EE900A04F54B50D3ED390AB8EE0A
:10D1F000670AF2EE0E1AB6EE001A1C3038F060F82C
:10D200003046FFF771FED5F82C3D07EE900A04F585
:10D210004C50D3ED390AB8EE670AF2EE0E1AB7EEAB
:10D22000001A203037F076FE3046FFF75DFED5F865
:10D230002C3D07EE900A04F54D501430D3ED390A19
:10D24000B8EE670AF2EE0E1AB1EE041A37F062FE7B
:10D2500095F863131A222046FFF716FA60B92122C7
:10D2600001212046FFF710FA95F8193D43F002031B
:10D2700085F8193D02B070BD074A137843F00803E2
:10D280001370F1E758260120605E0120DDCE010811
:10D29000F0250120D9CE01082C5F0120836833B925
:10D2A000C36823B94068003818BF012070470120C7
:10D2B000704700002DE9F0412DED048B92B004463B
:10D2C00002AD284605F00AFA94F8D433002B70D04A
:10D2D00004F580630FCB85E80F0094F81034D4ED8B
:10D2E000F28A94EDF38A94EDF49A002B61D094F8CD
:10D2F000E833002B5DD02846D4F8D883D4F8DC730B
:10D30000D4F8E063D4F8E443FFF7C8FF002855D110
:10D310002E4B01932D22002106A878F015FCA323A3
:10D320008DF8183095238DF8193046238DF81A3072
:10D3300056F0B8FB9FED260ADFED267ACDF81F10D8
:10D3400068EE808A28EE008A68EEA78A28EE278A8F
:10D35000FDEEE88ABDEEC88A18EE903A29EE000A82
:10D36000ADF8233018EE103A20EE270ACDF81B0056
:10D37000ADF8253015F0B4FABCEEC00ACDF8358012
:10D3800010EE103AADF82730019BCDF82930049B00
:10D39000CDF82D30059BCDF83130CDF83970CDF872
:10D3A0003D60CDF8414036F02BF92D2206A935F02D
:10D3B00065FA12B0BDEC048BBDE8F08101AA002132
:10D3C000284605F047FA0028A2D0A3E75241C07FC3
:10D3D000E02E65420000C84230B52DED028B8BB0C7
:10D3E000044624220D4601A8002178F0ADFBA323BA
:10D3F0008DF8043095238DF8053048239FED1F8A62
:10D400008DF8063056F04EFBD4ED847A2B68CDF8BB
:10D410000F3067EE887A95ED020ACDF80B1017EE03
:10D42000903AD4ED857ACDF8133067EE887A6B6840
:10D43000CDF8173017EE903ACDF80700CDF81B3035
:10D4400015F024FA10EE103A94ED860ACDF81F304C
:10D4500020EE080A15F01AFA10EE103ACDF8233033
:10D4600094F824338DF8273036F0CAF8242201A925
:10D4700035F004FA0BB0BDEC028B30BDE02E6542F6
:10D4800030B5104689B00D461446FFF707FF28BB9C
:10D49000002301931822002102A878F055FBA32352
:10D4A0008DF8083095238DF8093049238DF80A301E
:10D4B00056F0F8FAA3680593E3680693019BCDF84C
:10D4C0000F100793CDF80B008DF8135036F098F835
:10D4D000182202A935F0D2F909B030BD01AA002105
:10D4E000204605F04BF90028D2D0D3E710B590B014
:10D4F000044604A805F0F2F804A9204601F08AFBCE
:10D50000002846D001F0D2FD01A901F07DF902A961
:10D51000204600F0C3FC00283DD0DDED027AF1EE9C
:10D52000677A03AA002104A8CDED027A05F092F9EA
:10D5300008B91A4B03931F22002108A878F004FBB6
:10D54000A3238DF8203095238DF821304A238DF8C0
:10D55000223056F0A7FA069BDDED017ACDF82B308C
:10D56000079BCDF82F30F1EE677A039BCDF833306F
:10D5700017EE903ACDF83730029BCDF82710CDF852
:10D580002300CDF83B3036F03BF81F2208A935F0D8
:10D5900075F910B010BDDFED027AC2E75241C07FCD
:10D5A0005241C07F0023036043608360C360036116
:10D5B00043618361C36103627047000090F8C43225
:10D5C000B02202FB030390F8082393F8A13012B1B4
:10D5D000012B28BF01231846704700002DE9F04FAA
:10D5E00004468BB04FF0000A0D461BF037FA84F862
:10D5F00020A204F509704FF07E5755F0A9FB4FF4B7
:10D600007A73A4F87A3284F8805204F52170C4F851
:10D610006072C4F86472C4F86872002505F05EF8A0
:10D6200004F531790323C4F8983204F53A76C4F846
:10D63000AC52C4F8B052C4F8B452C4F8B852C4F8EA
:10D64000BC52C4F8C0524846FFF7ACFF04F54E7B0D
:10D650003046FFF7A7FFC4F82C53C4F83053C4F882
:10D6600034535846FFF79EFFC4F85C53C4F8605328
:10D67000C4F86453C4F86853C4F86C53C4F87053C6
:10D68000C4F87453C4F87853C4F87C53C4F8805376
:10D69000C4F88453C4F88853C4F8A453C4F8A853F6
:10D6A000C4F8AC53C4F8C053C4F8BC53C4F8B8535E
:10D6B000C4F8C853C4F8CC53C4F8D053C4F8E453E6
:10D6C000C4F8E053C4F8DC5304F57B70C4F8B473B9
:10D6D000C4F8D87305F002F804F5806004F0FEFF8A
:10D6E00004F2144304F586601D605D6004F58463F4
:10D6F00004F27C481D605D609D6004F0EFFF04F261
:10D70000444340461D605D609D606D4BC4F85434D9
:10D7100004F51073C4F8583404F51173C4F85C347C
:10D7200004F51273C4F8603404F51373C4F8643458
:10D7300004F25123C4F8683404F51473C4F86C344B
:10D7400004F58E6304F254421D605D609D60FFF736
:10D7500029FF04F59460FFF725FF04F59A6304F2AE
:10D76000BC501D605D609D6004F2DC431D605D6027
:10D770009D6004F59D631D605D609D6004F2F4434F
:10D780001D605D609D6004F204531D605D609D60DE
:10D7900004F214531D605D609D6004F5A763C2F838
:10D7A000D470C2F8D8701D605D609D6004F244536F
:10D7B0001D605D609D6004F5AC631F605D6004F2F8
:10D7C00084531D605D609D6004F5B2631D605D6003
:10D7D0009D6004F5B5631D605D609D6004F07EFF93
:10D7E00004F2CC5324221D605D6004F2D4535146F0
:10D7F0001D605D6004F2DC5340461D605D6078F0A2
:10D80000A3F904F5C060C8F82070C8F81070C8F813
:10D810000070FFF7C7FE04F2246304F27C601F600F
:10D820009D605D60DD6004F234631D605D609D603D
:10D8300004F5C8631D605D609D6004F24C631D606B
:10D840005D609D6004F5CB631D605D609D6004F2CA
:10D8500064631D605D609D6004F040FF194B1A49D0
:10D860001C60204631F04AFC51462422584678F08C
:10D870006BF9C4F85873C4F84873C4F8387304F5E6
:10D880002B7207CA04F52E7383E80700484694ED0F
:10D89000B01AD4EDAF0A94EDAE0A15F017FC354678
:10D8A000494668466E4615F033FB0FCE0FC50FCEC6
:10D8B0000FC533682B6020460BB0BDE8F08F00BF6A
:10D8C000D4E70908805E012070E6090810B5044617
:10D8D00088B001F057FC94F93E32012B02D1274861
:10D8E00004F0E4FE022B0AD1032384F83E3204A99B
:10D8F000012304F111008DF8103032F00BFA94F886
:10D900003E3284F8A83204F2544001F0F7FB94F957
:10D910003D32642B30D1652304A904F23D208DF8FB
:10D92000103032F035FA04A9204630F061FE18B309
:10D9300004238DF818300023CDE9013303930F231E
:10D940000593694604A831F029F8059B28B108AA77
:10D9500002EB8302009942F8581C0133112B059306
:10D96000EFD953F03BFE9DED031ADDED020A9DED6C
:10D97000010A652153F0F0FD08B010BD04E5090867
:10D9800070B500F52B7600F52E758CB00446314647
:10D99000284616F0DBFFE0B996E8070085E80700A7
:10D9A00004F5317194EDB01AD4EDAF0A94EDAE0ADE
:10D9B0000191084615F08AFB02AD019902A815F005
:10D9C000A7FA0FCD04F53A740FC40FCD0FC42B681E
:10D9D00023600CB070BD000013B540F2751200F565
:10D9E0000971044601A811F027FB04F2544001F02C
:10D9F0006FFD20461BF05EFA01A811F03FFB02B05C
:10DA000010BD0000F8B54B68C0F810328B68C0F844
:10DA10001432CB68C0F8183201F1100607460C46E4
:10DA200000F54E750FCE0FC50FCE0FC533682B60B6
:10DA300004F1440207CA07F54B7383E8070004F1B9
:10DA4000500207CA07F5577383E8070004F15C0228
:10DA500007CA07F55A7383E80700683494E807009B
:10DA600007F55D7383E80700384601F09FFC3846F0
:10DA7000BDE8F84001F082BC13B5044600F2544002
:10DA8000019003F03DF904F5BE610198009102F0A8
:10DA900025FD0099204602B0BDE81040FFF7B2BF57
:10DAA0004A78064BC2F340121A754A78C2F38012C4
:10DAB0005A750A78C2F300129A7570470D5F0120FB
:10DAC00013B540F24D32044600F5097101A811F07A
:10DAD000B3FA002104F2544001F028FF94F87832A0
:10DAE00023B120461BF068FF84F8780201A811F0EA
:10DAF000C5FA02B010BD000038B590F824330546D1
:10DB00000C462BB1032B0BD095F88032DB070CD4DD
:10DB100005F27C630FCB84E80F0095F88C0603E0D8
:10DB20001BF048FA0028EFD038BD0020FCE70000C9
:10DB300000F2544090ED350A7047000000F2544066
:10DB400090ED360A7047000010B490F824230C467C
:10DB50002AB1032A0AD000205DF8044B704700F573
:10DB6000B56007C884E807000120F5E75DF8044BBD
:10DB70001BF0DEB990F89C03431E58425841704791
:10DB800038B590F824330D468BB900F2544001F0BB
:10DB900007FD044610B90024204638BD01F05EFCA4
:10DBA000D5ED007A27EE800A85ED000AF4E7D0ED86
:10DBB000E67AC1ED007A90F89443002CEBD090ED1A
:10DBC000E47ADFED086AB4EEE67AF1EE10FAF7EEE9
:10DBD000006AB8BFB0EE667A67EE877AC1ED007A68
:10DBE000DAE700BF0000003490F82433032B01D1A2
:10DBF0001BF01EB90020704790F82423032A01D19E
:10DC00001BF090BA00F2544002F0EAB830B5054675
:10DC100085B00C469AB1032A1BD005F52B7016F07F
:10DC2000CFFE01A920468DED010ACDED020A8DED52
:10DC3000031A16F073FC0123184605B030BD90F8A6
:10DC4000F035002BF8D000F224630FCB84E80F00EE
:10DC5000E3E790F87832002BEED01BF03DFADCE7DA
:10DC600090F82423FFF7D2BF7FB590F8242332B178
:10DC7000032A4FF0000309D0039304930CE000F251
:10DC8000544007B05DF804EB01F0D4BC03A9039342
:10DC9000049305931BF0C2F89DED030ADDED040A21
:10DCA00007B05DF804FB000037B5044640F2C752E8
:10DCB0000D4600F5097101A811F0BEF9204629466C
:10DCC0001BF0A2F994F82433032B08BF044601A8E3
:10DCD00018BF002411F0D2F9204603B030BD000077
:10DCE00010B52DED028BB0F890361B0782B00446BC
:10DCF00030D5D0F838349FED198A07EE903AB8EE57
:10DD0000E77A01A927EE087A00F515708DED017A02
:10DD100031F0ECFFD4F83C3407EE903AF8EEE77AB5
:10DD200001A967EE887A04F51670CDED017A31F01D
:10DD3000DDFFD4F834349FED0A7A07EE903AF8EE1E
:10DD4000E77A01A967EE877A04F51770CDED017ABD
:10DD500031F0CCFF02B0BDEC028B10BD95BFD633C5
:10DD60000AD7233C90F82403003818BF01207047DD
:10DD700038B590F82423032A0C4604D11BF04EF842
:10DD80000125284638BD90F87056002DF9D000F2D4
:10DD9000646393E8070084E80700F2E710B590F8A1
:10DDA000242303460C461AB1032A0BD0002010BDD1
:10DDB00090F878060028FAD003F5BE63D3F88430D3
:10DDC0000B60F4E71BF040F8012084ED000AEEE759
:10DDD00030B590F8243385B005460C4623B1032BAB
:10DDE00009D0002005B030BD00F2544005B0BDE8B8
:10DDF000304002F075BA002302A9029303931AF08F
:10DE0000F5FF0028EDD001A928461AF0FBFF0028F5
:10DE1000E7D0029B2360039B6360019BA360E1E763
:10DE20001FB500230C4601A9019302930393FFF74A
:10DE3000CFFF28B1019B2360029B6360039BA3601B
:10DE400004B010BD90F824231AB1032A05D0002095
:10DE5000704700F2544002F077BA1AF0C7BF0000D2
:10DE600013B500230C46694600930193FFF7EAFFC0
:10DE700018B1009B2360019B636002B010BD0000DD
:10DE800090F824231AB1032A05D00020704700F22D
:10DE9000544002F04BBA1AF0B5BF000013B50C465F
:10DEA00001A9FFF7EDFF08B1019B236002B010BD8F
:10DEB00090F93E323BB990F8803213F0010F14BF55
:10DEC000032000207047032070470000F7B5044688
:10DED000FFF7EEFF0546002862D0032839D194F8F9
:10DEE00078326BB394F88032D8072BD501A920463D
:10DEF0001BF050F9BDF80430002B18BF002594F832
:10DF0000206206F0FD06012E4AD10023032D019365
:10DF100007D101A920461BF049F920461BF026F93C
:10DF2000064604F2544002F01FFB08B994F821039E
:10DF30009DF80430D90703D55A0701D59F0632D47E
:10DF400000252DE020461AF0B7FE002808BF002566
:10DF5000D5E70025D3E713F0020F2EE094F95032F5
:10DF600023B99DF80430DB092FD0E9E7002EF8D063
:10DF70000DF0ACFBFFF722FB022807D99DF8053016
:10DF80009806DDD59DF80430D906D9D5FB6A93F8FB
:10DF90009C30002BE5D118E0DA0601D41B0718D518
:10DFA000284603B0F0BD0028FAD094F82123B4F934
:10DFB0009036002ACFD013F0010FF1D1154B1F6816
:10DFC000FB6A93F89C30002BC8D19DF804309C0765
:10DFD000E2D405F065FC05F061FB0028B0D10DF03E
:10DFE00075FBFFF7EBFA0228AAD90DF06FFB90F84A
:10DFF000C432B02202FB030090ED2F7AF0EE007ADB
:10E00000B4EEE77AF1EE10FA9AD59DF80530DB0907
:10E01000C6D195E7605E01202DE9F04790F878328F
:10E0200092B00446002B00F0948020461BF022FAA8
:10E030002046FFF74BFF03287BD104F54E780027DD
:10E04000414620460097019702971BF01BF869464E
:10E0500020461BF00DF8009BC4F81032019BC4F859
:10E060001432029BC4F81832204601F09FF9204672
:10E0700001F084F913F0B2FF054620461AF0A8FE1D
:10E080000028A8BFC6B203AA4FF0FF312046BCBF8C
:10E0900095F80A9395F80B630397A8BFB1460497C8
:10E0A00005971AF0DFFE03A816F08AFC4FF00C0A61
:10E0B0000AFB095084EDD70AC4EDD80A84EDD91AB9
:10E0C00004F5577100F5117016F08AFC04F55D77C0
:10E0D0000AFB065584EDCB0AC4EDCC0A84EDCD1ABB
:10E0E0003A464FF0FF31204605F5C4751AF0CEFED2
:10E0F00095E8070006AE86E807003946304616F078
:10E10000D5FC04F53172414609A814F091FE314660
:10E1100009A814F00FFE09A9204684EDDA0AC4ED1F
:10E12000DB0A84EDDC1A1BF041F809A92046FFF751
:10E13000B7FC94F89236002B3AD109A804F0CEFA35
:10E1400009A920461AF042FF90B3012384F89236C1
:10E150002EE0D0F87C321BB955F09CFCC4F87C0250
:10E16000154B1B68D86A03685B68984788B155F0FF
:10E1700091FCD4F87C32C01AB4F87A32984204D9AF
:10E1800020461BF019FC84F8780294F878327BB1B1
:10E190004BE755F07FFCD4F87C32C01A41F287334C
:10E1A0009842E4D835F02CFA35F010FA0028DED188
:10E1B00012B0BDE8F08700BF605E012090F8243304
:10E1C00023B1032B4FF0000007D0704790F93E2297
:10E1D000032A04D10A70012070470870FBE7184633
:10E1E0007047000073B50D460DF107010446FFF7B7
:10E1F000E5FF064628B19DF807302BB1032B09D067
:10E200000026304602B070BD04F27C630FCB85E877
:10E210000F00F6E7294620461AF0CCFE94F8786203
:10E22000EFE7000037B50D460DF107010446FFF793
:10E23000C5FF28B19DF8072029462046FFF7E6FCD8
:10E2400003B030BD37B50D460DF107010446FFF7A9
:10E25000B5FF28B19DF8073023B1032B11D0002062
:10E2600003B030BD04F2F4531B682B6004F5BF63A8
:10E270001B686B6004F2FC531B68AB6094F8F005FC
:10E28000EEE7204629461AF0F3FE94F87802E7E715
:10E2900010B50446FFF70CFE18B1032807D0002084
:10E2A00010BD04F25440BDE8104001F04DB994F89F
:10E2B0007832002BF3D020461AF0FEFC0028EED076
:10E2C00094F8203203F0FD03012BE9D194F82403E4
:10E2D000C31E58425841E3E710B50446FFF7E8FD76
:10E2E00080B1032810D194F8780250B155F0D2FBD8
:10E2F000D4F87C32C01A44F62063984294BF0020C0
:10E30000012010BD0120FCE70020FAE708B5024615
:10E31000FFF7CEFD032804D110461AF047FF012075
:10E3200008BD0020FCE7000013B50C4601A9FFF76B
:10E33000EDFF20B1019B1C4214BF0120002002B060
:10E3400010BD000030B585B00446019102F0FEFD1D
:10E350000199054610B9002005B030BD019102F0C9
:10E36000C7FD01990028F6D0284602F0C5FD002817
:10E37000F1D0B4F890365907EED494F82133002B3D
:10E38000EAD00B4A1268D26A92F89C506DB103A988
:10E390002046FFF7BBFF30B19DF80E309A07DBD562
:10E3A000C3F38000D8E72846D6E71846D4E700BF75
:10E3B000605E012010B50446FFF77AFD032804D102
:10E3C0002046BDE810401AF0CBBD002010BD000073
:10E3D0002DE9F04190F824338CB00027032B06463A
:10E3E0000C46154600970197029719D11AF0F0FCD8
:10E3F0006A4680464FF0FF3130461AF047FDB8F1CB
:10E40000FF3FA760676027600DD113F0E7FD2B4643
:10E4100090F80B13224612F06FFE0CB0BDE8F081AD
:10E420004FF0FF38EBE713F0D9FD2B4622465FFA99
:10E4300088F112F061FE95ED000A684616F0FCFACC
:10E4400003A920468DED051A8DED030ACDED040AD2
:10E4500016F02CFB06F5317206F54E7103A814F088
:10E46000E7FC214603A814F065FC84ED021A84ED54
:10E47000000AC4ED010A95ED007ADFED037AA7EEFC
:10E48000271A84ED021AC8E70AE81C411FB5DFED20
:10E490000B7A20EE270A0C461946094BCDE90042BB
:10E4A000BDEEC00A18688DED020A064B9DF81820D3
:10E4B000C06A10F0B7FF04B010BD00BFE02E654287
:10E4C000605E012018E509082DE9F0472DED028B6B
:10E4D00092B0002504460F464FF07E5A00F54E716B
:10E4E00006A89046CDF818A009950895079515F04F
:10E4F000B7FC05F0D5F905F0D1F881462046FFF7C5
:10E50000D7FC032803D094F82433032B4FD19FED7D
:10E51000558ADFED558A00262379F2B2934247D916
:10E520000AAA71B22046CDF828A00D950C950B953E
:10E530001AF0B2FD0AA906A816F062F8B4EEC80AED
:10E54000F1EE10FA0DDD494ACDF800803B4648490E
:10E550002046FFF79BFF002012B0BDEC028BBDE808
:10E56000F0870AA906A803950495059516F032F8D8
:10E5700003A90EA88DED0E0ACDED0F0A8DED101A30
:10E58000CDED111A15F0B4FDB9F1000F0DD09DEDD0
:10E59000050AB0EEC00AB4EEE80AF1EE10FA04DDA6
:10E5A000344ACDF800803B46D1E70136B4E700237A
:10E5B00094F8806216F0010001D0012BCCD104F553
:10E5C000C0610AA8CDF828A00D950C950B9515F003
:10E5D00047FC0AA906A816F013F8DFED227AB4EE7C
:10E5E000E70AF1EE10FA05DD204ACDF800803B463F
:10E5F0002149ADE72046FFF75BFC03282DD12046DB
:10E600001AF09CFD94F88032DB0728D438BB0AA9A5
:10E6100006A803950495059515F0DCFF03A90EA83F
:10E620008DED0E0ACDED0F0A8DED101ACDED111AFC
:10E6300015F05EFDB9F1000F11D09DED050ADFED7B
:10E640000A7AB0EEC00AB4EEE70AF1EE10FA06DD7F
:10E65000084ACDF800803B46CAE70020D2E70120F7
:10E660007AE700BFC2B8323EC2B8B23E44E50908FC
:10E670004FE50908E39F090854E509082DE9F74328
:10E680001546044688460193FFF702FE019A0746A5
:10E6900038B92848284B00682946C06A10F0C2FEE5
:10E6A000019A019229462046FFF70EFF064668B3FD
:10E6B0002046FFF7FDFB94F93E12019A43B29942BE
:10E6C00007D01E4B1B4800682946C06A10F0AAFEFE
:10E6D0001CE094F82433834207D0019205F0E0F85F
:10E6E00004F0DCFF019A0028EBD12046FFF7E0FBA5
:10E6F00018B103280FD0124BE4E7134641462A46CF
:10E7000004F2544000F034FF00B107B9002630464F
:10E7100003B0BDE8F08394F87892B9F1000F01D10D
:10E72000084BCFE7134641462A4620461AF0D4FA52
:10E73000EAE700BF605E012058E5090864E50908C2
:10E7400094E5090883E5090890F82433032B01D1E7
:10E750001AF042BD0020704713B540F6783200F53C
:10E760000971044601A810F067FC20461AF0BCFBB2
:10E7700001A810F083FC02B010BD000008B50246ED
:10E78000FFF796FB10B1032806D008BDBDE808408E
:10E7900002F2544000F0ACBEBDE8084010461AF04A
:10E7A00011BD00000B4610B411462BB1032B09D04C
:10E7B00000205DF8044B70475DF8044B00F25440B4
:10E7C00000F0A2BE5DF8044B1AF000BC13B504467D
:10E7D000FFF76EFB0A46014620460192FFF7E2FF73
:10E7E00070B9084B019A1B68DB6A93F89C0038B13A
:10E7F00094F82413204602B0BDE81040FFF7D2BFC2
:10E8000002B010BD605E012070B590F89432DB0755
:10E8100086B004460D460CD403F02CF9437C242228
:10E8200002FB0300D0ED0B7AF1EE677AC5ED007ABA
:10E830003BE002A803F052FF01A92046FFF720FBAE
:10E84000E8B90CF043FF94F95032022B0646E3D1AD
:10E85000FEF7B4FE0228DFD996F8C4029FED147AC1
:10E86000B02303FB0066D4F88832D6F8B0209B1A98
:10E8700007EE903AF8EEE77A67EE877AD6E702A9D4
:10E880002046FFF7A3FF0028DBD0D4F88822039BA3
:10E89000DFED076A9DED017A9B1A07EE903AF8EEDC
:10E8A000E77AA7EEE67A85ED007A06B070BD00BF84
:10E8B0000AD7233CF0B50C4687B000F5097106462F
:10E8C00040F6DD3201A810F0B7FBA36853B9E36846
:10E8D00043B9636833B9002701A810F0CFFB38466D
:10E8E00007B0F0BD204603F0E3FF0028F3D094E822
:10E8F0000F0002AD85E80F000021284603F09AFFC3
:10E9000007460028E7D096F89432DB0704D434F0A9
:10E9100077FE192134F0B0FD95E80F0006F5217C53
:10E920008CE80F0096F8943243F0010386F8943295
:10E93000304600F073FD3EF079FA46213EF070FE5D
:10E940003EF074FA45213EF06BFE084BA2681B684E
:10E95000DB6A1A61E2685A6162689A6118F0D2FF54
:10E960000028B9D016F0F4FEB6E700BF605E0120C3
:10E9700038B5144B1B68DD6A2B6804465B68284673
:10E980009847F0B12B690BB96A69D2B1C4F88C32DF
:10E990006B69C4F89032A969002204F5217003F074
:10E9A000A1FE94F8943223F0030343F0030384F8A8
:10E9B00094323EF03BFABDE83840034A062139F074
:10E9C00003B938BD605E0120A8E5090813B5044607
:10E9D0000193FFF76DFA0328019B05D1204602B091
:10E9E000BDE810401AF082BB002002B010BD00004C
:10E9F00010B588B004460593FFF75AFA0328059B23
:10EA00004FF000000AD10690079006A802900B98DC
:10EA100001900A98009020461AF076FB08B010BDCD
:10EA200038B5044602F092FA0546D0B194F8243382
:10EA3000032B03D095F84641204638BD20461AF0F6
:10EA400083FAFF280446F5D00146284602F054FA1E
:10EA50000028EFD02146284602F04AFA0028E9D0E3
:10EA6000EAE70446E8E7000008B590F82433032BF2
:10EA700005D013F0B3FA90F90A03C0B208BD1AF03A
:10EA8000A7F9431CF9D1F4E708B590F8243383B112
:10EA9000032B03D1BDE808401AF092B933F08AF88D
:10EAA00040F64C524FF4801133F03CF84FF0FF30F9
:10EAB00008BD1846FCE7000090F82433032B01D171
:10EAC0001AF04EBE7047000090F82433032B01D19A
:10EAD0001AF076B8704700001AF0D6B810B50446A0
:10EAE0001DF0C6F82046FEF7E5FB2046BDE81040C5
:10EAF000FEF7FCBC90F824231AB1032A07D00120AA
:10EB0000704790F95002003818BF012070471AF082
:10EB100021BB000030B590F840348BB00446002B88
:10EB200064D1B0F89036DB0660D590ED957ADFEDD4
:10EB3000307AB0EEC77AB4EEE77AF1EE10FA11D57A
:10EB400090ED967AB0EEC77AB4EEE77AF1EE10FA6D
:10EB500008D590ED977AB0EEC77AB4EEE77AF1EE89
:10EB600010FA43D42046FFF7C5FF00283ED1D4ED6C
:10EB7000976ADFED207A9FED206A94ED967A0090F7
:10EB800066EEA76AD4ED957A27EE067A67EE867A66
:10EB9000FDEEE66ABDEEC77AFDEEE77A16EE903A34
:10EBA00017EE901A17EE102A06A803F0B5FD06A975
:10EBB0002046FFF779F8C8B13EF038F90546D4F899
:10EBC0005C02F9F7A9FCCDE90401D4F85802F9F781
:10EBD000A3FCCDE90201D4F85402F9F79DFC074AE1
:10EBE000CDE900010621284638F0EEFF0BB030BD1C
:10EBF000000000340000C8428096184BC0E50908A8
:10EC000090F824330BB1032B01D11AF015BE00206C
:10EC10007047000030B500F57B7304460D460FCBFE
:10EC200085E80F0094F8FC0330BD0000D0F898335D
:10EC30000B6090F894037047D0F8A0330B6090F805
:10EC40009D03704710B500F5697203460C4607CA6C
:10EC500084E8070093F8B00310BD000030B500F55C
:10EC60006D7304460D460FCB85E80F0094F8C4037E
:10EC700030BD000030B500F5866304460D460FCB6D
:10EC800085E80F0094F8400430BD000010B500F294
:10EC9000444203460C4607CA84E8070093F8500430
:10ECA00010BD00002DE9F0432DED028B8BB0054621
:10ECB0000E461746FFF7B4FE014680462846FFF78A
:10ECC00041FB0446002848D002F040F9414602F0DA
:10ECD00015F986ED000A95F93C32002B3ADD0CF06F
:10ECE000F5FCFEF76BFC012834D90CF0EFFC90F832
:10ECF000C432D5EDE47ADFED5D8A96ED000AB022EC
:10ED000002FB030095F93C32D0ED2F0A07EE103AD2
:10ED1000F4EEE87AB8EEC77AF1EE10FAB7EE008AB0
:10ED2000B8BFF0EE487A37EE201A20EE270A70EED0
:10ED3000C70A40F20E4013F013FED5EDE47AF4EE6C
:10ED4000E87AF1EE10FAB8BFF0EE487A80EE277A52
:10ED500086ED007A01233B7003E095F8203333B948
:10ED6000387020460BB0BDEC028BBDE8F08395F8FF
:10ED700024334FF00009CDF80490CDF80890CDF879
:10ED80000C9043B1032B10D0CDF81090CDF8149017
:10ED9000CDF818907CB902233B703246414605F20B
:10EDA000544001F027FB0446DBE701A928461AF08E
:10EDB000BFF80446E8E795F82433002BEBD004A90C
:10EDC0002846FFF763FF04460028E4D001A904A801
:10EDD00015F01CFE07A8CDED080A8DED091A8DED82
:10EDE000070A16F027FA04A8B0EE408A16F022FAB5
:10EDF00095F93C32002B30DD07EE903AF8EEE77AD9
:10EE000040F2544070EE670A37EE801AF5EEC00A01
:10EE1000F1EE10FA48BFDFED160AF4EE410AF1EE0A
:10EE200010FAB0EE480AC8BFB0EE601A13F098FDB1
:10EE3000B0EE408AD5EDE47A9FED0C7AF4EEC77A15
:10EE4000F1EE10FAB7EE007AB8BFF0EE477A88EE2E
:10EE5000277A032386ED007A7DE7B5EEC08AF1EECE
:10EE600010FA48BF9FED028AE4E700BF00000034BB
:10EE70000000000038B50446FFF7F6FD94F826338D
:10EE80008342054604D013F0A9F8294611F094FFF7
:10EE90002046FFF7E9FD84F8265384F82503204631
:10EEA000FFF7E2FD84F827032046FFF7EDFD04F5A8
:10EEB000607184F828032046FEF746FE84F88C0330
:10EEC00000F0CCFA04F5677284EDE40A04F566718B
:10EED0002046FFF7E7FE04F5687184F894032046A6
:10EEE000FEF74EFE04F5697184F89D032046FEF797
:10EEF0007BFE04F56D7184F8B0032046FEF7B0FE8A
:10EF000004F5727184F8C4032046FFF79BF904F5F9
:10EF1000767184F8D4032046FFF784F904F57B71F9
:10EF200084F8E8032046FEF7E7FD04F5806184F8E5
:10EF3000FC032046FFF756F984F810042046FEF73C
:10EF400093FE04F2144004F5836380ED000AC3EDE0
:10EF5000000A15F071FC04F21C4304F5846120469C
:10EF600083ED000A04F22C42FFF732FA04F58661C1
:10EF70002046FFF72BFC80B194F840349BB9012365
:10EF800084F84034204600F049FA3DF04FFF452117
:10EF90003EF046FB2046FEF7A3FE94F8403413B93A
:10EFA0002046FFF7B7FD04F244412046FEF7E0FE9D
:10EFB00084F8500438BD000037B50D46044600F013
:10EFC000E1F81DB913F00AF811F0C6FF4FF4EA7228
:10EFD00004F5097101A810F02FF894F881322BB9CB
:10EFE0002046FFF7C5FC012384F88132224B1D68BF
:10EFF000A86A03689B6998472046FEF7C1FC204633
:10F00000FEF73AFD204600F03BFA2046FFF704F8F1
:10F01000286B30B10368D4EDD80ADB6894EDD70AC9
:10F020009847D4F81C0208B155F08CFC204600F03B
:10F0300065F82046FEF74AFF94F8A83284F82403C6
:10F0400083420ED084F8A80298B10C4D0C4B0328D3
:10F0500008BF1D463DF0EAFE0A4A2B46062138F05D
:10F06000B3FD2046FFF706FF01A810F007F803B034
:10F0700030BD054DEEE700BF605E012056B50908C2
:10F080004FE50908ECE5090854E50908D0EDE47AF4
:10F090009FED057AF4EEC77AF1EE10FAB7EE000AAA
:10F0A000A8BFB0EE670A704700000034014B186833
:10F0B000704700BF805E012070470000704700006D
:10F0C0007047000000207047002070470120704703
:10F0D00003681B6E1847000000207047002070472F
:10F0E00000207047002070477047000000207047E4
:10F0F00000207047002070477047000070470000F4
:10F1000008B512F06BFF90F80A0308BD30B52DED7D
:10F11000028B9FED1A1ADFED1A0A91ED000A87B0F3
:10F1200005462D200C468DED011ACDED000A13F099
:10F1300017FC9DED011ADDED000AF0EE408A2E204D
:10F1400094ED010A13F00CFC9DED011ADDED000AAF
:10F15000B0EE408A2F2094ED020A13F001FC03A9BF
:10F1600005F52B70CDED038A8DED048A8DED050A32
:10F1700030F0F2FE07B0BDEC028B30BDC2B8323EBB
:10F18000C2B832BE10B5044654F084FCD4F80C3337
:10F190001BB1C21AB2F57A7F12D30A4A1268D26A38
:10F1A00092F89C2002B15BB9C4F80C0394F83D427C
:10F1B00012F014FF80F8054304F072FB80F825403C
:10F1C00010BD00BF605E01202DE9F0432DED028BE4
:10F1D00091ED007AD1ED037A87B08DED047AB0EE2F
:10F1E000C77AB5EEC07AF1EE10FADDE91087DDF8E6
:10F1F0004C90CDED057A0C4615461E4606DCF0EE29
:10F20000E77AF5EEC07AF1EE10FA02DD04A815F007
:10F2100087FB6B20B7EE001AFFEE000A9DED050A92
:10F2200013F09EFB6C2089ED000AB7EE001AFFEE8A
:10F23000000A9DED040A13F093FB04A888ED000A70
:10F2400015F0D4FAB7EE008A002852D00023C9F88E
:10F25000003088ED008AD4ED067A67EEA77AF4EEE6
:10F26000C87AF1EE10FA4ADB0023336085ED008A9C
:10F27000DFED3F0A96ED000A7C20B7EE001A13F08E
:10F280006FFB86ED000A95ED000A7D20B7EE001AAF
:10F29000FFEE000A13F064FB85ED000AD4ED067A58
:10F2A000129BDFED346AF1EE677AC3ED007A96EDDA
:10F2B000007AF0EEC77AF4EEE67AF1EE10FA2BD58A
:10F2C00003AB02AA01A9204613F060FF9DED018A5D
:10F2D000B0EE480A74F058F885ED000AB0EE480A1E
:10F2E00074F0A8F987ED000A07B0BDEC028BBDE809
:10F2F000F08304A815F066FA0028A7D1ABE738EE32
:10F30000670A13F08BFA86ED000A94ED087AC7EECF
:10F31000007AC5ED007AABE794ED076AC6EE077A8E
:10F32000C7ED007A96ED007AB0EEC77AB4EEE67AD1
:10F33000F1EE10FAC4D495ED007ADFED0F6AB0EE6D
:10F34000C76AB4EE666AF1EE10FAB9DCB4EE477A39
:10F35000F1EE10FAB4D6B0EEE77AB4EE667AF1EEDA
:10F3600010FAADDCF4EE677AF1EE10FABCD7A7E73D
:10F370000000000000000034FFFF7F7F1FB500F594
:10F380001D73039300F51C73029300F51B73019327
:10F3900000F51A73009300F5187200F5197300F563
:10F3A0004E71FFF711FF05B05DF804FB9FED196A80
:10F3B000D0ED846ADFED187A90ED860A66EE866AF3
:10F3C00020EE060A26EEA77A10B5BDEEC77AC0ED8C
:10F3D0007E6A80ED817A90ED857A27EE067A044682
:10F3E00067EE275A60EE277AFDEEE55AFDEEE77AE2
:10F3F000C0ED825A17EE903A002BBCBF03F50C43C8
:10F40000A033C0F80C3280ED7F7A13F03FFA84ED20
:10F41000800A10BDE02E65420000C8421FB50E4BA9
:10F420001B680446B3B1684603F058F969462046A4
:10F43000FFF720FC20B16A4600212046FEF720F8A5
:10F4400094F89432DB0705D504F52172012120469A
:10F45000FEF716F804B010BD2861012008B502F0CF
:10F4600009FBBDE8084001F0E3BD000010B580F8DD
:10F470001013044654F00EFBC4F8140310BD000032
:10F4800010B590F81033044653B154F003FBD4F890
:10F490001433C01AB0F57A7F84BF002384F8103388
:10F4A00094F8183353B154F0F5FAD4F81C33C01A59
:10F4B000B0F57A7F84BF002384F8183310BD0000B4
:10F4C00000F5AA700B4607C883E8070001207047C3
:10F4D0000023C0F89C30C0F89830C0F89430C0F8D1
:10F4E000A830C0F8A430C0F8A030C0F8AC307047E5
:10F4F00070470000024B0B604FF07C531360704765
:10F50000000048427047000010B500F5B4700C468A
:10F510000FC884E80F00204603F0D4F830B1FFF79D
:10F52000C5FD00F521700FC884E80F00204603F0E8
:10F53000C9F880F00100C0B210BD000010B504464B
:10F5400003F0F8FB204610BD10B5D0F8603104463A
:10F550005BB154F09FFAD4F86031C01A41F288339D
:10F56000984294BF0020012010BD0120FCE700005C
:10F5700013B5009303680192DB6D9847DDE9002124
:10F58000044628B90448054B0068C06A0FF04AFFDA
:10F59000204602B010BD00BF605E012058E509089A
:10F5A00013B50446019101F0D1FC2368019ADB6B8D
:10F5B000014608B190F84611204602B0BDE810405F
:10F5C0001847000090ED007ADFED0F7AB0EEC77AB1
:10F5D000B4EEE77AF1EE10FA14D590ED017AB0EEC0
:10F5E000C77AB4EEE77AF1EE10FA0BD590ED027A15
:10F5F000B0EEC77AB4EEE77AF1EE10FA4CBF012014
:10F6000000207047002070470000003410B501F062
:10F610009DFC044658B190F8461101F069FC30B1E8
:10F6200094F846112046BDE8104001F065BC00206A
:10F6300010BD00002DE9F0432DED028B8FB0036863
:10F6400000259B6B0395049505950695029502A9E7
:10F6500004469847064638B1FFF700FFDDED027A11
:10F6600027EE800A8DED020A0CF030F8FDF7A6FFB8
:10F670000746002E50D0DDED027AD4ED646A94ED99
:10F68000657A23680B9527EE877A67EEA67A8DED6B
:10F69000097ACDED0A7A0C950D955B6B0BA9204686
:10F6A00009AD98470BA9284615F00AF8012F8DEDF2
:10F6B000030ACDED040A40F2B3800CF007F890F88D
:10F6C000C432DFED5B7AB02505FB030090ED308A94
:10F6D00028EE278AB0EE480A73F056FEF0EE408A14
:10F6E000B0EE480A73F0A6FFCDED0B8A8DED0C0A43
:10F6F0000BF0ECFF90F8C43205FB030090ED2F0AED
:10F700000BA814F0FDFF09AD8DED050ACDED060A3D
:10F7100005A896BB03C885E00128CED89DED020A56
:10F72000B5EEC00AF1EE10FA7FDD07AED4F89421F1
:10F73000D4F8903107923046089315F00BF82368FF
:10F740000B950C950D955B6B0BA920469847DDED4D
:10F75000077A9DED0B7A77EE877A9DED0C7ACDEDE9
:10F76000077ADDED087A77EE877A09ABCDED087A76
:10F7700096E8030083E8030049E0236993ED000A5B
:10F78000B7EE008A38EE408A14F0BAFF04F5BC796F
:10F790008DED090A4846B0EE480ACDED0A0A14F08C
:10F7A000AFFF0BA92846CDED0C0A8DED0B0A14F026
:10F7B00087FF04F5C47603AFC4ED5F0A314684EDDC
:10F7C0005E0A384614F08CFF04F5C0788DED090A06
:10F7D0004046B0EE480ACDED0A0A14F091FF0BA99D
:10F7E00028468DED0B0ACDED0C0A14F069FF97E861
:10F7F000030084ED600AC4ED610A86E8030049460F
:10F80000404614F05DFF8DED090ACDED0A0A9DED2D
:10F81000090ADDED0A0A0FB0BDEC028BBDE8F083EA
:10F82000DDE9030185E80300F1E709950A95EEE7B4
:10F8300035FA8E3C10B590F84213044603F056FC9E
:10F840007C23C0B203FB0044D4F8A00010BD00002C
:10F85000044B026F1B68DB6A5A60426F9A60826FCA
:10F86000DA607047605E0120F0B58FB0044612F098
:10F87000B5FB002302930393049390F80A1301ABA2
:10F8800002AA054611F0DEFB04F19407D8B39DED02
:10F89000010AB5EEC00AF1EE10FA34DD02A815F047
:10F8A000DBF804F1B00684ED2C0AC4ED2D0A84EDDA
:10F8B0002E1A3946304615F0DFF804F17C01304647
:10F8C00015F08EF804F1880105A88DED050ACDED3F
:10F8D000060A8DED071A15F083F808A88DED080AC1
:10F8E0009DED010ACDED090A8DED0A1A15F0A4F877
:10F8F0000BA904F128008DED0B0ACDED0C0A8DED5E
:10F900000D1A13F0EFFC95F80A030C2303FB0050CB
:10F91000394600F5117015F063F884ED2C0AC4ED3A
:10F920002D0A84ED2E1A0FB0F0BD00002DE9F0472E
:10F930007E4B00251F682DED028BC0F89C50C0F84F
:10F940009850C0F89450C0F88450C0F88050C567F3
:10F95000C0F89050C0F88C50C0F88850C0F8B8502B
:10F96000C0F8B450C0F8B0500446F86A03688AB0D2
:10F970005B680E46984704F12809002854D054F0DB
:10F9800089F842F20F7398424ED8FB6A9FED688A5D
:10F9900093ED010A84ED1C0AD3ED020AC4ED1D0AA1
:10F9A00093ED031A484684ED1E1A13F08FFB3DF0C9
:10F9B0003DFAD4ED1E7A67EE887A054617EE900A76
:10F9C000F8F7AAFDD4ED1D7A67EE887ACDE9040137
:10F9D00017EE900AF8F7A0FDD4ED1C7A67EE887A4E
:10F9E000CDE9020117EE900AF8F796FD514ACDE9EC
:10F9F00000010621284638F0E7F894ED1E8AB0EEA3
:10FA0000480A73F0C1FC84ED650AB0EE480A73F051
:10FA100011FE84ED640A54F03DF8C4F864010AB0A4
:10FA2000BDEC028BBDE8F087A6B194ED1C0AB4EEE4
:10FA3000400AF1EE10FA0DD6D4ED1D0AF4EE600A7C
:10FA4000F1EE10FA06D694ED1E1AB4EE411AF1EE5C
:10FA500010FA67D712F0C2FA90F80B334FF00C0A85
:10FA60000AFB030303F5C473074693E8070007AED8
:10FA700086E807004FF01508B2EE028AF2EE068A19
:10FA8000304615F0D7FBB4EEC80AF1EE10FA11D5E6
:10FA900008F1FF3818F0FF0815D1304615F0CAFB01
:10FAA000F1EE047AB4EEE70AF1EE10FA1CDC2567F9
:10FAB000656731E0304615F0BDFBB4EEE80AF1EEC3
:10FAC00010FAE5DCE9E7384611F07AF9384611F02A
:10FAD00043FA97F80B330AFB037303F5C47393E8F7
:10FAE000070086E80700CBE7DDED098A9DED088A6F
:10FAF0009DED070A68EEA80AE8EE080AF1EEE00AB2
:10FB000073F064FEF1EE680A84ED1D0AB1EE480A56
:10FB100073F05CFE84ED1C0A9FED071AD4ED1D0AFC
:10FB200094ED1C0A484613F0D1FA66E7605E0120A6
:10FB3000E02E654260E70908000000000021FFF7A1
:10FB4000F5BE000037B5044608461546019115F08C
:10FB500071FBB7EE007AC7EE007AB4F8D0300198A6
:10FB60000133A4F8D03094ED337A37EE277A84ED60
:10FB7000337AB0EE007AF4EEC77AF1EE10FA06D5D9
:10FB8000B6EE007AF4EEC77AF1EE10FA0DDC9FEDD6
:10FB90000E7AF4EEC77AF1EE10FA13D59FED0B7AD8
:10FBA000F4EEC77AF1EE10FA0CDDB0EE670A14F04D
:10FBB00043FF012085ED000AC5ED010A85ED021A1B
:10FBC00003B030BD0020FBE700247449BD37863503
:10FBD00070B52DED028B00F1280600F134058AB0D6
:10FBE00029460446304614F0A3FFB6EE008A20EE04
:10FBF000088A2846B0EE480A14F01EFF07A93046CE
:10FC0000CDED080A8DED091A8DED070A14F0FEFE00
:10FC100030468DED010AB0EE480ACDED020A8DEDB9
:10FC2000031A14F009FF07A928468DED070ACDED48
:10FC3000080A8DED091A14F0E9FE04A901A88DED5A
:10FC4000040ACDED050A8DED061A14F085FF324643
:10FC500001A920468DED070ACDED080A8DED091AA0
:10FC6000FFF770FF58B953F015FF0121C4F8600188
:10FC70002046FFF75BFE0AB0BDEC028B70BD2A4642
:10FC800004A92046FFF75EFF0028ECD004F14002F3
:10FC900007A92046FFF756FF0028E4D0EBE7000055
:10FCA00030B52DED028B0D4683B091F8421304461A
:10FCB000284603F01BFAC1B27C2000FB01519031B1
:10FCC00004F1280013F092F868468DED000ACDED9E
:10FCD000010A14F0B1FDDFED1C7AB4EEE70AF1EE93
:10FCE00010FA05D59FED190A03B0BDEC028B30BDAB
:10FCF000684614F015FE684614F078FD0028F1D12E
:10FD0000284694ED428A03F059FBF0EE400AB0EE2B
:10FD1000480A12F04FFD80B9284603F04FFB84EDEE
:10FD2000420AB0EE408A73F02FFB84ED430AB0EE36
:10FD3000480A73F07FFC84ED440A04F58671684636
:10FD400014F032FDD0E700BF0000003400000000D6
:10FD50009FED0C7AB4EEC70AF1EE10FA0BD4DFED8A
:10FD60000A7AB4EEE70AF1EE10FA07DCC0EE077A81
:10FD7000B0EE670A7047F7EE007AF9E7F2EE047A20
:10FD8000F6E700BFF3665F3F58A00B4108B51C3093
:10FD900014F052FDF1EE007AB4EEE70AF1EE10FA3B
:10FDA0009DBFF1EE027A37EEC00ADFED047A9FEDD7
:10FDB000040A98BF20EE270A08BD00BFCDCC4C3EF8
:10FDC000CDCCCC3D08B5836993F9000038B10BF078
:10FDD0007DFCFDF7F3FB012894BF0020012008BD46
:10FDE000F8B52DED028B054603F05AFD03F056FCE5
:10FDF0000446B8B3FFF75AF990F8213393B3284675
:10FE0000FFF7E0FF064668B30BF060FC90F8C432E1
:10FE1000B02707FB030090ED2F7AF0EE087AB4EEDE
:10FE2000E77AF1EE10FA1DD495ED1E8A0BF04EFC28
:10FE300090F8C432DFED1E7A07FB030090ED300A24
:10FE400098EE270A12F038FDDFED1A7AB0EEC00AFC
:10FE5000B4EEE70AF1EE10FA08DC53F01BFE34466C
:10FE6000C5F85001BDEC028B2046F8BD05F5AA701F
:10FE700015F0E0F9B0EE408A0BF028FC90F8C4329F
:10FE80009FED0D7A07FB0303D3ED2F7A67EE877A98
:10FE9000B4EEE78AF1EE10FADFD553F0FBFDD5F8AA
:10FEA0005041001BB0F5FA6F8CBF00240124D9E744
:10FEB000E02E654200003442CDCC4C3F10B50A4BD9
:10FEC0001B68DB6A93F89C3004465BB953F0E2FD93
:10FED000D4F86431C01A44F61F6398428CBF0020E6
:10FEE000012010BD0020FCE7605E0120F8B52DED7B
:10FEF000068B04460BF0EAFB054603F0D1FC0646F0
:10FF000005F0A0FD002840F0AA802046FFF768FF1A
:10FF1000002800F0A7803046FFF78CFCD4F8DC30D6
:10FF2000984200F018813046FFF784FCD4F8DC30AA
:10FF3000DFED8E7AC31A08EE903AF8EE688A304602
:10FF400068EEA78AFFF776FC94F8BC30C4F8DC00B2
:10FF5000F3B9304603F0B4FBD0B104F1280796F8AA
:10FF600042233946304603F02DFAD4ED1D0AB0EE97
:10FF7000401A384694ED1C0A13F0A8F80023C4F880
:10FF80009030C4F88C30C4F88830012384F8BC3039
:10FF900020463146FFF784FE95F8C40205EB0015B4
:10FFA000B0EE408A2B6FC4F8E03004F1B000D4ED1D
:10FFB000129A15F03FF96368DFED6D7A93ED007AE0
:10FFC000B4EEE77AF1EE10FA68EE299AB0EE40AAA4
:10FFD00001D5C3ED007A2046B0EE4A0AFFF7B8FE1D
:10FFE000636820EE299A93ED000A29EE009AFFF744
:10FFF000CDFE29EE009A204684ED249AFFF75EFF9D
:020000040802F0
:1000000038B1D4ED247AB2EE007A67EE877AC4ED87
:10001000247AF0EE007AF4EEE78AF1EE10FA10D5C9
:10002000DFED547AB4EEE7AAF1EE10FA09D5DFED70
:10003000527A69EEA79AD4ED2A7AE9EEA87AC4ED4D
:100040002A7A9FED4E0A94ED367ADFED4D7AB0EEC6
:10005000C88A28EE008AA7EE278A84ED368ABDEC8E
:10006000068BF8BDFFF722F890F82133002B72D0F1
:100070002046FFF7A7FE00286DD095F8C42205EBB7
:100080000213196FD4F8E0308B4264D0B02606FB1F
:10009000025292ED2F7AF0EE087AB4EEE77AF1EEA2
:1000A00010FA58DBCB1AC4F8E01008EE903A95F835
:1000B000C4329FED341A94ED1E0ADFED337A06FB4D
:1000C0000353D3ED309A69EE819AF8EE688A39EEDF
:1000D000C00A68EEA78A12F02FFCB0EE409A73F0C7
:1000E000A9FA94F8BC30B0EE408AF3B1F3EE047A8A
:1000F000F4EEE78AF1EE10FA17DC95F8C40206FB7D
:10010000005595ED2F7AF2EE027AB4EEE77AF1EE31
:1001100010FAFFF64AAFDFED1D7AB0EEC99AB4EEE1
:10012000E79AF1EE10FAFFF640AF9FED198AD4ED91
:100130001D0A94ED1C0AB0EE691A04F1280012F0B1
:10014000C5FF012384ED248A84ED238A84ED228A6D
:1001500084F8BC3029E7BDEC068B04F188009FEDE4
:100160000D0ABDE8F84014F0BBBC00BFBD378635B2
:10017000CDCC4C3DC2B8B23E0AD7233CCDCC4C3E90
:10018000CDCC4C3F35FA8E3C6F12833A1904863F32
:1001900000000000EC51783F30B50C2303FB010157
:1001A00001F1C003144693E807008BB004AD85E865
:1001B000070094E8070083E807002846FFF702FAE3
:1001C00007AB58B194E8070083E807009DED070AE4
:1001D000DDED080A9DED091A0BB030BD95E807006A
:1001E000F2E70000F0B52DED028BD0F818318B60EE
:1001F000D0F81C31CB6085B004460D4601F03AFCC6
:1002000006460BF063FAA36993F90030022B074608
:100210004BD1FDF7D3F9022847D997F8C432B02261
:1002200002FB0373D3F8B0100022284602F05AFAFA
:10023000D4ED4A0A94ED490A284602F067FD94F885
:100240002C3163B353F026FC9FED228A97F8C41239
:100250008DED018A01AA064638460AF0B5FAD4F8AF
:1002600020019FED1D0A361A07EE906AF8EE677AB4
:1002700040F23C4027EE800AB6EE001AF0EE480A43
:1002800012F06EFBDDED017A30EE270A04F1F0008A
:100290008DED010A14F034FA284602F037FD94F887
:1002A0002C0105B0BDEC028BF0BD707C242303FB58
:1002B000006696ED0B8AFEF7F9FED0EDA27A9FED6F
:1002C000077AF8EEE77AE8EE077AFDEEE77A17EEBE
:1002D000901AA9E7000000006F12833A0000C8429C
:1002E00030B589B0044668460D4602F0F7F9694614
:1002F0002046FFF709F918B90024204609B030BD9F
:1003000004A802F0EBF9204604A9FFF76BFF0446AE
:100310000028F1D004A9684602F000FC85ED000A2F
:10032000C5ED010A85ED021AE7E700001FB50023BD
:100330000C4601A9019302930393FFF7D1FF08B183
:10034000039B236004B010BD30B585B001AD002320
:100350000C462946019302930393FFF7C1FF03461E
:1003600018B195E8030084E80300184605B030BDD5
:10037000F8B52DED028B06460F46154600F0E6FD5A
:100380000446A0B1394600F0B3FD80B1204639469D
:1003900000F0B2FD044650B100F0D8FD394600F03F
:1003A000ADFD85ED000ABDEC028B2046F8BDFEF7E1
:1003B0007DFE90F82033B7EE008A7BB13046FFF720
:1003C00001FD044650B1D6ED538AFFF747F8C8EE59
:1003D000007A67EEA87AC5ED007AE4E7D6ED538A95
:1003E000FFF73CF8C8EE007A002467EEA87AC5ED66
:1003F000007AD8E770B52DED048B1646FFF7B8FFED
:10040000054670B3FEF752FE90F93C424CB30BF038
:100410005DF9FDF7D3F8012823D9E4B207EE904A3D
:10042000B8EE678A0BF052F990F8C43296ED009A54
:10043000B02202FB0300D0ED2F8AFFF70FF838EE51
:10044000281A78EEC80A40F2654029EE000A12F038
:1004500087FAB0EE408AFFF701F8C8EE007AC6EDE1
:10046000007ABDEC048B284670BD000038B50D46FF
:100470000BF02CF90446FDF7A1F8022881BF94F88F
:10048000C402B02303FB0040D43089BF07C800205A
:1004900085E80700012038BD30B585B000230D4642
:1004A00001A9019302930393FFF7E0FF044620B1F3
:1004B000039B2B60204605B030BD01F0DBFA417C88
:1004C00000F092FF04460028F4D001F0D3FA00F0C7
:1004D00051FEB1EE400A85ED000AEBE7F8B5036F77
:1004E0004B60436F8B60836FCB6000F14C070C4611
:1004F000054601F110060FCF0FC60FCF0FC63B68A0
:10050000336005F1280104F1340013F0A9FC2346FF
:10051000012203F8442B05F1B00207CA83E8070063
:1005200005F1940207CA04F1500383E8070005F1BE
:100530001C0207CA04F15C0383E8070004F174019C
:100540002846FFF793FF04F1840184F880002846D1
:10055000FFF7A2FF04F18C0184F888002846FFF71A
:1005600041FE84F89C00F8BD08B503F099F9BDE898
:10057000084003F093B8000010B5044614F008FBDF
:1005800050B904F10C0014F003FB28B904F1180071
:10059000BDE8104014F0FCBA012010BD38B500F1E0
:1005A000280504462846FFF7E7FF28B12046012129
:1005B000BDE83840FFF7BAB9D4ED107AB7EE007A4B
:1005C000F4EEC77AF1EE10FA06D5BFEE007AF4EE3B
:1005D000C77AF1EE10FA12DC2046FFF7F9FA284646
:1005E000FFF7CAFF0028E1D1D4ED107AB2EE047A09
:1005F000F0EEE77AF4EEC77AF1EE10FAD6DC38BD09
:1006000010B5044614F016FE2046BDE8104014F064
:100610007BBA00002DE9F04F2DED048B9FEDCA8AC7
:1006200095B00446F0EE408A8DED028A8DED038A86
:100630008DED048AFFF75AFC11F0D0FC002305462B
:1006400095F87921012AA8BF012293423FD20021C7
:10065000284610F01DFB01230028F1D008AB0BAA9F
:10066000002128468DED0B8A8DED0C8A8DED0D8ACB
:1006700010F042FD9DED080AB5EEC00AF1EE10FA49
:1006800023DD0BA814F0E8F911A904F128008DED81
:10069000110ACDED120A8DED131A12F04BFB0EA8C4
:1006A0008DED0E0AB0EE680ACDED0F0A8DED101A31
:1006B00014F0C2F911A904F1E4008DED110ACDED99
:1006C000120A8DED131A14F0D7F90123B8E795F843
:1006D0000B130C2303FB015104F1280B01F5C4712A
:1006E000584612F027FB84ED070A94ED3F0AC4ED4B
:1006F000080A70EE288A84ED091AC4ED3F8A0AF0D0
:10070000E5FF0646FEF7D2FC90F821330193204620
:10071000FFF758FB80B13046FCF750FF02280BD999
:1007200096F8C4226169B02303FB026391F90010BB
:1007300093F8D200884263DA94ED3F7ADFED837A52
:10074000B4EEE77AF1EE10FA61D4D4ED538AFEF7F5
:100750005DFF58B100F0FAFB90F8461100F0CEFBB7
:10076000F0EE408AFEF77AFE60EE288A236C626B18
:10077000A16A1393B0EE680A11A81292119114F0B5
:100780005BF904F5AA7102A88DED020ACDED030A0A
:100790008DED041A14F070F953F07CF9002307462C
:1007A00084F814312046FFF70DFB002865D096F839
:1007B000C422B02302FB033232445268C4F8182129
:1007C00096F8C42202FB033333449B68C4F81C31FF
:1007D00053F060F90123C4F8200184ED498A84EDC7
:1007E0004A8A84F82C31D4F80031002B58D102AB5E
:1007F00093E80700C4F80071F03484E8070006E0CD
:1008000006EB0212176FD4F80021BA4204D115B0DA
:10081000BDEC048BBDE8F08FD43393E8070094F867
:1008200014310DF1080C8CE807001BB904F1F0033A
:1008300083E807000123604684F8143104F5AA71A7
:1008400014F0E4F811A904F14C008DED110ACDED7E
:10085000120A8DED131A12F09BFAB5EEC00AF1EEF2
:1008600010FA8DED110AD8BF9FED370ACDED120AAF
:100870008DED131A84ED530A94E794ED3F7AD4ED8D
:10088000497ADDED026AE6EE877ADDED036AC4EDB2
:10089000497AD4ED4A7AE7EE267AC4ED4A7AA2E79D
:1008A000D4ED3F7A254B8DED058AF5EEC07AF1EE59
:1008B00010FA8DED068A0793A9D9214B9FED217A75
:1008C0001B68DB6A67EE877A93F89CA0B7EE007A24
:1008D000C7EE279ABAF1000F4AD094F8143113B931
:1008E000019B002B42D0E36804F1F001D3ED008AB4
:1008F00002A814F08BF869EEA88A8DED110A11A8F0
:10090000B0EE680ACDED120A8DED131A14F094F8CA
:100910000EA905A88DED0E0ACDED0F0A8DED101A6A
:1009200014F0AAF805A8FFF76BFE05A814F04AF921
:10093000F0B153F0AFF8C4F8600168E7000080BF81
:10094000605E01200AE81C4100000000CDCC4C3E56
:10095000CDCC4C3FCDCC4C3D920A06BF920A063F0F
:10096000C2B8B23E728A0E3C5B821839DDF804A030
:100970005FED0B8A0023CDE90833CDE90A33CDE9D9
:100980000C334FF0FF32009204F1E40895F879211E
:10099000012A1046A8BF0120834255D20123002A14
:1009A000FAD095F82D130029F6D0B0EE690A40462A
:1009B00014F096F80DF12C09BAF1000F3FD0424621
:1009C00000212046FFF7E8FB8DED0B0ACDED0C0A68
:1009D0008DED0D1A4846FEF7F5FD70BB4846FFF752
:1009E0000FFE484614F0EEF838BB05A9484614F04F
:1009F000B3F805A94846CDED090A8DED0A1A8DED2B
:100A0000080A14F095F808A8B0EE409A14F012FC09
:100A1000009B33B9F4EEC08AF1EE10FAD8BFB0EE05
:100A2000680AB5EEC09AF1EE10FAF7EE008A4FF0C0
:100A3000000358BFF0EE408A00930123A6E798E830
:100A4000070089E80700C5E7009B002B7FF471AF22
:100A5000002384F804312046FFF7C2F938B120465C
:100A6000FFF7B0F9002840F025818DED0A8A95F84E
:100A70000A3395F878219A4240F233812B4493F857
:100A80002C33002B00F02D8195F80B3395F879214C
:100A90009A4240F226812B4493F82D33002B00F02C
:100AA000208108A9584612F073F98DED080ACDEDA2
:100AB000090A8DED0A1A08A814F06AF8002840F017
:100AC000178108A814F07EF8002840F011815FED2E
:100AD000617A94ED357A68EEA78A5FED637AE7EE86
:100AE000278A04F1B000C4ED358A14F0A3FBA36893
:100AF0005FED687A93ED007AB4EEE77AF1EE10FAE2
:100B0000F0EE408A00F1F8802046B0EE680AFFF768
:100B10001FF908A813F090FFA3688DED110ACDED21
:100B2000120A8DED131A93ED000A11A813F084FF39
:100B3000204684ED1F0AC4ED200A84ED211AFFF738
:100B4000BDF928B1B2EE000A04F17C0013F0C8FF31
:100B5000019BB3B33046FCF731FD012831D996F83B
:100B6000C402B02303FB006696ED2F7AF0EE087AFC
:100B7000B4EEE77AF1EE10FA23D595F80B030C23C7
:100B800003FB005595ED627AF1EE0C7AB4EEE77A4C
:100B9000F1EE10FA15DBD4ED1D7A1FED917AF4EE2B
:100BA000C77AF1EE10FA0CDD1FED947AF4EEC77AF5
:100BB000F1EE10FA05D5B6EE000A04F17C0013F050
:100BC0008FFF5FED997AF4EEE78AF1EE10FA22D505
:100BD0001FED9C0A08A813F02FFF0EA88DED0E0A3A
:100BE00094ED3F0ACDED0F0A8DED101A13F024FF9E
:100BF00011A904F1A0008DED110ACDED120A8DEDC1
:100C0000131A13F039FFD4ED2B7A94ED3F7A77EE77
:100C1000877AC4ED2B7A94ED2B7AF1EE047AB4EE58
:100C2000E77AF1EE10FA3BDB11F0D8F95FEDB27A1A
:100C300094ED2B1A94ED280A21EE271A40F2C930C0
:100C4000F1EE410A8DED011ACDED000A11F088FE9A
:100C50009DED011ADDED000A84ED280A40F2CA304C
:100C600094ED290A11F07CFE9DED011ADDED000ADC
:100C700084ED290A40F2CB3094ED2A0A11F070FE7F
:100C800004F1A00184ED2A0A04F1940013F0F4FEAB
:100C900084ED2A8A84ED298A84ED288A84ED2B8AC2
:100CA0000023C4F8E430C4F8E830C4F8EC3084ED34
:100CB0003F8A9CE5E368F7EE000A93ED000A11F025
:100CC00079FD00283FF4D1AE94ED1C0AB0EEC00AC5
:100CD00072F0B0FCDDED0A7A27EE800A8DED0A0A8B
:100CE000C5E68DED0A8A8DED098A8DED088AE2E66A
:100CF0002046FFF753FC1CE6C3ED007A04E700BF73
:100D00002DE9F04D2DED0E8BA0B0044611F066F9E3
:100D1000D0EDC67A90ED618AF4EE487AF1EE10FAE1
:100D200048BFB0EE678ADFED677AB4EEE78AF1EE8E
:100D300010FA0EDD0023C4F8E430C4F8E830C4F83B
:100D4000EC300023C4F8FC3020B0BDEC0E8BBDE8C5
:100D5000F08D2046FEF788FD2046FEF739FFB0EE05
:100D6000480A2046FFF756FC2046FFF717FCFEF71F
:100D70009DF916AD00F53A7204F1280116A812F09B
:100D800057F80FCD04F14C060FC60FCD0FC62B68D8
:100D9000336004F1740204F1780304F1700104F18A
:100DA0004C0012F0F3F994ED1E8AB0EE480A72F08E
:100DB000EBFA84ED650AB0EE480A72F03BFC20467F
:100DC00084ED640AFEF744FDFEF770F904F5B47192
:100DD000FDF750FF52F05EFED4F89831C31A632B32
:100DE000B2D9C4F8980132F00BFC9FED378A054662
:100DF00052F058FED4ED1C7A67EE887A074617EE5B
:100E0000900A0E46F7F788FBD4ED1D7A67EE887AD4
:100E100041EC1D0B17EE900AF7F77EFB94ED1E0ACE
:100E200020EE080A41EC1C0B11F030FDD4F8D40080
:100E300010EE108AF7F770FB8246D4F8D8008B4684
:100E4000F7F76AFB41EC180BD4F85401F7F764FB91
:100E500041EC190BD4F85801F7F75EFB41EC1A0B83
:100E6000D4F85C01F7F758FB94ED53EA41EC1B0B07
:100E7000FEF7F4FACEEE007A17EE900AF7F74CFB85
:100E8000CDE9140140468DED12BB8DED10AB8DED1B
:100E90000E9B8DED0C8BCDE90AABF7F73DFB0B4BB1
:100EA00001930B4B0093CDE908018DED06CB8DED41
:100EB00004DBCDE90276074B074A0849284632F0A1
:100EC00027F941E7CDCC4C3EE02E654265C00908CC
:100ED000BBC009088CE7090897E7090854E5090829
:100EE00070470000002070477047000000207047E6
:100EF0000020704700207047002070479FED010AD6
:100F0000704700BF000000009FED010A704700BF5E
:100F100000000000002070477047000010B5044634
:100F2000143000F019F804F12C0000F015F804F169
:100F3000700053F097FD04F1F00053F093FD4FF073
:100F4000FF33C4F84C31204610BD0000014B186837
:100F5000704700BF845E01207047000008B52DED8A
:100F6000048BB0EE609AF0EE408A00F00FF9B0EE1C
:100F7000408A89EE280A72F093FCDFED0B7A20EEAE
:100F8000270A72F025FCDFED097A38EE278ADFEDBB
:100F9000087A28EE278AF7EE007A37EEC00A28EEA4
:100FA000000ABDEC048B08BD41D3423E3393884315
:100FB000A1D81943FFF7D2BF08B52DED048B9FEDE3
:100FC000179AF0EEE07AF4EEC97AF1EE10FAF0EE4C
:100FD000408AB0EE608A04D5B7EE000ABDEC048BFF
:100FE00008BD00F0D3F8DFED0E7A9FED0E7ADFED4D
:100FF0000E6A70EE277A9FED0D0AE8EEC77A27EEAB
:10100000800A88EE007AC6EE877AF4EEC97AF1EEAD
:1010100010FAE1DBB1EEE70AE0E700BF00000034C0
:1010200033938843F4FDD43BCDCC9C3F48A18F4300
:10103000427CD0ED257A242101FB020292ED0B0ABD
:10104000D2ED090A30EE270AFFF7B6BF38B52DED0D
:10105000088BDFED21AA9FED21AA9FED21BA05465D
:10106000B0EE409AF0EE609AB0EE408A1524013C52
:10107000A4B25CB3F0EE490A2846B0EE480AFFF786
:101080006DFFF0EE490A70EE698A284638EE2A0AAA
:10109000FFF764FFB0EEE87A70EE697AB4EECA7AD0
:1010A000F1EE10FA77EEE87A10D468EEAA8A40F2F0
:1010B000631088EEA70AB0EE4B1A38EE400AF0EE45
:1010C0004A0A11F04DFCB0EE408AD0E7B0EE480A73
:1010D000BDEC088B38BD00BFCDCCCC3D0AD7233C3E
:1010E00000247449002343608360C360036143614B
:1010F0008361C361002380F82030704790F820207E
:10110000531CDBB2062B80F8203000EB820288BF34
:10111000002382ED010A88BF80F82030704700006C
:101120004FF0FF3310B543610E4BC0F8A8300023D9
:10113000044680F8C830A830FFF7D4FF0A4BC4F843
:10114000A83004F5867051F003FE084B08491C6076
:1011500020462DF0D3FFD4F89030C4F894302046C8
:1011600010BD00BFB0E90908C0E90908885E012088
:1011700058EA090808B5A83033F070FADFED027AB2
:1011800020EE270A08BD00BF00007A4490ED3C0A1B
:10119000DFED057AB0EEC07AB4EEE77AF1EE10FA40
:1011A00048BF90ED3D0A70470000003473B5D0F899
:1011B000A43004460E4663B152F06CFCD4F8A4305F
:1011C000C01A42F20F73984203D894ED280A02B075
:1011D00070BD114B1D687DB195F846112846FFF78B
:1011E0008BFE48B195F8461101AA2846FFF77AFE12
:1011F00010B19DED010AEAE7242101FB064494EDBC
:101200000A0ADFED067AB4EEE70AF1EE10FA58BFEB
:10121000B0EE670ADBE700BF845E012000000C42ED
:1012200008B561B10378022B02D9064852F002FCDE
:101230005A1C027000EB83004160012008BD084683
:10124000FCE700BF78E809082DE9F84305460E469B
:101250009146002400F13C082B7CA34211DD0023C1
:101260004A46314601200DF063FD242363430746BF
:10127000002158F803000DF06BFD874204D00134C3
:10128000EAE70020BDE8F8830120FBE770B50B46D4
:10129000064614469AB111469847054628B9236870
:1012A00020465B68BDE87040184701463046FFF7AE
:1012B000B7FF20B92B6828465B689847EFE770BDF9
:1012C000F0B50D4685B011461A46CDE90213044625
:1012D000FFF7BAFF034698B90A4800684068042738
:1012E0000668CDE90037DDE902123668064BB047E3
:1012F00002462946204605B0BDE8F040FFF7C6BFCC
:101300000022F6E7605E0120801A06007FB5D0ED6E
:10131000247A9FED2B7AF0EEE77AF4EEC77A012378
:10132000F1EE10FA0446037609D49030002303A9A5
:10133000019003932EF0C2FC01982EF0B7F8002222
:1013400076232049E2632266C4F884202046FFF712
:10135000B7FF2378032B30D0237C032B2DD0D4F878
:101360000031DA0403D5637E0BB9012363760025CF
:10137000637EEB40DB07EAB20BD40135082DF7D1D1
:1013800023781BB1237C0BB16368B3B90E4801F01D
:101390008DF93820019201F0C5FC064618B1019A7A
:1013A000214653F06BFE31462046FFF739FF237884
:1013B000032B02D0237C032BDFD104B070BD00BF10
:1013C000000000342D4C070894E80908054B1B6801
:1013D0002BB141694A1C02D0184632F0DBB800201C
:1013E000704700BF2861012002290BD8242303FB8A
:1013F000010191F8390030B191F83A0018B191F833
:101400003B007047002070472DE9F047044652F03A
:1014100041FBD4F8F86042F21073861B9E4288BFED
:10142000C4F8F80000274FF0240942F2107A237C18
:10143000FDB2AB421CD929462046FFF7D5FF70B15B
:1014400009FB054898ED0D0AD8ED097AD4ED250A77
:1014500030EE270A2046FFF7F9FD88ED0C0A5645C5
:1014600004D909FB054030302EF020F80137DEE7C3
:10147000617C2046FFF79AFE84ED3D0ABDE8F087C7
:1014800070B52DED028B044686B052F003FBD4F804
:101490009830C31AB3F57A7F05463FD33C4B94EDA1
:1014A000257A1B689FED3B8ADB6AD4ED247A93F89A
:1014B0009C60F0EEC76AF4EEC86AF1EE10FA22D52D
:1014C000F0EEE76AF4EEC86AF1EE10FA1BD502A856
:1014D00001F004F916BBFDF7E9FD02A9FDF7CAFB0F
:1014E000E0B1DDED037A9FED2C7AF8EEE77A67EE56
:1014F000877AB0EEE77AB4EEC87AF1EE10FA11D43A
:10150000C4ED257A11E077EE676AB7EE006AF0EE77
:10151000E66AF4EEC66AF1EE10FA1EDC06B0BDEC27
:10152000028B70BD1D4BC4F89430C4F89850FDF781
:10153000BDFDFDF711F92046FFF766FF3BF076FC95
:101540000546D4F89400F6F7E7FF154ACDE9000107
:101550000621284636F038FBE0E7F0EEE76AF4EEC5
:10156000C86AF1EE10FAD9D4002EC9D020469030C6
:1015700080ED007A2DF09AFF3BF058FC094A0121DA
:1015800006B0BDEC028BBDE8704036F01DBB00BF5D
:10159000605E0120000000340AD7233C6F12833ABA
:1015A000DDE80908B8E80908F0B52DED048B85B031
:1015B000044640F2723200F5867103A80DF03CFD3E
:1015C000D4ED227AD4ED236A9FED796A637C37EEFD
:1015D000E67A2422B0EEC77AB4EEC67AF1EE10FABB
:1015E000C1BF9FED747A67EE877A9FED737AE6EE5E
:1015F000877A02FB03430025C4ED237A93F8396010
:101600002378E9B28B4206D904EB8103013558688F
:1016100000F09EFAF4E7DFED698A9FED698A9FED9D
:10162000699A0027237CFDB2AB4264D9242303FBD3
:10163000054393F83920002A5BD0D3ED0C7AF4EE01
:10164000E87AF1EE10FA0BDBF4EE677AF1EE10FABD
:1016500006D6F0EEE77AF4EE487AF1EE10FA04DD01
:10166000242303FB05435A6A1A63242303FB05431F
:10167000D3ED090AD3ED0D7A93F8382070EEA70A5E
:10168000A2B993ED0C0A2046FFF794FCD4ED257A1D
:1016900030EE670AB4EE400AF1EE10FA16D72423B2
:1016A00003FB0545002385F83A3022E0012A09BFF3
:1016B000D3ED0C7A93ED0B0A77EEE00AD4ED3B7A8A
:1016C00004BF80EE897A87EE270AE3E7F0EEC07A5E
:1016D000F4EE487A2423F1EE10FA03FB0545E1DC31
:1016E000012385F83A30D4ED237A37EE800A85ED70
:1016F0000B0A013796E7627C20461146FFF774FE1D
:1017000048B1242101FB024292ED0B0AD16904F198
:10171000A80032F083FF94F99C10277C002907DB96
:10172000B94205DACAB211462046FFF75DFE68B934
:1017300000226274D5B2AF4209D929462046FFF78C
:1017400053FE01320028F5D0657400E06274204633
:10175000FFF796FE2046FFF739FE10B1204653F002
:1017600019FC637C242505FB034393F83930B3420D
:1017700016D031F045FF4FF6FF7131F00BFF78B115
:10178000607C05FB004494F83930002B14BF002224
:101790000422019231F034FF019A122131F08CFEC3
:1017A00003A80DF06BFC05B0BDEC048BF0BD00BFD1
:1017B0000AD7233C0AD7A33C48E17A3F0000003413
:1017C000FFFF7F7F002019462DE9F04F0446007C83
:1017D0000F4687B004F13A0300220121D5B2A84296
:1017E00003F1240305D903F8231C03F8241C013258
:1017F000F4E76F4B1E68F06A03685B68984740B176
:101800003BF014FB6B4A062107B0BDE8F04F36F001
:10181000DBB93BF00BFB684A062136F0D5F9002313
:1018200003A904F1880003932EF048FA0A2552F028
:1018300031F980462046FFF7B7FE52F02BF9A0EBB6
:101840000800B0F5FA7F02D95C4800F02FFFB06ABB
:1018500003680A215B689847617C2046FFF7C4FD56
:101860000028E7D0B06A036864215B68013D9847AF
:1018700015F0FF05DBD1524B05951B888DF80650FE
:10188000CDE90355ADF80430052552F003F9804643
:101890002046FFF789FE52F0FDF8A0EB0800B0F5F6
:1018A000FA7FD1D8617C2046FFF79EFD0028EFD05B
:1018B00094F810B00DF10C08A14601AA4FF0000AEF
:1018C0005FFA8AF18B4516D92046FFF78DFD50B19E
:1018D000D8ED007A99ED097A137877EE877A01339B
:1018E000C8ED007A13700AF1010A08F1040809F141
:1018F00024090132E4E7B06A036864215B68013DB2
:10190000984715F0FF05C0D1A9464FF02408237C65
:101910005FFA89F6B34226D906AB334413F8143C78
:1019200033B908FB064686F83B3009F10109EEE7BA
:10193000002FFAD007EE903A06AA02EB8602F8EEE4
:10194000E77A12ED030AD4ED250A204680EE270A35
:10195000FFF77CFB08FB064002A930308DED020A40
:101960002EF0ACF9E1E7617CDFF85C902046FFF7F0
:101970001DFC002684ED3D0A4FF02408237CF7B2BD
:10198000BB420FD908FB074393F83B3043B13BF010
:101990004DFA7B1C4A46062136F016F90135EDB2A8
:1019A0000136EBE70DB907484FE707B0BDE8F08F08
:1019B000605E0120F8E8090823E9090839E9090807
:1019C000709D090875E9090853E9090808B5037C01
:1019D000022B02D9034852F02DF85A1C0274184603
:1019E00008BD00BF94E9090838B5057C024600240B
:1019F000E1B28D4206D91046FFF7F6FC013400280B
:101A0000F6D138BD281E18BF0120FAE770B50D4683
:101A100009780729044606D8027E437E22B90122AE
:101A20008A401343437670BD002BFCD000262278F9
:101A3000F3B29A42F7D904EB830329465868036846
:101A4000DB6898470136F2E737B50D460192FFF79C
:101A5000CBFF0199044630B90448054B00682A467B
:101A6000C06A0DF0DFFC204603B030BD605E01208F
:101A700047E00A08014B1868704700BF885E0120E4
:101A80007047000073B543681B7C8B4205460C46CB
:101A900042D900F10801212201A80DF0CDFA51F040
:101AA000F9FF6A68242303FB0423D969411AB1F5BD
:101AB000FA7F33D2196A401AB0F5FA6F2ED2D3EDFD
:101AC000097A9FED177AF0EEE77AF4EEC77AF1EE35
:101AD00010FA54BF01200020242606FB04F31A4408
:101AE0009FED107A82F8390069680B44D3ED0A7AC9
:101AF000F4EEC77AF1EE10FA06D49FED0B7AF4EE0D
:101B0000C77AF1EE10FA04DD06FB0411002381F818
:101B1000393001A80DF0B2FA02B070BD0020DBE749
:101B200000000034000048C30000484310B5044BD7
:101B30000446C0E90031083051F00AF9204610BDD2
:101B400050EB09084368242000FB0131CA63704749
:101B500013B50368019104469B689847236801996F
:101B60001B69204602B0BDE810401847F8B52DEDBE
:101B7000028B43681B7C8B4205460C46F0EE408A84
:101B8000B0EE608A1FD951F085FF24276B68674348
:101B90003B4493ED090AF0EE680A064610F00AFE8F
:101BA000A0B96B68242202FB04331E626B682421F7
:101BB0004C432344C3ED098A6B68234483ED0A8AAE
:101BC00069680C44E661BDEC028BF8BD6B683B4470
:101BD00093ED0A0AF0EE480A10F0ECFD0028E0D080
:101BE000E4E70000DFED2A7AB0EEC07AB4EE677A5F
:101BF000F1EE10FA49DCB4EE400AF1EE10FA44D6E8
:101C0000436893F9FC3063B190ED087ADFED217AF7
:101C1000F0EEC76AF4EEE76AF1EE10FA03D580ED54
:101C2000080A01232BE077EE407A37EE006AF0EEE7
:101C3000E77AC7EE866ADBB29FED176A07EE903A45
:101C400026EE866AF8EE677AB4EEE76AF1EE10FAED
:101C50009FED126A15DDF2EE047A66EEA76A436A1A
:101C6000C6EE267A013343620023F7EE006A76EE71
:101C7000E76A27EE800AA7EE260A80ED080A1846D2
:101C80007047F0EE467A0123EFE70023F7E700BF45
:101C9000FFFF7F7F0000003400004843CDCCCC3DE7
:101CA00090F83C35934207D900EB8200D0F8140538
:101CB00010B103689B6A1847002070472DE9F34173
:101CC00005466E4686E80C00134B45F8043B044677
:101CD0000F4600F5C87828462C3500F00FFCA845C3
:101CE000F9D196E8030004F5A863C4F8387583E8D1
:101CF0000300089BC4F84835084920462DF0FEF93A
:101D0000074B1A6812B1074851F094FE20461C6038
:101D100002B0BDE8F08100BF38ED090800EC090809
:101D20008C5E012064EB09082DE9F74F90F83C65C3
:101D30000446002E4DD17F2380F84C3500F5C87540
:101D400000F21458071D5FFA86F91822FF21284671
:101D500073F0FAFE85F8589097F924A0BAF10A0FAB
:101D60004DD039DCBAF1040F0FDCBAF1020F0FDDF0
:101D7000442000F0D7FF834620B13B462A46214647
:101D800053F01AFAC8F800B002E0BAF1090F2AD0ED
:101D9000D8F8000050B1296EC5F85CA031B1254BD0
:101DA00043F826102DF0B8FB2DF0AEFB58F8040BCD
:101DB00009F101095FFA89F920B103689B68984726
:101DC00084F83C950136092E05F1640507F12C07CE
:101DD000B9D103B0BDE8F08FBAF1190F1DD0BAF137
:101DE0001F0FC5D0D4E7382000F09CFF83460028A1
:101DF000C8D03B462A46214653F056FEC2E7302063
:101E000000F090FF83460028BCD0CDF800903B4600
:101E10002A46214653F0E2FFB4E7482000F082FF53
:101E200083460028AED03B462A46214654F048F867
:101E3000A8E700BF905E012090F83C358B4283BF3D
:101E4000642303FB010090F8D501002070470000D7
:101E500090F83C358B4283BF642303FB010090ED77
:101E60006A0A9FED010A70470000000090F83C35B7
:101E70008B4206D900EB8100D0F8140508B153F06D
:101E80004DBB9FED010A70470000000010B490F8B0
:101E90003C458C420A4614D900EB8104D4F8144521
:101EA0007CB1E468246A640603D55DF8044BFFF74F
:101EB000DDBF642101FB020393ED6A0A5DF8044B68
:101EC00070479FED010AF9E70000000090F83C35EB
:101ED0008B420BD900EB8100D0F8140538B1C368F0
:101EE0001B6A1A4214BF012000207047002070476F
:101EF00070B590F83C35934204460E46154601D81D
:101F0000002070BD00EB8203D3F814050028F7D041
:101F100003689B6998470028F2D0642202FB0544BD
:101F2000D4F8AC313360ECE770B590F83C359342AF
:101F300004460E46154601D8002070BD00EB820312
:101F4000D3F814050028F7D003689B699847002848
:101F5000F2D0642202FB0544D4ED6C7AF4EE677A89
:101F6000F1EE10FAE8D6C6ED007AE6E770B590F823
:101F70003C35934204460E46154601D8002070BDFC
:101F800000EB8203D3F814050028F7D003685B69DF
:101F900098470028F2D0642202FB0544D4F8B431FB
:101FA0003360ECE790F83C3593420ED900EB8203A6
:101FB000D3F814355BB1642303FB020292F8E40109
:101FC00030B1D2F8E0310B607047002070471846FE
:101FD0007047000008299DBF2C2303FB01004068C7
:101FE000002070472DE9F04F4B4B2DED028B1B6805
:101FF000DB6A93F89C3089B00446002B00F08680A1
:10200000DFF82CB19FED458A4FF0000994F83C357C
:102010005FFA89F5AB4279D904EB8503D3F814054F
:1020200000285DD003685B6B9847642303FB05437E
:10203000074693F8D431834252D2032861D8DFE8AF
:1020400000F04F025259364E4FF000083AF0EEFEC3
:1020500094F83C25AA4284BF642202FB05424FF05B
:10206000640105F1010301FB05458CBFD2F8A821ED
:1020700018EE102A8246D5F8B001CDE90632F6F7FF
:102080004BFA079ACDE904011046F6F745FA069B8C
:102090000096CDE902015A460421504635F094FDE0
:1020A0000123204A84F84D3585F8D471D372D4F8D1
:1020B00048354BB3002255B25957481C03D041450F
:1020C00002F10102F7D194F94C35AB4208DBD4F8A8
:1020D0004435D4F8400542463146984784F84C557B
:1020E00009F1010992E72C2303FB05430E4E93F9F6
:1020F0002B80ABE72C2303FB05430C4E93F92C807C
:10210000A4E70026B046A1E71D46DCE709B0BDEC18
:10211000028BBDE8F08F00BF605E01200000000070
:1021200091EB09080D5F01202EEC0A0888EB0908E5
:10213000A0EB090890F83C358B4207D900EB8100F1
:10214000D0F8140510B10368DB6918470020704708
:1021500008299CBF642303FB010000F5C870704789
:1021600090F83C35934207D900EB8200D0F8140573
:1021700010B103685B6A1847002070472DE9F04FE3
:10218000002493B005460E46174621462F2206A886
:10219000059405F2145973F0D7FC05F1280A4FF0A5
:1021A0002C0B05F5F6730BFB04F259F8040B1AF926
:1021B0000210E5B230B951B90134092CF3D14FF016
:1021C000010813E0642262439A58914212D01548E4
:1021D000154B006801930135EDB20095134BC06AB1
:1021E000324639460DF01EF94FF00008404613B054
:1021F000BDE8F08F05A93322039353F071FA039BD6
:10220000804605A90028D7D1064801910135EDB2D5
:1022100000680095054BC06A324639460DF002F958
:10222000E4E700BF605E01200DF70908C8EB09086C
:102230002DE9F04FDFF88090DFF880A0DFF880B064
:102240008DB00646002796F83C35FCB2A3422ED945
:10225000642505FB046595F8DC3133B395F8DD1191
:1022600019BB4FF001082022444404A889F81980C2
:1022700073F06AFC07EE904A4AF21043F8EEE77AF0
:1022800003AA4C21ADF8283050462423CDED037A23
:1022900035F0ACFA3AF0CAFD9BF80030054A0094DC
:1022A000042135F091FC85F8DD810137CBE70DB0D5
:1022B000BDE8F08FD8EB09080D5F0120A96101206E
:1022C000CD2201202DE9F04F2F4B1E6885B004462A
:1022D00046B1D0F83815304631F05CF910B13046CF
:1022E00030F004F851F0D6FB4FF0000801904FF0A9
:1022F0002C0A4FF0640B94F83C355FFA88F5AB423A
:1023000039D904EB8507D7F8140588B30AFB0543D0
:102310000BFB054993F92820D9F8EC118A4227D103
:1023200032B30268D2689047D7F814050268126B7E
:10233000904799F8D52112B1019BC9F8D831BEB1A7
:10234000D4F83815304631F025F988B151F0AAFBA0
:10235000CDE9021002460B46D7F81405294653F082
:10236000B7FBDDE90232D7F81405294653F026FC05
:1023700008F10108BFE72046FFF734FE204605B00C
:10238000BDE8F04FFFF754BF286101202DE9F04769
:102390004FF000082DED028B04468946B0EE408ACE
:1023A000474601264FF0640A94F83C355FFA88F5F9
:1023B000AB421AD929FA05F3DB070AD504EB8503EA
:1023C000D3F8140578B10368B0EE480A9B6B9847C0
:1023D00006400AFB054508F1010895F8D4319F42F3
:1023E00038BF1F46E0E70646F3E727B97F23A4F886
:1023F0004C35034BDF72BDEC028B3046BDE8F087F5
:102400000D5F012090F83C358B4207D900EB81002D
:10241000D0F8140510B10368DB6B18470020704733
:102420000B46114690F83C259A4207D900EB8300F1
:10243000D0F8140510B103681B6C184770470000F2
:1024400070B504460E46002594F83C35E9B28B423F
:1024500005D932462046FFF7E3FF0135F4E770BDAA
:102460002DE9F84390F83C550246002400F1280677
:102470002C2700F5F6784FF06409E1B28D420FD9B0
:1024800007FB04F309FB04F0F35658F800008342FD
:1024900009D11BB11046FFF7CFFC10B10134ECE7B6
:1024A0000120BDE8F8830020FBE7000010B590F89C
:1024B0003C258A42044617D9642202FB010393F8A3
:1024C000D431022B03D004D9032B18BF00231846A4
:1024D00010BDFFF797FF48B92046FFF7C1FF00285E
:1024E0000CBF06230123F2E70023F0E70623EEE703
:1024F000014B1868704700BF8C5E012010B503497E
:1025000004462CF0FBFD204610BD00BFB8ED0908C5
:1025100010B50446203044F08FF9044B04491C6088
:1025200020462CF0EBFD204610BD00BFB45E01201C
:1025300028EF0908F7B5B7EE000A00220221044689
:102540002CF0CCFB204653F023FD44F063FA144BEF
:102550001D680646E86A03685B6A98470B460221D5
:1025600002460091304644F07DF9B4F94A60002EED
:1025700014DDEF6A3B6838465B68B4B2984728B10F
:1025800097F84D3013B1C92EA8BFC824A86A0368B4
:102590005B68214603B0BDE8F040184703B0F0BDCA
:1025A000605E012010B5044653F0A8FC2046BDE84B
:1025B000104053F0D3BC00002DE98048284BDFF8D1
:1025C000A490DFF8A4A0DFF8A4B01446012293B0D1
:1025D00005460E461A704FF0000851F05BFAD9F824
:1025E00000300393A0EB080241F287339A4207467A
:1025F0001FD9CDE9005603985346342205A9C06A75
:102600000CF010FF214605A8049450F01FFCCDE902
:10261000005603985B46342205A9C06A0CF002FFFD
:1026200004943AF003FC049B05AA022135F0B4FAA5
:10263000B8463AF0FBFB39F0F7FC3AF0F7FB3BF019
:1026400039FB0A2105A80CF0DDFC039B986A03689E
:1026500005215B68984705A80CF0E0FCBDE700BFCA
:10266000B85E0120605E0120A8EE09088D010B080C
:102670000FB400B595B016AA002152F8043B03929E
:1026800005A83C220193049173F05EFA054A019B70
:10269000402104A850F082FB039A034804A9FFF7E5
:1026A0008BFF00BFB0EE0908C6EE09080FB407B5EE
:1026B00004AA034852F8041B0192FFF77DFF00BFF4
:1026C000D8EE090808B50449102273F0E3F9B0FA0E
:1026D00080F0400908BD00BFBC5E0120102200212F
:1026E00073F032BA0378416023F00D03022A0370BD
:1026F00008D0032A0AD0012A03D1DBB243F0010338
:1027000003707047037843F00803F9E7037823F078
:10271000050343F00503F3E773B504460E4615467B
:102720000193FFF7DBFF2046C4E90265069A019991
:10273000FFF7D8FF02B070BD4B6843600A7803789A
:1027400062F3000303700B780278C3F3800363F332
:10275000820202700B78D2B2C3F3C00363F3C302E8
:10276000027070470078420704D4030704D400F0D5
:10277000010070470320704702207047F0B585B014
:1027800005461646FFF7EEFF88420F4605D16B68F7
:1027900033600124204605B0F0BD032801D1002498
:1027A000F8E70329FBD001280BD0022816D018BB6C
:1027B0006D68012F22D0022F2ED0002FEFD135606F
:1027C000E7E7FCF773FC90F89432DB07E7D56D6818
:1027D000FCF76CFCD0F888321D44EAE76846FFF746
:1027E0007DFFFCF763FC6946FCF744FA04460028C9
:1027F000D0D06D68019BEFE70025DAE7FCF756FCC7
:1028000090F8944214F00104C9D0FCF74FFCD0F8C2
:102810008832ED1A3560BDE76846FFF75FFFFCF7C9
:1028200045FC6946FCF726FA04460028B2D0019B15
:10283000EFE7000073B501AA05460E46FFF79EFFBD
:10284000044620B1019932462846FFF74BFF204647
:1028500002B070BD13B5144601AAFFF78FFF48B14F
:10286000DDED017A9FED047AF8EEE77A67EE877A7C
:10287000C4ED007A02B010BD0AD7233C07EE900ADF
:102880009FED090AF8EEE77A08B527EE800A70F0A6
:102890007BFDDFED067AB4EEE70AF1EE10FAD8BF61
:1028A000B0EE670A08BD00BF50E0EF300AD7233C06
:1028B00010B50446806810F0DBF920B1E068BDE88F
:1028C000104010F0E9B910BD73B5856804460E4696
:1028D0001DBBC36823B98B688360CB68C3600125C7
:1028E000636873B92378DB070BD52046FFF73AFFFF
:1028F00001AA01463046FFF741FF10B1019B63601A
:1029000005462046FFF7D4FF20B9B368A360F368FB
:10291000E3600125284602B070BD0025E0E7000015
:102920000D4B83424FF000038B4106DA00F1255036
:1029300000F5311000F5E0507047084B98424FF019
:10294000FF3371EB0303BEBF00F1564000F51300E7
:1029500000F52440704700BF00D2496B002EB694AA
:1029600090EA010F01D4401A7047C317401A63EB75
:10297000E1710D4B83424FF000038B4106DA00F109
:10298000255000F5311000F5E0507047074B984294
:102990004FF0FF3371EB0303BEBF00F1564000F56B
:1029A000130000F52440704700D2496B002EB69406
:1029B00070B52DED028B84B0044668460D46FFF7D6
:1029C0008DFEFCF773FB6946FCF754F9064608B325
:1029D000A368029ADFED128A03999B1A07EE903AD8
:1029E000F8EEE77A67EEA87AC5ED007AE068FFF7BF
:1029F000B7FF08EE100AA068024402EBD272B8EEEC
:102A0000C88A5010FFF73AFF28EE288A28EE000AFD
:102A100085ED010A304604B0BDEC028B70BD00BFED
:102A2000F67C8E3F37B500230C4601AA02210546ED
:102A30000193FFF7A3FE10B9002003B030BD21467B
:102A40002846FFF7B5FF0028F6D0DDED017AF8EE55
:102A5000E77AC4ED027AF0E710B52DED028B8468B9
:102A60008A680B46111B08EE901AC168D868FFF7F8
:102A700077FF224402EBD27208EE100A5010FFF7E3
:102A8000FDFEB8EEC88AF8EEE88A28EE000A20EECD
:102A9000000AA8EEA80ABDEC028BB1EEC07A9FED49
:102AA000020A27EE000A10BD8262363CF0B52DED19
:102AB000028B0D4689B08C680646D0E90271E86841
:102AC000FFF74EFF08EE100AE01900EBD07040103F
:102AD000FFF7D4FE73686A689FED0E1A9B1A07EE23
:102AE000903AE41BB8EEE77AF0EE400A07EE904A1F
:102AF0009FED090AB8EEC88AF8EEE77A28EE008A58
:102B000027EE011A27EE800A68EE200A09B0BDEC14
:102B1000028BF0BD0AD7233C8262363C84B004B0FD
:102B2000FFF7C4BF38B52DED028B0C460246C168D5
:102B3000E068FFF715FF9568A46808EE100A6019B1
:102B400000EBD0704010641BFFF798FE07EE904A30
:102B5000F8EEE77AF8EEC80A87EE807ABDEEC70A8B
:102B600010EE103A5B4200EE103AB8EEC00A70F078
:102B70002DFEDFED087A30EE270ABDEC028BB5EEB4
:102B8000C00AF1EE10FA44BFDFED037A30EE270AF7
:102B900038BD00BFDB0FC93FDB0FC94030B52DED9D
:102BA000028B0B4685B08C68D0E90251D868FFF7DC
:102BB000D7FE08EE100A601900EBD0704010FFF746
:102BC0005DFE641B07EE904AF0EE400AB8EEC88A3C
:102BD0009FED060AF8EEE77A28EE008A27EE800AD3
:102BE00068EE200A05B0BDEC028B30BD8262363C37
:102BF00082B002B0FFF7D2BFF0B52DED028B0B46CD
:102C00008F68D0E9025185B0D868FFF7A9FE7B191B
:102C100003EBD37304465810FFF730FE781B10EE19
:102C2000106AF5F767FC14A3D3E90023F5F7CCFC91
:102C3000F5F7C2FF08EE100A2046F5F75BFC0EA37D
:102C4000D3E90023F5F7C0FC044630460D46F5F7FE
:102C500063FC02460B4620462946F5F7B5FCF5F71E
:102C6000ABFF00EE900AB0EE480A05B0BDEC028B57
:102C7000F0BD00BFAFF300800000004050CC863FA5
:102C8000094B984206DDC0F1D64000F5930000F5EF
:102C9000A4407047054B9842BEBFC0F1144000F5F8
:102CA000360000F53850704700E9A43500175BCABC
:102CB000F8B52DED028BDFED148A076820EE280AA7
:102CC0000646FDEEC07A0D4617EE904A04EBD4702E
:102CD00007EB6000B0EE608AFFF7D0FD28EE288A8F
:102CE0003819C8EE007AFFF7CBFF306017EE900A74
:102CF000F6F73CF92B68C01841EBE371FFF710FEC3
:102D0000BDEC028B2860F8BD02AAB34200F10C01B1
:102D10000830FFF7CDBF00000148FFF7DFBC00BF60
:102D2000BC5E01200121884238BF08466EF078BBA6
:102D3000FFF7F8BF08B16EF077BB7047FFF7FABF37
:102D4000F8B506460F46144622B96EF06DFB2546CF
:102D50002846F8BD10461EB9BDE8F8406EF030BBFD
:102D60006EF02EFB05460028F2D0BC4222463146CA
:102D700028BF3A4672F09EFE30466EF055FBE7E7FC
:102D800037B504460846089D11461A460368019562
:102D90009DF81C5000951D68069BA84720602046A2
:102DA00003B030BD00214FF0FF3310B500220363A4
:102DB000044601600171C0F80510417280F82510C9
:102DC00000F13C0300F50B70D9709A60DA601A616B
:102DD0005A619A61DA611A625A629A62DA631A6413
:102DE0005A649A64DA641A655A659A65DA65DA662D
:102DF0001A675A677C339842E6D1214604F516706B
:102E000006F006FE044B1A6822B904491C602046ED
:102E10002CF074F9204610BDCC5E012080F1090829
:102E200073B5D0F83C3201919942044613D0D0F8E2
:102E30004032994218D0D0F844328B4216D1022049
:102E40000AE0D4F8343253B3D4F838324BB34FF0ED
:102E5000030002B070BD002094F822308342F8D8FD
:102E6000431C84F82230F4E70120F5E7D0F8306203
:102E7000002EE6D194F841233546B6009AB1A31945
:102E8000C3F83012A319019AC3F83C2294F82230F7
:102E9000AB429CBF6B1C84F822302846D9E7012640
:102EA000E8E70226E6E704F50C7001A930442DF0AE
:102EB00013F8E7E738B504460D462CF083FF291DCB
:102EC000201D2CF07FFF05F1080104F108002DF012
:102ED00053F805F1140104F114002DF04DF805F13B
:102EE000200104F120002DF047F805F12C0104F138
:102EF0002C002CF0FBFE05F1300104F130002DF028
:102F000003F805F13C0104F13C002DF035F8AB6B02
:102F1000A3636B6B636338BD2DE9F043A1B000235D
:102F2000002500F13C0706468DF8075003930493F3
:102F3000059306930793089309930A930B931093B1
:102F40001193129313931493159316931793189345
:102F50001C931D931E9300F50F78B94658F8043B57
:102F6000F3B1F26E934223D0D6F8E820934221D0F9
:102F7000D6F86421934213D10221EBB299420FD0CB
:102F8000C1EB411109EB8104214601A8FFF792FF33
:102F900039462046FFF78EFF01A93846FFF78AFF22
:102FA0000135032D07F17C07D8D121B0BDE8F083AE
:102FB0000021E2E70121E0E72DE9F04704460E4653
:102FC0001546804607464FF0000A31462046FFF777
:102FD00027FF7A6FB2425FFA8AF90ED1C3B2022B91
:102FE0000BD87C2202FB0A44012084F83E0084F8BE
:102FF0003F3085F80090BDE8F0870AF1010ABAF188
:10300000030F07F17C07E0D1002731462046FFF788
:1030100007FFD8F86C205FFA87F912B9C3B2022B08
:1030200019D90137032F08F17C08EED1314620462B
:10303000FFF7F6FEC2B2C2EB421304EB830393F830
:103040003E7067B9022A0BD8012083F83E0083F84E
:103050003F202A70CFE77C2000FB0744C4E700270D
:103060004FF07C0904F13E0A31462046FFF7D8FEB6
:10307000034609FB07F05FFA87F81AF8002012B937
:10308000DBB2022B09D90137032FEDD194F82300CD
:1030900004280BD9144850F0CDFC0444012084F8D6
:1030A0003E0084F83F3085F80080A4E704F54377BC
:1030B000002157F8043BB342CAB208D1904202D86B
:1030C000531C84F8233003322A70002093E73BB965
:1030D000411C04EB800084F82310C0F80C63F2E775
:1030E00001310529E5D1F0E7B8EF0908C9B200EBD5
:1030F0008101D1F83C3253B1026F93420AD0D0F82B
:10310000EC20934208D0D0F86821934206D04FF0CB
:10311000030070470020704701207047022070476D
:103120002DE9F8430F469146044600F5BA7894F825
:103130003E5035B97C344445F9D100252846BDE8D8
:10314000F88300234A46394601200BF0F1FD0021A7
:103150000646E06E0BF0FCFD8642EBD1EEE7000088
:10316000012303FA01F1D0F8083319420AD14AB118
:1031700090F82030032B1FBF591C80F8201000EB63
:1031800083004261704700002DE9F043DFF87C8046
:1031900085B0044600F50F7600257C27B14656F829
:1031A0000C3CD9F800209342E9B206F1040619D18B
:1031B000C3B12046FFF79AFFC0B207FB004090F86A
:1031C0003E307BB903A9A9F10C0003932CF084FED7
:1031D00039F02CFE56F8043C009342462B46012160
:1031E00034F0F2FC0135032DD8D104F16C0504F55F
:1031F000F074296821B9AB6813B128462BF014FA92
:103200007C35A542F5D105B0BDE8F083D4EF0908BF
:1032100038B504461546FFF769FFC0B2022808D842
:103220007C2303FB004029465030BDE838402CF099
:1032300093BE38BD38B504461546FFF757FFC0B2F8
:10324000022808D87C2303FB004029465C30BDE8F7
:1032500038402CF081BE38BD37B50D4604468DEDA3
:10326000010AFFF743FF022D07D8C0B27C2303FBFE
:10327000004001A968302CF021FD03B030BD0000F2
:1032800038B50546FFF732FFC4B2022C13D8C4EBA1
:103290004414A4003C3504F10800284400212BF01C
:1032A000C3F904F1340104F1300029442844BDE895
:1032B00038402CF011BE38BD70B505460E46144698
:1032C000FFF714FFC3B2022B0DD87C2000FB035381
:1032D00094E80700443383E8070031462846BDE8F8
:1032E0007040FFF7CDBF70BD37B504461546FFF7F8
:1032F000FDFEC0B2022809D87C2303FB00400DF17B
:10330000070140308DF807502CF05CFD03B030BD54
:103310001FB590F92C30044623B390F921300BB33C
:103320006846FFF7DBF9FBF7C1FE6946FBF772FC65
:10333000C0B1DDED037A9FED0C0AF8EEE70ADDED92
:10334000027AF8EEE77A0123C0EE800A84F83D3372
:1033500087EE800A06F0AEFDDFED047A20EE270A44
:1033600084ED0A0A04B010BD8096184B35FA8E3CE5
:10337000024690F9210058B192F8400340B111443F
:1033800091F92C0220B192F92400033818BF0120D2
:103390007047000038B590F8223005465BB1002434
:1033A0002346E1B22846FFF7E3FF08B10133DBB261
:1033B0000134032CF5D1184638BD000090ED0A0AFF
:1033C0007047000038B50C46D1ED066A1146054637
:1033D000FFF78CFEC3B27C2000FB0353D4ED087AC8
:1033E000D3ED260A94ED076AD3ED255A93ED245ABE
:1033F00026EE600A67EEA00AA5EEA70AF0EE607A54
:10340000E5EE867AB7EE007AA6EEE67A67EEE60A91
:10341000B1EE400AE5EE070A70F0D8F99FED071A01
:10342000DFED070A40F658000FF09AFAD5ED0A7A58
:10343000BDE8384030EE270A0FF07EBADB0F494076
:10344000DB0F49C02DE9F04190F822308B42044651
:103450000D4602D20020BDE8F081FFF747FEC0B262
:1034600004F13C06C0EB401006EB8000083011F080
:10347000E1FEDFED157AB0EEC00AB4EEE70AF1EE38
:1034800010FAE7D429462046FFF730FEC5B27C206B
:1034900000FB05473B6F002BDCD0032DDAD000FB8F
:1034A00005603030D7F86C802BF0FEFED7E91B3278
:1034B000934201D1984505D07C2000FB0544C4F817
:1034C0006C80C7E70120C6E7000000342DE9F74F04
:1034D00004460E46174600F50F7A4FF0000B5AF8D7
:1034E000049B5FFA8BF8B9F1000F26D041462046C5
:1034F000FFF73EFF08B341462046FFF7F7FD7C2368
:10350000C0B203FB004090F83E505DB908F10103E2
:103510001B4ADBB2394630464FF040FC284603B028
:10352000BDE8F08F5AF8102C914506D0154A39465F
:1035300030464FF033FC0025F0E70BF1010BBBF1F7
:10354000030FCCD14FF0000894F822305FFA88F1D5
:103550008B420DD920460191FFF774FF054620B933
:1035600001992046FFF704FF20B908F10108EBE7B5
:103570000125D3E7044A394630464FF00FFCCDE72A
:10358000FCEF090811F0090836F009082DE9F041AF
:103590002DED048B90F842139FED348ADFED348AD1
:1035A0009FED349A82B00646FFF7A0FD06F13C0776
:1035B000C5B27C2000FB057554354FF0000896F825
:1035C00022205FFA88F39A424ED919463046FFF717
:1035D000CFFE10B908F10108F1E719463046FFF7B0
:1035E00085FDC4B27C2000FB0474D4ED157AF0EEA6
:1035F000E77AF4EEC87AF1EE10FA04F154040ED52D
:10360000D4ED017AF0EEE77AF4EEC87AF1EE10FA32
:1036100005D5002002B0BDEC048BBDE8F081294641
:10362000204611F017FEB4EEE80AF1EE10FAF0DCD5
:103630002946204611F00CF9B4EEC90AF1EE10FA51
:10364000E7DC2146284611F04BF868468DED000A6C
:10365000CDED010A11F0F0F8DFED077AB4EEE70ADC
:10366000F1EE10FAB6DDD4E70120D3E70000003414
:10367000DB0FC93F920A863F00004843022910B57C
:10368000044608D8FFF732FD7C23C0B203FB004498
:1036900094F83D0010BD0020FCE7000013B590F841
:1036A000421301910446FFF7E9FF30B1019920462A
:1036B00002B0BDE81040FFF75BBE02B010BD0000D5
:1036C000F7B590F921500446002D73D090F840537F
:1036D000002D6FD090F84213FFF7D0FF94F83D33E0
:1036E000064613B92046FFF713FE002594F8202064
:1036F000EBB29A4207D904EB83030135586903689A
:103700009B689847F2E750F0C5F90027224604F578
:10371000BA7140F2F315D2F89C30C31AAB428CBF99
:103720000023012382F83D307C32914247EA0307AF
:10373000F1D194F92430032B07D194F83C33002BBA
:103740003BD0D4F83803002849D167B1236B01334B
:1037500009D02FF055FF216B2FF01CFF18B12FF06F
:103760004FFF2EF0D7FE94F92C32002B3AD194F96A
:103770002D32CBBB94F92E3213B1022384F842339D
:1037800094F842132046FFF779FF8642054611D090
:103790002FF036FF4FF6FF712FF0FCFE50B1002DD9
:1037A00014BF0022042201922FF02AFF019A032164
:1037B0002FF082FE284603B0F0BD012384F83C338D
:1037C0000420FFF7AFFA054610B1214606F0C0F914
:1037D00094F92430C4F83853032BB2D0B5E706F07F
:1037E000D1F9B2E70023C9E70123C7E738B590F95B
:1037F00021300446D3B190F84053BDB1FFF776FCB9
:10380000C0B2022812D87C2303FB0044D4ED1A7AFC
:103810009FED087AF4EEC77AF1EE10FA06D4B7EE0F
:10382000087AF4EEC77AF1EE10FA00DD002528469A
:1038300038BD00BFABAA2A3F70B5D0F8085315F4C5
:10384000003504460E460DD190F840335BB90A7836
:10385000072A07D8012303FA02F290F83F331343F3
:1038600080F83F3370BD94F82020EBB29A42F9D92A
:1038700004EB8303314658690368DB6898470135D8
:10388000F1E7000038B505466C242B591BB1002127
:1038900028192AF0C9FE7C34B4F5F07FF5D138BD83
:1038A000014B1868704700BFCC5E012010B504467C
:1038B000006810B103685B689847204610BD00009F
:1038C00010B50446006810B103685B68984720464D
:1038D00010BD000010B50446006810B103685B68B5
:1038E0009847204610BD00002DE9F04FD0F808534E
:1038F0008DB015F4807B9DF858909DF85CA004462F
:103900000F461646984660D1FFF70AFC0546002888
:103910003FD0CDE906BB069B04934FF0000B424617
:1039200039462046CDE905BBFFF7FAFB06460028DD
:103930003DD0CDE90ABB0A9A089200234A4608A95D
:10394000CDE9093304A8534600F042FF074608A812
:10395000FFF7C0FF09A8FFF7BDFF0AA8FFF7B0FFF8
:1039600016B10BA8FFF7ACFF04A8FFF7B3FF05A83B
:10397000FFF7B0FF06A8FFF7A3FF15B107A8FFF7F1
:103980009FFF3A46082120460DB0BDE8F04FFFF7F3
:10399000E7BB04230E49CDE9010309680D4B0093F1
:1039A000496833463A4606A8FFF7EAF9B3E7042325
:1039B0000749CDE901030968064B0093496843466E
:1039C0003A460AA8FFF7DCF9B5E70DB0BDE8F08F7D
:1039D000605E0120801A06002DE9F04F9146012417
:1039E000D0F808238BB08C40144098469DF854A022
:1039F0009DF850309DF858B006460F4635D11A460E
:103A000041460593FFF78CFB059B054600B3CDE9C6
:103A10000844089A069200235A46514606A8CDE962
:103A20000733C847044606A8FFF754FF07A8FFF767
:103A300051FF08A8FFF744FF15B109A8FFF740FFA1
:103A40002246394630460BB0BDE8F04FFFF788BB41
:103A500004220749CDE901020968064A0092496833
:103A6000424608A8FFF78CF9D3E70BB0BDE8F08F0A
:103A7000605E0120801A06002DE9F04FB04BDFF8A0
:103A8000CC921D6804466868036889B09B689847B3
:103A9000002607464FF001084FF0080A08FA06F31F
:103AA0003B4240F02D820136202EF7D16868DFF8C6
:103AB0009CA20368DB689847002607464FF001097F
:103AC0004FF0060809FA06F33B4240F02B8201361C
:103AD000202EF7D16868DFF8789203689B689847D2
:103AE000002607464FF001084FF0080A08FA06F3CF
:103AF0003B4240F028820136202EF7D168680368E7
:103B00009B6898470026804601274FF01A0907FA5C
:103B100006F313EA080F40F026820136202EF6D174
:103B200068680368DB689847002607464FF0010A7B
:103B30004FF01A09B0460AFA06F33B4240F02E82D3
:103B40000136202EF7D16868DFF808920368DB6839
:103B50009847002607464FF0010AB0460AFA06F3D6
:103B60003B4240F036820136202EF7D16868DFF8FC
:103B7000E4910368DB689847002607464FF0010A86
:103B8000B0460AFA06F33B4240F033820136202E5B
:103B9000F7D16868DFF8BC9103689B6898470026F6
:103BA00007464FF001084FF0020A08FA06F33B42BD
:103BB00040F02F820136202EF7D16868DFF894910B
:103BC00003689B689847002607464FF001084FF0AE
:103BD000020A08FA06F33B4240F02B820136202EFF
:103BE000F7D16868DFF8709103689B6898470026F2
:103BF00007464FF001084FF0060A08FA06F33B4269
:103C000040F02E820136202EF7D16868DFF8489107
:103C10000368DB689847002607464FF0010AB04664
:103C20000AFA06F33B4240F02B820136202EF7D1F0
:103C3000444BDFF82891079307AF04264FF00C0A96
:103C4000686803689B6898474FF0000805904FF03C
:103C5000010B059A0BFA08F3134240F0218208F198
:103C60000108B8F1200FF4D168680368DB68984751
:103C70004FF0000805904FF0010B059A0BFA08F37E
:103C8000134240F01E8208F10108B8F1200FF4D170
:103C9000013E16F0FF0607F10107D1D16868DFF891
:103CA000C0A003689B6898474FF001080746B146DB
:103CB00008FA06F33B4240F017820136202EF7D176
:103CC0006868DFF89CA00368DB6898470026074611
:103CD0004FF00109B04609FA06F33B4240F0148266
:103CE0000136202EF7D16868DFF878A003689B685A
:103CF0009847002607464FF00108B14608FA06F338
:103D00003B4240F011820136202EF7D16868DFF87F
:103D100054A00368DB689847002607464FF0010966
:103D2000B04609FA06F33B4240F00E820136202EDF
:103D3000F7D16868044B079303689B68984713E0C2
:103D4000605E01200C0D0E0F20212223C16A0208A3
:103D5000E17A0208417202085D4702080D7002080C
:103D6000256D0208B5770208BA4A804600264FF052
:103D7000010909FA06F313EA080F1AD00DF11C0A1B
:103D80000427F3B24FF0000B1AF8011B0091CDE9A4
:103D9000019B102120460593FFF71EFE94F8231087
:103DA000052900F0BC80013F17F0FF07A94A059BD9
:103DB000EAD10136202EDCD168680368DB689847B9
:103DC000A44A804600264FF0010B0BFA06F313EAD3
:103DD000080F1AD00DF11C090427F3B24FF0000AA6
:103DE00019F8011B0091CDE901AA10212046059385
:103DF000FFF7F2FD94F82310052900F09080013FB1
:103E000017F0FF07934A059BEAD10136202EDCD13B
:103E10006868DFF848A203689B68984700278046D7
:103E20004FF0010909FA07F313EA080F15D010261D
:103E3000FBB24FF0000B5246CDE9019B00960321E7
:103E400020460593FFF7C8FD94F82320052A66D085
:103E50000136F6B2142E059BEDD10137202FE1D1AA
:103E60006868DFF8F4A103689B68984700278046DC
:103E70004FF0010909FA07F313EA080F15D01426C9
:103E8000FBB24FF0000B5246CDE9019B0096152185
:103E900020460593FFF7A0FD94F82320052A3ED085
:103EA0000136F6B2182E059BEDD10137202FE1D156
:103EB0006868694E0368DB689847002780464FF0C2
:103EC000010A0AFA07F313EA080F15D014255FFA5E
:103ED00087FB4FF000095B46CDE90199009532461A
:103EE00015212046FFF778FD94F82330052B16D0D6
:103EF0000135EDB2182DEED10137202FE1D10EE0C2
:103F00001E230093CDE9018AF3B24A4600212046E0
:103F1000FFF762FD94F82330052B7FF4C4AD09B0A0
:103F2000BDE8F08F1E230021CDE90031CDF80880D7
:103F3000F3B252462046FFF74FFD94F82330052B8D
:103F40007FF4C5ADEBE70D230093CDE9018AF3B211
:103F50004A460C212046FFF73FFD94F82330052BFD
:103F60007FF4C9ADDBE7F1B26923CDE900790C221A
:103F700020460591FFF7B8FC94F82330052BCED0EE
:103F80006823CDE9007905990C222046FFF7ACFCA7
:103F900094F82330052B7FF4C0ADC0E7F1B269235C
:103FA000CDE900890C2220460591FFF79DFC94F88D
:103FB0002330052BB3D06823CDE9008905990C2265
:103FC0002046FFF791FC94F82330052B7FF4B8AD21
:103FD000A5E71C230093CDE90188F3B24A460521E9
:103FE0002046FFF7F9FC94F82330052B7FF4BBAD96
:103FF00095E71E230093CDE90188F3B24A460521D7
:104000002046FFF7E9FC94F82330052B7FF4BEAD82
:1040100085E71C230093CDE9018AF3B24A460521C6
:104020002046FFF7D9FC94F82330052B7FF4C2AD6E
:1040300075E71E230093CDE9018AF3B24A460521B4
:104040002046FFF7C9FC94F82330052B7FF4C6AD5A
:1040500065E700BF357E02087D540208A14C0208C6
:104060000C230093CDE9018AF3B24A46062120468B
:10407000FFF7B2FC94F82330052B7FF4C3AD4EE775
:104080000C230093CDE90188F3B24A46062120466D
:10409000FFF7A2FC94F82330052B7FF4C6AD3EE772
:1040A000CDE901BA3B7800934A465FFA88F30721CD
:1040B0002046FFF791FC94F82330052B7FF4CFAD19
:1040C0002DE70023CDF808A001933B7800934A46E2
:1040D0005FFA88F307212046FFF77EFC94F823302F
:1040E000052B7FF4D0AD1AE70C230093CDE90189AD
:1040F000F3B252460F212046FFF76EFC94F82330AE
:10410000052B7FF4DAAD0AE70C230093CDE9018893
:10411000F3B252460F212046FFF75EFC94F823309D
:10412000052B7FF4DDADFAE630230093CDE901895C
:10413000F3B2524609212046FFF74EFC94F8233093
:10414000052B7FF4E0ADEAE630230093CDE901884A
:10415000F3B2524609212046FFF73EFC94F8233083
:10416000052B7FF4E3ADDAE670B50446FFF784FC77
:1041700094F82330052B29D0002594F83F33EB40E9
:10418000DB07E8B215D40135082DF6D194F82330B9
:10419000052B1BD094F8203013B194F82230ABB922
:1041A0000B4B0C491B6898690368BDE870401B689D
:1041B000184703F087FB02460028E4D0112120466F
:1041C000FEF7CEFF94F82330052BDCD170BD00BF85
:1041D000605E012050F009082DE9F04F90F9213080
:1041E00089B00446002B00F00481012300F50C7512
:1041F00080F84133024600F50F712B462E46D06EF3
:10420000002859D0002384F8413394F94030642BBE
:104210005BD094F9BC30642B00F08D8094F9383178
:10422000642B00F08A80D4F830722FBB01A920469D
:104230002AF0DEF900B30C230593012306978DF8CD
:104240001830714B07936946BDF80430049704A8F1
:10425000ADF810308DF800702AF0A0FB9DF9001029
:1042600051B1022908DC38B1C9B27C2303FB0141FA
:104270006C3128462BF048FE94F841B3BBF1000F97
:104280005DD0E36E6367D4F8E830C4F8F030D4F85A
:104290006431C4F86C3194F8233003F1C30204EBA9
:1042A00082020021042B7CD852F8040B10610133E8
:1042B00042F8041CDBB2F5E753F8040B0028A1D147
:1042C0008B4202F17C029AD19FE7002066238DF891
:1042D00010307C2303FB004004A940302BF058FD34
:1042E00004A920462AF084F900289CD004238DF8E4
:1042F00018300023CDE90133039331230593694638
:1043000004A82AF04BFB059B28B108AA02EB830204
:10431000009942F8E01C0133332B0593EFD94DF09F
:104320005DF99DED031ADDED020A9DED010A66219E
:104330004DF012F977E70120C8E70220C6E7012710
:10434000A94655F8043B23B1AB600137042FF7D1E0
:1043500097E7AA46B8465FFA88F3022BF5D8DAF851
:10436000002055F8043C9A4205D104A95046CDF8E6
:1043700010B02BF0C9FD5AF8043B08F101020BB94B
:104380009046E8E704A906EB88000193CDF810B049
:104390002BF0BAFD019BAB6001A948462BF0B4FDA0
:1043A000D3E794F8413313B92046FEF7B5FD94F8EE
:1043B00022300BB3154B1B68986A036864215B6855
:1043C00098472046FFF77CF994F83E3003B9E3663E
:1043D00094F8BA300BB9C4F8E83094F836310BB918
:1043E000C4F86431FAF762FEFAF7CCFE0123A4F8B0
:1043F000403309B0BDE8F08F2046FFF7B5FE94F8D2
:104400002230002BE0D0D5E7A08B0A08605E0120A7
:10441000704700000120704701207047436898688A
:104420007047000010B5054B03600446C06A10B128
:1044300003685B689847204610BD00BF14F5090863
:10444000406803689B6A184733B46C46406884E848
:104450000C000368DD6A94E80C00AC4602B030BC86
:104460006047000010B50446FFF7DCFF2046FEF76A
:1044700061FC204610BD000040680AF08BBB0000C4
:10448000406801230AF086BB40680AF05FBB000069
:1044900040680A220AF004BB40680AF019BB000019
:1044A00090F8313013B1002101F028B970470000B5
:1044B00040680AF093BB000073B50446052500264A
:1044C000E06A8DF8076003680DF10702DB680121DF
:1044D000984778B19DF807300C2B09D0102B05D0E8
:1044E000092B07D184F8333002B070BD1523F9E7EA
:1044F0001423F7E7013DE3D12846F5E710B4C06A7D
:1045000003681C690822A44601235DF8044B31218D
:104510006047000010B4C06A03681C690122A44609
:1045200000235DF8044B322160470000F7B50446D4
:10453000C06A03685B6998470546002871D0E06A45
:1045400003685B69984703689B689847E06A03685B
:104550009B69984760B9344B34491B689869036874
:104560001B6898472B682846DB689847002655E06B
:104570002046FFF7CFFF0028F4D02046FFF79CFF2E
:104580000028EFD0E06A03680121DB6A98472046E3
:10459000FFF7B4FF30B9244B25491B6898690368BD
:1045A0001B68DEE7E06A0368DB69984730B91E4B99
:1045B00020491B68986903681B68D2E7E06A94F891
:1045C0003310012784F8317003685B6A9847E06A0A
:1045D00003689B6A98470146204601F0F1F80646B9
:1045E0000028BFD094F830301BB13946204601F086
:1045F000F7F894F83210204601F018F92B68284695
:10460000DB689847E06A009403681D6A0A4B0193CF
:1046100002AB13E90C0042F21071A847304603B018
:10462000F0BD0646FAE700BF605E012080F409088D
:10463000A6F40908C5F409082D47020870B500253D
:1046400086B0CDE9005500230446C06A8DF80850B5
:1046500005930393049303686A469E681021092317
:10466000B047A0B19DF8003013F0010615D194F8C1
:1046700034300133DBB2052B84F8343007D12046C7
:10468000FFF748FF2046FFF739FF84F83460E06AFF
:1046900003681B6B984706B070BD9DF8083084F81E
:1046A00034501B07F3D4BDF901309FED1E6A06EEAE
:1046B000903ABDF9033007EE103ABDF90530F8EE37
:1046C000E66A07EE903ACDED036AF0EEE66AB8EEE0
:1046D000C77AF8EEE77AF4EEC66AF1EE10FA8DEDDD
:1046E000047ACDED057A0DD5B0EEC77AB4EEC67A70
:1046F000F1EE10FA06D5F0EEE77AF4EEC67AF1EEB6
:1047000010FAC4D49FED080A03A810F0E9F9B2EE3C
:10471000040A03A810F0E4F90A2203A9204601F0D4
:10472000EBF8B4E7000000349A99193EFFF786BF12
:1047300010B5044B044640F8043BFFF7CBF8204685
:1047400010BD00BF2CF5090810B50446FFF7F0FFB7
:104750002046FEF7EFFA204610BD0000F7B50368CB
:104760000F4616461BB90024204603B0F0BD0024B6
:10477000046008200193FEF7D5FA054620B1124BDC
:104780000360019B4360019401A8FFF7A3F8002D8B
:10479000E9D03820FEF7C6FA04460028E3D000F03E
:1047A000ADFE0A4BE562236084F8307084F8326015
:1047B0002046FFF7BBFE05460028D5D123682046DA
:1047C0005B6898472C46CFE72CF5090814F50908D3
:1047D0002DE9F74F046806460D4690469946002C91
:1047E0006CD00B68002B49D0236820469B6A984701
:1047F00003689B689847012328680DEB030200219A
:104800000AF0C8F998B39DF80130EA2B2FD1DFF8F0
:10481000F0B04FF0060A28680023802206210AF033
:1048200095F920B3DBF80070B86A03680A215B6869
:104830009847002328681A4606210AF087F9B0B184
:10484000B86A03680A215B689847012328680DEB62
:10485000030206210AF09EF948B19DF8014014F0C8
:1048600040042FD00AF1FF3A1AF0FF0AD3D1306882
:1048700003689B6A98470368DB68984700241DE03B
:10488000022223460F2128680AF060F9B86A0368FB
:1048900001215B689847306803689B6A9847036802
:1048A000DB689847336834604A46414601A8019363
:1048B000FFF754FF044601A8FFF70CF8204603B0A9
:1048C000BDE8F08F224623460F2128680AF03EF902
:1048D000B86A036801215B68984702232146306863
:1048E0000DEB03020AF056F904460028C8D0B86957
:1048F000024903681B689847B9E700BFECF4090850
:10490000605E0120002100F0F9BE000070B5044691
:104910008CB00426013E76B2731C4AD0E06A15239F
:104920006A465D210AF036F90028F3D0E06A1523C3
:1049300006AA5D210AF02EF905460028EAD01522C4
:1049400006A9684671F0A6F80028E3D19DF800306A
:1049500084F830309DF8073084F832309DF81430F8
:1049600084F83C309DF813309DF8102084F83D30D9
:104970009DF80F3043EA0223E3879DF8013084F865
:1049800031309DF8083084F83330039B9DF80C20BB
:10499000C3F30F23A3869DF80B3043EA0223E3867B
:1049A000049BC3F30F232387019BC3F30F23638768
:1049B00007E0054B05491B68986903681B68984721
:1049C000002528460CB070BD605E012060F5090826
:1049D0002DE9FF4104460023C06A8DF807300368C3
:1049E000DFF850819B6A984703689B689847E06AA4
:1049F00003680A21DB6C9847E06A0A2204210AF066
:104A00004FF80425013D6DB26B1C32D000234B21C1
:104A1000E06A82220AF09AF8D8F800600746B06A85
:104A2000036802215B689847002FEBD001231A46E8
:104A30004B21E06A0AF08AF80746B06A036802214F
:104A40005B689847002FDDD0E06A01230DF1070273
:104A500040210AF09FF80028D4D09DF80720322A80
:104A600010D0002DCED1B069304903681D683223C3
:104A7000A847E06A03689B6A98470368DB68984721
:104A800000254EE02046FFF741FF0028F1D0E06A04
:104A90000123172251210AF059F80028E9D05222A7
:104AA000E06A012311460AF051F80028E1D0E06ADB
:104AB000012338224C210AF049F80028D9D0E06AB5
:104AC00003689B6A98470368DB689847E06A05219A
:104AD00009F0FEFFE36A2046996800F071FE054682
:104AE000F8B194F84410204600F0A0FE94F8453048
:104AF0001BB10121204600F073FEE06A0368022129
:104B0000DB6C9847E06A02940368DE6A084B039303
:104B100004AB13E90C0044F21B11B0474EF0BAFF8E
:104B20002064284604B0BDE8F08100BF88F509087C
:104B30009D4C0208605E012070B5C58F90F93D6004
:104B4000AD03B5FBF2F2A2F5804404FB04F2D511EB
:104B500090F83C200498D201624306FB05225212D1
:104B6000A03002F58012424312134A43DB0003EBEC
:104B7000623000B270BD000010B5848E53005C43FB
:104B8000B0F93A30C91AC38FD31AB0F93820B0F946
:104B90003600534304F500449B10C3EBC13300EBD4
:104BA0002440044993FBF0F04FF400420DF006FF5F
:104BB00000B210BD0080FFFF10B52DED028B8AB052
:104BC00004460823C06A05AA422109F0E3FF18B190
:104BD000BDF81A20D30719D4E06A09F0FFFF4EF0A0
:104BE00059FF236CC31AFA2B0CD9206400238222AC
:104BF0004B21E06A09F0AAFF0123E06A1A464B2123
:104C000009F0A4FF0AB0BDEC028B10BDBDF9141071
:104C100094F932300093920894F930300392C9101D
:104C20002046FFF789FFBDF9161094F93330039A37
:104C3000009308EE900A94F93130C9102046FFF72E
:104C40007BFFBDF91810039A491008EE100A2046A0
:104C5000FFF792FF07EE900AF8EEE88AF8EEE77A9F
:104C6000B8EEC88AB3EE000A07A8CDED097ACDEDFB
:104C7000078A8DED088A0FF047FFB2EE040A07A8F5
:104C80000FF02EFF4EF006FF0A22206407A92046EF
:104C900000F032FEE06A09F0A1FFB3E7FFF78CBF36
:104CA000F7B503680D4616461BB90024204603B02D
:104CB000F0BD0027076048200193FEF733F8044653
:104CC00050B100F01BFC0D4B2360019BE362019788
:104CD00084F8446084F8455001A8FEF7FBFD002CE1
:104CE000E3D02046FFF774FE05460028DED1236896
:104CF00020465B6898472C46D8E700BFC0F50908F6
:104D000010B5044B044640F82C3BFEF7E3FD20466B
:104D100010BD00BFC0F5090810B50446FFF7F0FF4D
:104D20002046FEF707F8204610BD0000002100F0E5
:104D3000E5BC0000F8B504460D4617461E4600F0D7
:104D4000DDFB094B23602B68E362002200232A600D
:104D500084F8307084F831606365A365E365236689
:104D60006366A3662046F8BDD8F50908F8B51C4669
:104D700009331646DB086A46A2EBC30300AF9D4623
:104D8000C06AA31C6A4609F005FF054628B1224601
:104D90000DF10201304670F08DFE2846BD46F8BD8B
:104DA0002DE9F34106460F4614464EF073FE114BB3
:104DB000D3F800800546D8F82800036801215B6815
:104DC000984701230DF1070207213046FFF7CEFF78
:104DD00060B19DF80730DA0702D4B7EB531F05D056
:104DE0004EF058FE431BA342E5D3002002B0BDE8BD
:104DF000F08100BF605E01202DE9F041DFF86082A4
:104E000092B0044602AF002646F02002E06A00237A
:104E1000D2B2502109F09AFE002800F00C8103253F
:104E2000013D6DB26A1C00F00681D8F80030986A26
:104E300003684FF496719B68984701230DF10602B1
:104E400055212046FFF792FF002800F0F4809DF8DE
:104E5000063013F0E00F40F0EE80DB07E0D50223D0
:104E60000DF1060252212046FFF780FF002800F0D6
:104E7000E280BDF8063001365BBA202E27F8023BEF
:104E8000C2D1BDF824309DF826109FED6D7ADFED7C
:104E90006D6A9FED6D6A43F30B0207EE902A1B09C2
:104EA00003F47063BDF82620F8EEE77A0B4343F372
:104EB0000B03C4ED0D7A07EE903A02F470639DF88F
:104EC0002820F8EEE77A134343F30B03C4ED0E7A80
:104ED00007EE903A9DF92230F8EEE77AC4ED0F7AAA
:104EE00007EE903A9DF92930F8EEE77A67EE877A77
:104EF00007EE103AB8EEC77A9DF92A30C4ED107A61
:104F000027EE267ADFED517A84ED117A07EE103A1A
:104F1000B8EEC77A9DF92B30E7EE267AC4ED127A07
:104F200007EE903AF8EEE77A9DF9233067EEA67A1D
:104F3000DFED476AC4ED137A07EE903A9DF92C3005
:104F400007EE103AB8EEC77A9DF92E3027EE267A92
:104F5000F8EEE77A84ED157A67EE867A07EE103A76
:104F60009DF93030C4ED147A07EE903AF8EEE77A06
:104F70009DF92D3067EEA67AB8EEC77AC4ED177AA0
:104F800027EE267A07EE903A84ED167AF8EEE77A65
:104F90009FED307A9DF92F3067EE877AC4ED187A4D
:104FA00007EE903A9DF93130F8EEE77A06EE903A46
:104FB00067EE877AF8EEE66AC4ED197ADFED267AB5
:104FC000BDF93830E6EE877A07EE103A9DF93230B7
:104FD000C4ED1A7AB8EEC77AF3EE077AE7EE067AEE
:104FE00007EE103ADFED1D6AC4ED1B7AB8EEC77A02
:104FF00027EE267A84ED1C7A9DF9333007EE103ABD
:10500000B8EEC77A9DF9343027EE267A84ED1D7A02
:1050100007EE103A9DF9353007EE903AB8EEC77AB0
:10502000F8EEE77A27EE267A67EEA67A84ED1E7A06
:10503000C4ED1F7A00E0002012B0BDE8F08100BF8F
:10504000CDCC4C3E0000803B0000003B0AD7233C07
:105050000000003D0000803817B7D1B80AD7A33A46
:10506000605E012073B501230E460DF10702062193
:105070000446FFF77BFE18B90025284602B070BD34
:105080009DF80730013B012B0CD80023E06A1A463B
:10509000062109F05BFD0028EED006220021204603
:1050A000FFF77EFEE06A00233246062109F04EFD3E
:1050B00005460028E0D0262231462046FFF770FE44
:1050C000DBE7000013B501230DF1070207210446B9
:1050D000FFF74CFE10B9002002B010BD9DF807305C
:1050E0001B070CD50023E06A1A46062109F02EFDA5
:1050F0000028F0D0062200212046FFF751FEE06A8A
:1051000000230722062109F021FD0028E3D0132205
:1051100007212046FFF744FE0028DCD0E06A002388
:105120000522062109F012FD0028D4D017220521FE
:105130002046FFF735FE0028CDD001212046FFF79D
:1051400091FFC9E7F7B50446C06A544F03689B6AEC
:10515000984703689B689847E06A03680A21DB6CFC
:105160009847E06A0A22042109F09AFC0525013DCE
:105170006DB26B1C00F08980E06A0023B6227E21AC
:1051800009F0E4FC0028F2D03B68986A0368182113
:105190005B686E4698470123324600212046FFF7A0
:1051A000E5FD0028E3D09DF80030332BDFD1204609
:1051B000FFF722FE002868D0E06A002380225021F9
:1051C00009F0C4FC002860D02046FFF77BFF0028D0
:1051D0005BD0E06A002386222E2109F0B7FC00286C
:1051E00053D0E06A00232422042109F0AFFC0028F8
:1051F0004BD0E06A00230222062109F0A7FC002818
:1052000043D0142202212046FFF7CAFDE06A0023A2
:105210000722052109F09AFC002836D001212046FA
:10522000FFF720FF002830D0E06A03680321DB6C21
:105230009847E06A03689B6A98470368DB68984769
:10524000E06A172109F044FCE36A2046996800F0FF
:10525000B7FA0546B0B194F83110204600F0E6FAEE
:1052600094F830301BB10121204600F0B9FAE06A11
:105270000368DF6A0A4B0094019396E80C0042F23F
:105280001071B847284603B0F0BDE06A03689B6A16
:1052900098470368DB6898470025F3E7605E0120C4
:1052A0007954020810B586B00C236A4631210446B1
:1052B000FFF75CFD002800F0D5809DF80A309DF8CE
:1052C00009209FED697A9FED696ADFED694A94EDE7
:1052D000115A94ED1D4A94ED1E3A1B0403EB022370
:1052E0009DF80B2003EB02631B1207EE903AF8EED9
:1052F000E77AF7EE006AA7EE876A9DF801309DF81D
:105300000020D4ED147A94ED107A77EEA67A1B047F
:10531000A7EE867A03EB02239DF8022094ED0D6A36
:10532000D4ED157A03EB02631B12F0EE475A07EE39
:10533000103AB8EEC77A35EE265A27EE247A9DF851
:1053400004309DF80320A5EE076A1B0403EB02233B
:1053500094ED1B7A9DF8052094ED135A35EEC77A2B
:10536000D4ED185AA7EE876A03EB02631B12F0EE26
:10537000667AE7EE257A9DF80620D4ED125AC6EE3D
:10538000273A03A9204607EE903AF8EEE77A75EE41
:10539000A65A67EEA47A94ED0E6A9DF80730D4ED14
:1053A0001C4AA5EEA76A1B0403EB0223D4ED165A90
:1053B0009DF80820F0EE467A94ED196AE7EE257A1A
:1053C00003EB02631B12F0EE665AE7EE065A0A225E
:1053D00035EE265A87EEA56A07EE903ADFED255A9C
:1053E000F8EEE77A67EEA57AD4ED0F5AE5EE275A84
:1053F000D4ED177A94ED1A5AE7EE275AF0EE667A52
:10540000E7EE057AE4EEC46AC5EEA72AF0EE637A09
:10541000E4EEC67A94ED1F7A87EEA65AF0EE467A4D
:10542000E4EE637AC7EEA65AF0EE437AD4EE077A3A
:10543000A4EEC37A26EE476AB2EE047AA7EEA36A18
:1054400025EE075AC6EE267A65EE875A77EEA27ADF
:105450008DED035A67EE877ACDED045ACDED057ACE
:1054600000F04AFA06B010BD5B9E803A85EBCBC1D6
:1054700047ABE73BF61BEB3BFFF714BF30B51346DA
:10548000026885B00D461AB90024204605B030BD2B
:1054900000210160802001930392FDF743FC044644
:1054A00020B1019B2A4603A9FFF744FC03A8FEF79D
:1054B00011FA002CE8D02046FFF744FE05460028EC
:1054C000E3D1236820465B6898472C46DDE700005F
:1054D00010B5044B044640F82C3BFEF7FBF9204680
:1054E00010BD00BFD8F5090810B50446FFF7F0FF5E
:1054F0002046FDF71FFC204610BD0000064B10B5EE
:1055000003600446FEF7CCF9A06004F10C004DF0F6
:105510001FFC204610BD00BFF0F5090873B5054615
:105520007C23AC682E7903FB0643C6EB461604EBDE
:105530008604084693F8A41001900FF067FB94F9D5
:105540003C3001983BB9AB6893F8251002B0BDE838
:1055500070400FF05BBB94F84010F7E737B58468F4
:10556000057901917C2303FB054595F83F3004EB59
:105570008304D4F84C325BB14EF08CFAC5F89C0031
:105580000199D4F84C0203B0BDE8304003F0F8BDF7
:1055900003B030BD2DE9F04F90F804A08768CAEB46
:1055A0004A144FEA840806460D4607F13C0B08F101
:1055B00008018BB0594428460FF05EFA3179B06883
:1055C0000BEB8404FEF712F938B17C2303FB0A735A
:1055D00093ED1A0A28460FF083FA7C2303FB0A7323
:1055E00093ED146ADFED3A7AD3ED156AB0EEC67A20
:1055F000B4EEE77AF1EE10FA0FD5B0EEE67AB4EE3B
:10560000E77AF1EE10FA08D594ED077AB0EEC77A92
:10561000B4EEE77AF1EE10FA1BD47C2303FB0A7395
:10562000D86D196E5A6E9B6D02900391049007918C
:1056300001A829468DED016ACDED056A0692089212
:1056400009930DF077FB85ED000AC5ED010A85EDA4
:10565000021A7C2303FB0A770023C7F88C30C7F8B3
:105660008830C7F88430B06890F95C3208F13C09A2
:1056700008F14808D944D8446BB133795BB9414645
:1056800000F5167004F034FA414628460BB0BDE828
:10569000F04F0FF0F1B990F93430012B0BD190EDB0
:1056A0000E0A48460FF0C8F984ED120AC4ED130A39
:1056B00084ED141AE8E7022BE6D1FCF719FF00226B
:1056C00001A9FCF715FC0028DED09DED010AE8E7F2
:1056D0000000003410B5037984687C2202FB034487
:1056E00007C904F1900383E807004EF0D3F9C4F82A
:1056F0009C004EF0C5F9C4F8A00010BDF0B50546F9
:1057000085B0A6220E4600F10C0103A809F094FC16
:10571000AC682F797C2303FB0743D3F8B42022B96C
:1057200003A809F0ABFC05B0F0BDBEB196ED007A60
:10573000D3ED2A7A67EE877AC3ED2A7A96ED017A5D
:10574000D3ED2B7A67EE877AC3ED2B7A96ED027A4A
:10575000D3ED2C7A67EE877AC3ED2C7A7C2607EEA0
:10576000902A06FB0741A831B8EE670A0846019166
:105770000FF0CAF901992846FFF7ACFF06FB074373
:105780000022C3F8B020C3F8AC20C3F8A820002240
:10579000C3F8B420C4E7000073B5044680682379D9
:1057A00001917C2606FB03000D466C3001A92AF00E
:1057B0008BFBA368227906FB02331D6702B070BD24
:1057C00070B5021D044680680E46FDF7F5FB0546E0
:1057D00018B131462046FFF7DFFF284670BD0000B4
:1057E00007B5826803797C2000FB032090F93C0018
:1057F00002280BD002F13C00C3EB43138DF80710D5
:1058000000EB83000DF107012AF0B8FA03B05DF850
:1058100004FB0000836802797C2101FB023393F9C9
:105820003C00003818BF01207047000083680279EF
:105830007C2000FB023383F8A4107047F8B50546BE
:1058400008460F460FF0BEF910B100242046F8BDFF
:1058500038460FF09DF904460028F6D1AB6893F95D
:1058600034637EB138460FF0E5FC95ED097ADFED43
:105870001F7AF0EEC76AF4EEE76AF1EE10FA03D58C
:1058800085ED090A0124E1E777EE407A30EE076AF8
:10589000F0EEE77AC7EE866AF6B207EE906A9FED01
:1058A000146AF8EE677A26EE866AF4EEC67AF1EEAE
:1058B00010FA48BFB2EE046ADFED0E7A45BFAB6A5C
:1058C00066EE866AB0EE676A87EEA66A46BF013367
:1058D000AB620124F7EE007A77EEC67A20EE060A74
:1058E000A7EE270A85ED090AB0E700BF00000034E3
:1058F00000004843CDCCCC3D2DE9F74304460E468D
:105900001746FFF70BFE31462046FFF727FE3146CC
:105910002046FFF73FFE31462046FFF78FFF30B3AA
:1059200004F10C01992201A809F086FBA56894F8FE
:1059300004804FF07C0909FB0854A8343146204606
:105940000FF09AF809FB0851D1F8B4300133C1F8CF
:10595000B4304FB1BB4207D35B08C1F8B430B0EEEE
:10596000000A20460FF0D0F801A809F087FB03B029
:10597000BDE8F08310B50446FDF7B8FBC0B23C3477
:10598000C0EB401004EB800010BD0000F8B50A4EDB
:10599000044600F5167704F5137555F8040B08B1A5
:1059A00003F022FFBD42F8D13368986A03680121F1
:1059B0005B689847EFE700BF605E012008B5FFF71E
:1059C000E5FF0000F0B5144E00EB81077378044644
:1059D000D7F84C026FF3410387B00D467370C8B11E
:1059E00002F0F0FA68B1737843F0100373702C443E
:1059F0000023A372D7F84C0207B0BDE8F04002F0D4
:105A000065BAD7F84C12684602F00CFB009B012BDC
:105A1000EDD1E8E707B0F0BD2C5F012070B5064678
:105A20000D46002445FA04F3DB07E1B202D5304607
:105A3000FFF7C8FF0134032CF4D170BDFF21FFF73D
:105A4000EDBF000030B500F5137587B000F5167492
:105A500055F8041B21B9A542FAD1002007B030BD8A
:105A6000684602F0DFFA009B013B022BF3D80120CD
:105A7000F4E700002DE9F0472DED028B88B00446D5
:105A80000D469046B0EE408AFDF7F8FD30B900268D
:105A9000304608B0BDEC028BBDE8F08729462046B1
:105AA000FDF766FC06460028F1D004EB8507D7F821
:105AB0003C22D7F830329A4206D037F0B7F95C4A28
:105AC000032132F081F8E2E7D7F84C3283B94FF482
:105AD0009870FDF727F9814608B102F089FFC7F8F1
:105AE0004C92B9F1000F03D137F0A0F9514AE7E722
:105AF000B4F84A32D90711D505F0E8FD90F808232B
:105B000090F8C43232B9B02202FB030090F8A13001
:105B1000012B03D837F08AF9474AD1E72046FFF72F
:105B200091FF20B9454A537843F00203537094F92A
:105B3000353053B329462046FFF71CFF90F900305B
:105B4000002B53D029462046FFF714FF90F804900D
:105B5000B9F12B0F19D829462046D7F84CA2FFF7E8
:105B600009FF94F9353090F90020022BD4BF0021B1
:105B70000121012BD4BF00230123003A009118BF5B
:105B800001224946504602F0B5F9631900229A7283
:105B900075B3D4EDC10AB4F84822D7F84C0270EEC0
:105BA000A00A2B46B0EE480A414602F0C3F994F829
:105BB0003E33002B31D1224A069412680127E77345
:105BC000906A0268156D1F4A0792029309224FF4EA
:105BD0000063CDE9003208AA12E906001A4BA84773
:105BE000C8B937F023F9194A02216AE79946B2E7A2
:105BF00029462046FFF7BEFE90F90030002BC8D0A2
:105C0000D4EDC10AB4F84822D4F84C022B46B0EEC9
:105C1000480A4146C9E784F83E7300230DF1170195
:105C200004F124008DF817302AF0B2F830E700BFF5
:105C300000F6090832F6090855F609082C5F01201C
:105C4000605E0120BD59020873F609087EF6090856
:105C50002DE9F0412DED028B002443739DF8203097
:105C6000837305460F469046B0EE408A264647FAB3
:105C700004F3DB07E1B210D5B0EE480A42462846ED
:105C8000FFF7F8FE064640B939462846FFF7C6FE3C
:105C9000BDEC028B3046BDE8F0810134032CE6D127
:105CA000F6E70000F8B500242DED028B05460F46FF
:105CB000B0EE408A427383732646E1B2B0EE480AE2
:105CC0003A462846FFF7D6FE0134002818BF06469C
:105CD000032CF2D1BDEC028B3046F8BDF0B500EBE1
:105CE00081030D46D3F84C129BB0044611B9002035
:105CF0001BB0F0BD0BA802F079F96319987A00285F
:105D0000F6D10B9A002A48D0042AF0D101229A72C7
:105D10000DAA07CA02AB83E8070010AA07CA05AF9D
:105D200087E8070013AA07CA9DED180A08AE86E89F
:105D300007001A46294620468DED010AFDF7BCFAF8
:105D40003A4629462046FDF763FA32462946204660
:105D5000FDF770FA9DED010A29462046FDF77CFA11
:105D60009DF8643083B129462046FFF703FE90F981
:105D700000304BB194F93530012B05DD9DF85D20E5
:105D800029462046FDF7B0FA2046FFF75BFE20B912
:105D9000034A537843F0040353700120A8E700BF7F
:105DA0002C5F01202DE9F0410546884600F5137768
:105DB0000024012657F8043BE1B26BB148FA04F322
:105DC000DB0709D52846FFF789FF002857F8040CA0
:105DD00008BF002602F07AF80134032CEAD13046DD
:105DE000BDE8F0812E4B2DE9F04F1F68FB6A93F858
:105DF0009C8087B00446B8F1000F38D1DFF8A8A026
:105E000000F5137600F1030B054656F8040BA5EBDD
:105E100004095FFA89F9E8B102F0C0F828B19AF8EC
:105E2000013043F008038AF8013056F8040C02F000
:105E3000C9F8F8B9637B6BB1AB7A5BB956F8041C4F
:105E4000684602F0EFF8009B042B03D14946204638
:105E5000FFF744FF01355D45D7D1124B204683F84B
:105E60001280FFF7EFFD054630B10123237407B020
:105E7000BDE8F08F8046EDE7237C002BF7D0A37BB5
:105E8000002BF4D0B86A03684FF47A715B689847C6
:105E9000B86A03689B6B294607B0BDE8F04F184706
:105EA000605E01200D5F01202C5F0120F0B5002510
:105EB00087B000F513762C46012756F8041B41B134
:105EC000684602F0AFF8009B1BB107FA05F31C43CC
:105ED000E4B20135032DF0D1204607B0F0BD00003B
:105EE0002DE9F04F2DED028B03270E7C9FED348AB8
:105EF00091B005468846B946AC5D0134E4B2B4FBC6
:105F0000F9F303EB4303E41AE4B205EB8403D3F89B
:105F10004C1209B9AC554CE003A802F083F8DDF847
:105F20000CB00BF1FF33022BF4D8304630F024FCD8
:105F30008246304631F0EAFB00F11B039A4508D255
:105F4000304632F04BF8002011B0BDEC028BBDE8BA
:105F5000F08FAC55284698F810A0FFF7A7FFDDEDAD
:105F6000057A8DF83100FCEEE77A9DF810208DF867
:105F7000332017EE903A8DF8343006AB03CB1B88F4
:105F8000ADF83D305C221B23CDE90032CDF8350061
:105F9000CDF8391009AABF2150468DED098A8DED43
:105FA0000A8A8DED0B8A8DF830408DF832B030F0D2
:105FB0004DFC013F17F0FF079ED10120C4E700BF51
:105FC000000000002DE9F04F0F7CA1B00646884686
:105FD000032500EB070999F805400134E4B20323D7
:105FE000B4FBF3F303EB4303E41AE4B206EB8403DC
:105FF000D3F84C1211B989F805400AE011A801F054
:10600000F5FFDDF844A0BAF1030F08DCBAF1000F88
:10601000F1DA013D15F0FF05DDD1012012E0AAF112
:106020000402032AF5D8384630F0A6FB83463846EA
:1060300031F06CFB00F13602934506D2384631F060
:10604000CDFF002021B0BDE8F08F89F80540304633
:1060500098F810B0FFF72AFFDDF848E0CDF80CE023
:10606000DDF84CE0CDF810E0DDF850E0CDF814E0BC
:10607000DDF854E0CDF818E0DDF858E0CDF81CE08C
:10608000DDF85CE0CDF820E0DDF860E0CDF824E05C
:106090003219DDF864E01C9BCDF828E0DDF868E0FB
:1060A00092F80AC09DF874109DF87520CDF82CE088
:1060B0000E93DDF86CE01E9B8DF835008DF83C10DA
:1060C0008DF83D20CDF830E08DF834408DF836A0C5
:1060D0008DF837C02422CDF83E303623CDE900328A
:1060E000C0212C2303AA584630F0B0FB91E70000F2
:1060F0007FB58A8B0B464AF2B9518A4205465FD07A
:106100004AF2BA518A4274D04AF2B8518A420BD14B
:10611000474A1268D26A92F89C203AB136F086FE5D
:10612000444A052131F050FD042479E0D3ED007A92
:10613000F5EEC07AF1EE10FAF6D49FED3F7AF4EE68
:10614000C77AF1EE10FAEFDC93ED017ADFED3B6AEE
:106150001C6993ED030AB0EEC77AB4EEE67A93EDCC
:10616000027AFCEEE77AB0EEC77AF1EE10FAB4EEFE
:10617000E67A17EE903A54BF01260026F1EE10FAA7
:1061800054BF01220022003C18BF012413F0FF017C
:1061900010D18DED030A0292FCF7F6FF9DED030A84
:1061A000029A234631462846FFF77CFD0028BBD0E3
:1061B000002435E0134600943246FFF749FDF5E729
:1061C000D3ED007AF5EEC07AF1EE10FAACD49FED83
:1061D0001A7AF4EEC77AF1EE10FAA5DCFCEEE77A53
:1061E00017EE903A13F0FF0108BFFF21FFF7DAFD29
:1061F000DCE7D3ED007AF5EEC07AF1EE10FA93D435
:106200009FED0D7AF4EEC77AF1EE10FA8CDCFCEE1D
:10621000E77A17EE904A14F0FF0404D1FFF70EFC62
:10622000204604B070BD2146FFF7F8FBC0E700BF71
:10623000605E0120B0F6090800007F4300000034D2
:10624000F0B58BB00E4614460746FFF793FB54306B
:1062500007C884E8070031463846FFF78BFB90ED0E
:10626000057ADFED267AB0EEC77AB4EEE77AF1EE82
:1062700010FA054611D590ED067AB0EEC77AB4EE65
:10628000E77AF1EE10FA08D590ED077AB0EEC77A0A
:10629000B4EEE77AF1EE10FA24D431463846FFF72F
:1062A00069FB016A426A836AE869D5F814E0D5F8A7
:1062B00018C0099001A8CDF804E00291039204915E
:1062C000CDF814C00693079208930CF0DFFE98B146
:1062D000214601A80CF02EFD84ED000AC4ED010A50
:1062E00084ED021A31463846FFF744FB00F10801FD
